:020000040802F0
:1000000000000120A901020825790208C970020830
:10001000B9770208D10E0208ADAF02080000000057
:10002000000000000000000000000000658C0208D5
:10003000A911020800000000018002086D9E02085C
:10004000C3010208C3010208C3010208398402087F
:10005000C3010208C3010208C3010208C301020868
:10006000C3010208C3010208C3010208C301020858
:10007000C3010208C3010208C3010208C301020848
:10008000BD100208C9100208C301020800000000E8
:10009000000000000000000000000000C301020892
:1000A000C3010208C3010208C3010208C301020818
:1000B000C3010208919F0208C3010208C30102089C
:1000C000C3010208C3010208C3010208C3010208F8
:1000D000C3010208A9AA0208B5AA0208000000008C
:1000E000C3010208C3010208C301020800000000A6
:1000F000000000000000000000000000C301020832
:1001000000000000C3010208C3010208C301020885
:1001100000000000000000000000000000000000DF
:10012000C3010208D5100208E1100208C301020849
:10013000C3010208000000000000000000000000F1
:10014000000000000000000000000000C3010208E1
:10015000C3010208ED100208F9100208C1AA020842
:10016000C3010208C30102080000000000000000F3
:10017000000000000000000000000000000000007F
:1001800000000000C30102080000000000000000A1
:10019000C3010208DFF80CD000F0C0FC00480047A3
:1001A000C51E030800000120064880470648004796
:1001B000FEE7FEE7FEE7FEE7FEE7FEE7FEE7FEE717
:1001C000FEE7FEE7399F0208950102082DE9F05F7E
:1001D0000546002092469B468846064681464024B6
:1001E0001BE0284641464746224600F060F8534649
:1001F0005A46C01A914110D311461846224600F0C3
:1002000047F82D1A67EB01084F46224601200021CE
:1002100000F03EF817EB00094E41201EA4F1010446
:10022000DFDC484631462A464346BDE8F09F2DE9CB
:10023000F0410024061B254671F1000605DA012471
:100240000027D0EB070067EB0101161E73F10006D3
:1002500005DA0027D2EB0702012567EB0303FFF75E
:10026000B5FF86460E4617469C46AC4204D0002594
:10027000D0EB050E65EB010624B10020D2EB0007A0
:1002800060EB030C704631463A466346BDE8F081A8
:10029000202A04DB203A00FA02F100207047914046
:1002A000C2F1200320FA03F3194390407047202A3B
:1002B00004DB203A21FA02F00021704721FA02F310
:1002C000D040C2F120029140084319467047000017
:1002D0000649074A0868504343F23902104408604F
:1002E0004008704701490860704700005C0A002020
:1002F0006D4EC64110B5431A934209D2831888182F
:1003000003E010F8011D03F8011D521EF9D210BDC3
:1003100040EA01039B0703D009E008C9121F08C087
:10032000042AFAD203E011F8013B00F8013B521E07
:10033000F9D210BDD2B201E000F8012B491EFBD268
:1003400070470022F6E710B513460A4604461946E0
:10035000FFF7F0FF204610BD421E12F8013F002BB0
:10036000FBD111F8013B02F8013B002BF9D170479A
:1003700030B505462A460B4612F8010B13F8014B1F
:1003800008B1A042F8D01CB1002802D06D1CF1E7E2
:10039000284630BD10B5044604E00B7800F8013B58
:1003A00003B1491C521EF8D2204610BDCAB2401EED
:1003B00010F8011F8A4202D00029F9D100207047AD
:1003C000421C10F8011B0029FBD1801A704710B5A0
:1003D000002200E0521C835C8C5CA34201D1002B04
:1003E000F8D1D8B2E1B2401A10BD30B504460020B1
:1003F000034600E05B1C934203D2E05CCD5C401BF3
:10040000F8D030BD034611F8012B00F8012B002A6B
:10041000F9D11846704730B505460020034600E084
:100420005B1C934205D2EC5CC85C201A01D1002C05
:10043000F6D130BD10B5484304460BF097FE0028B6
:1004400005D00021002C02D0641E0155FAE710BD32
:1004500070B506460AF08AFE046805460A220021A5
:10046000304600F05DFA2C6070BD2DE9FE4F8046ED
:1004700081EA0300C00F0C46009021F0004123F0F8
:100480000045B8EB0200A94105D2404621469046FE
:100490001C460B46024623F00040104347D0270D70
:1004A000C7F30A00C3F30A510290401A0190402892
:1004B0006BDAC3F3130040F4801B0098924620B11E
:1004C0000023D2EB030A63EB0B0B01985946C0F1F2
:1004D00040025046FFF7DCFE06460D4650465946A0
:1004E000019A00F00BFA10EB08006141002487EA42
:1004F000115284EAE7731A4340D0009A62B3019A1A
:10050000012A4FEA075215DC001B61EB02014FF094
:10051000004202EA0752CDE90042001C41F5801179
:1005200032462B4600F043FA03B0BDE8F08F404658
:100530002146F9E7001B61EB0201001C41F5801325
:1005400000185B412018A2F5001747EB030140EAB1
:10055000D570B6196D4111E06D084FEA360645EACF
:10056000C0754FEA0752001B61EB0201001C41F508
:10057000801149084FEA30000019514132462B469C
:1005800003B0BDE8F04F00F003BA0098012240002C
:100590000023D0EB020263EBE073009821464FEAA0
:1005A000E074B8EB000061EB0401E9E783F000437D
:1005B0005BE781F0004158E72DE9FE4F81EA030433
:1005C00004F0004421F0004100944FF0000B23F0B0
:1005D000004350EA01045ED052EA03045BD0C3F347
:1005E0000A54C1F30A552C44A4F2F3340194A0FB3D
:1005F0000254C1F3130141F48011C3F3130343F414
:10060000801301FB024400FB034E840A970A44EA6C
:10061000815447EA8357A4FB076802958D0A05FBBE
:1006200007854FEA932C04FB0C542705029D4FEAE3
:10063000065847EA1637B5EB08056EEB070C870E30
:10064000920E47EA811742EA8312A7FB0201B6EB3A
:100650000B0164EB00042B0D43EA0C335E1844EBF2
:100660001C50DA465146E7FB0201C5F313044FEA7A
:100670000B3343EA14534FEA0432019C43EA060366
:10068000A4F10C040294009CCDE900B400F08FF9B1
:1006900003B0BDE8F08F00200146F9E72DE9F04DE9
:1006A00081EA030404F0004B21F0004514464FF0AA
:1006B000000A23F0004150EA050220D054EA01026A
:1006C0001DD0C5F30A570246C5F31303C1F3130047
:1006D000C1F30A5640F4801543F48013A7EB0608D3
:1006E000101BD64608F2FD3873EB050002D308F163
:1006F000010801E092185B41B8F1000F03DA002015
:100700000146BDE8F08D00204FF480110646844676
:100710000EE0171B73EB050705D3121B63EB0503F4
:1007200006434CEA010C49084FEA300092185B413D
:1007300050EA0107EDD152EA030012D082EA040028
:1007400083EA0501084305D0101BAB4106D2012204
:10075000002306E000224FF0004302E06FF00102A8
:1007600053101AEB06004CEB085110EB0A0041EB5A
:100770000B01BDE8F04D00F00BB90EB5C10F80EADA
:10078000E0700844CA07002140F233438DE80E00B0
:100790000A460B4600F00BF903B000BD0EB540F25F
:1007A000334102910021CDE900110A460B4600F0C9
:1007B000FEF803B000BD0EB540F2334202920022B3
:1007C000CDE90022134600F0F2F803B000BD70B589
:1007D000C1F30A5201F000450024C1F3130140F2B5
:1007E000FF3341F480119A4201DA002070BD40F2DB
:1007F00033439A42A2F2334203DC5242FFF757FDE1
:1008000000E090402C43F1D0404270BDC1F30A5249
:1008100010B5C1F3130140F2FF3341F480119A4245
:1008200001DA002010BD40F233439A42A2F2334273
:1008300003DC5242FFF73BFD10BD904010BDC1F3F9
:100840000A52C1F3130140F2FF3341F480119A427E
:1008500002DA00200146704740F233439A42A2F286
:10086000334202DC5242FFF722BDFFF711BD000008
:1008700030B5041E71F1000404DB4FF00044404227
:1008800064EB0101141E73F1000405DB1C464FF0FC
:100890000043524263EB04038B4208BF824230BDE7
:1008A00030B5041E71F1000404DB4FF000444042F7
:1008B00064EB0101141E73F1000405DB1C464FF0CC
:1008C0000043524263EB0403994208BF904230BD9B
:1008D00030B50B46014600202022012409E021FA10
:1008E00002F59D4205D303FA02F5491B04FA02F50D
:1008F0002844151EA2F10102F1DC30BD202A06DBDE
:10090000CB17203A41FA02F043EAE07306E041FADD
:1009100002F3D040C2F120029140084319467047CB
:100920002DE9F04791460F4680460446002614F80C
:10093000015B2DB100F004F90068405DC007F6D1FD
:100940002B2D02D02D2D18D0641E4A463946204644
:1009500000F0FAF827B13968A14201D1C7F8008048
:1009600071054FF002040BD54042002803DD0AF068
:10097000FDFB0460A007BDE8F08746F48066E4E76D
:100980000028F8DA0AF0F2FB04606FF00040F2E7AA
:1009900010B5141E73F1000408DA401C41F1000187
:1009A00092185B411A4301D120F0010010BD2DE9DE
:1009B000F04D92469B4611B1B1FA81F202E0B0FAD5
:1009C00080F220329046FFF763FC04460F4640EA6F
:1009D0000A0041EA0B0153465A46084313D0114618
:1009E00053EA010019D0C8F140025046FFF75FFCFE
:1009F00005460E46504659464246FFF749FC084315
:100A000005D0012004E020463946BDE8F08D0020E5
:100A1000054346EAE0762C4337430A986305E40A27
:100A2000A0EB08000022FD0A44EA47540A3002D530
:100A300000200146E9E7010510196941DDE9084593
:100A400000196941BDE8F04DA2E770B521F00043FF
:100A500003430CD0C1F30A550024D5EB040564EB25
:100A60000403D617AD1AB34102DB0020014670BD66
:100A7000201841EB025170BD2DE9F04D00231A46BC
:100A80001B1A8A4103DB00200146BDE8F08DC1F34B
:100A90000A52C1F3130141F480154FF0000BD10746
:100AA00002D100186D41521E0027044640F2FF118A
:100AB000384601EB620A3E468046024600204FF46B
:100AC0008011FFF7F4FBC2197141BB1846EB01001E
:100AD000B4EB030C75EB000C04D3E41A65EB0005D2
:100AE00017460E46241908F101006D41804634284E
:100AF000E3DDF91946EB0600091BA84103D24FF0CC
:100B0000FF32134601E0002213461BEB070046EBC1
:100B10000A51BDE8F04DFFF73BBF0000064C074D02
:100B200006E0E06840F0010394E8070098471034BD
:100B3000AC42F6D3FFF732FBE4BE030804BF030860
:100B40000048704724AF03082DE9F05F8246007823
:100B5000002715468B460AF10104B946302801D01A
:100B60009DB113E014F8010B0127782803D0582811
:100B700001D045B10AE00DB1102D07D10027102595
:100B800014F8010B02E0082500E00A250026B04613
:100B90000EE005FB080005FB06F1012701EB1046FE
:100BA0001FFA80F8B6F5803F00D3B94614F8010B60
:100BB000294600F018F80028EBDABBF1000F05D049
:100BC0000FB1641E00E05446CBF80040B9F1000FAD
:100BD00006D00AF0CBFA02210160C81EBDE8F09FE2
:100BE00048EA0640FAE73A2800D2303820F02002DE
:100BF000412A01D3A2F13700884201D34FF0FF30E0
:100C0000704770B58C1810F8015B15F0070301D11F
:100C100010F8013B2A1106D110F8012B03E010F85F
:100C2000016B01F8016B5B1EF9D12B0705D4002382
:100C3000521E0DD401F8013BFAE710F8013BCB1A24
:100C4000921C03E013F8015B01F8015B521EF9D519
:100C5000A142D8D3002070BD454910B54A6822F49E
:100C600040324A604A6843681A434A6001684A68E9
:100C700022F480724A6001684A68036942EA0322EA
:100C80004A6001684A6822F040724A6001684A6816
:100C900083681A434A6001688A6822F400628A60A5
:100CA00001688A68C3681A438A60816A6FF070625B
:100CB000D14201688A6822F070628A6001688A689D
:100CC0000CD0836A1A438A6001688A6822F0405215
:100CD0008A6001688A68C36A1A4301E022F04052C0
:100CE0008A6001688A6822F002028A6001688A6864
:100CF000836942EA43028A60016A002901684A68FE
:100D00000FD042F400624A6001684A6822F46042EF
:100D10004A6001684A68174C436A04EB43331A433C
:100D200001E022F400624A600168CA6A22F470029B
:100D3000CA620168CA6A838B0F4C04EB03531A43DF
:100D4000CA6201688A6822F400728A6001688A684F
:100D5000036B42EA43228A6001688A6822F4806257
:100D60008A6001688A68406942EA8020886010BD14
:100D70000023014000E0FFFF0000F0FF094910B52B
:100D80000020488100F004F906F0E8FA05F0D2FDF1
:100D900004F004FC06F0ECFA01F0AEFEBDE81040F1
:100DA00009F0A0BD0400002010B5002007F008FDE8
:100DB00014F036FE07F0CAFA00F0B4F808A004F008
:100DC0003FFD08F081F906F0E7FA06F0BDFA16F0EB
:100DD00021F901F01DFDBDE8104009F075BD0000CE
:100DE0000D0A7374617274696E67207178777A2066
:100DF0006170706C69636174696F6E0D0A00000048
:100E000010B5FFF7BBFFBDE8104019F01DB910B5D4
:100E100000F002F8002010BD70B5264807F006FB70
:100E20002549002007F0BCFE0021084607F0C4FD5C
:100E3000224C002102232246084607F051FD204D96
:100E400020232A460321002007F04AFD40232A469A
:100E50000121002007F044FD80232A4602210020C2
:100E600007F03EFD1749002009F070FF16490120E8
:100E700009F06CFF1549022009F068FF04222146A1
:100E8000002000F001FC01222146022000F0FCFBC2
:100E9000A61432462146012000F0F6FB0822214626
:100EA000002001F01FFE32462946012001F01AFE03
:100EB000002070BDA07B0020C07B00200004024009
:100EC00000000240547C0020D47C0020947C002050
:100ED000FEE710B500231A4603E0845C521C23444D
:100EE0009BB28A42F9D3D84380B210BD074910B5EE
:100EF000002048700649086007F01CFABDE8104061
:100F000000224FF48051034802F0ABBBE000002008
:100F1000980200200000024001484078704700001D
:100F20002801002000B587B01C216846FFF709FAA8
:100F300000208DF8010002208DF800000E4801907D
:100F40004FF480700290C0000490402005906946E4
:100F5000002009F00FFE0A480849C0F89015094919
:100F6000C0F89C150849C0F898150849C0F89415B0
:100F700005F076FB07B000BDF42900205D100208E3
:100F800054240020551002088B1002089910020802
:100F90007CB52F4C607858B1002501280CD0022870
:100FA00025D18DF8005001A9019509F0CFFD39E058
:100FB000BDE87C4005F0C6BA8DF8005001A90220BA
:100FC000019509F0C3FD4FF47A760AE09DF8000020
:100FD00003280DD06560334601226946019804F06C
:100FE0001EF96946002009F071FD0028EED07CBD95
:100FF000606840B105F08AFC6168401AC828EAD9E7
:1010000000206070E7E705F081FC6060E3E700BF67
:101010009DF8000003280CD0C4F808509DF800008B
:1010200009F0C6FF6946002009F050FD0028EFD006
:101030007CBDA06840B105F069FCA168401AC828D1
:10104000ECD900206070E9E705F060FCA060E5E7FE
:10105000280100200146002009F038BD0FB44FF4EC
:10106000007100B5ADF5017D83AB6846829A0AF048
:101070004FF86846FFF7A4F902466946002009F0D8
:10108000D7FE0DF5017D5DF814FB01B5012269461F
:10109000002009F0CDFE08BD10B50446FFF790F919
:1010A00021460246BDE81040002009F0C1BE000004
:1010B000014948700020704728010020014801F0D4
:1010C000DDBF0000D47D0020014801F0D7BF000043
:1010D000347E0020014801F0D1BF0000947E002042
:1010E000014801F0CBBF0000147D0020014801F051
:1010F000C5BF0000F47E0020014801F0BFBF000022
:10110000747D002001681823CAB2103AB2FBF3F2D2
:10111000054B6FF30901032A9B5CC36500D9091DC8
:1011200081650846704700008CA6030810B501468B
:1011300000208B698A6A4FF0C07453B1B3F5005F29
:1011400015D072B1012A0CD0022A0AD0032A09D183
:1011500004E01AB1012A06D0022A03D1C96AC901E2
:1011600000D5012010BDC96AA142FAD010BD002AE5
:10117000F7D0012AF2D0022AF3D0032AF3D010BD0F
:1011800030B50468256825F480252560046863600F
:101190008368402B036803D099600068C26030BD4B
:1011A0009A600068C16030BD704700002DE9F043CF
:1011B0008DB015460E4681462422534901A8FFF7FB
:1011C00099F8D9F80800514C332E416BA269D1F837
:1011D000008020D01CDC4D4901AB4FF0000789692D
:1011E000042E01EB410C03EB8C0128D007DCB6B1D7
:1011F000012E1ED0022E22D0032E36D11FE00E2E3D
:101200005BD00F2E74D0152E64D0322E2DD102E07B
:10121000343E072E29D872B3012A6ED155E0A7615A
:10122000E761DDE9012104F001F9E069401CE061BA
:1012300063E004F01DF9404605F022FB5DE0334A0F
:101240009269521C042E0DD08968022E11D00225FD
:1012500029421BD0C4E90627032A0DD32A490022BC
:1012600050391BE0097A4907F4D401200DB0BDE8DC
:10127000F0830125ECE723E002EB420153F8212043
:1012800003EB8101496804F0D1F836E0E069401CC5
:10129000E061032807D31C490022A0394FEA090066
:1012A00004F04AFC29E00E2000904B4642F21072F6
:1012B0000021404604F024FC1FE053F82C20E1E715
:1012C000D5E9000106F0E6FA17E0D5E9000106F0DD
:1012D000F7FA12E0D5E900010AAB0DA205F00AFD0C
:1012E00001280AD1DDE90A0106F0C4FA05E0FFE7AA
:1012F000002006F073FA012801D00020B6E7024969
:101300000022B0390548CBE7F4A50308F00100201E
:101310002B434349443A2025700D0A007879002078
:101320002DE9F84F074680683B4C0025426B0E269E
:101330000B46D2F80090A2784FF47A7A4FF4E13855
:1013400041F2883C032960D007DC4FF461216BB186
:10135000012B13D0022B06D116E0042B28D00E2B24
:101360003FD00F294CD00120BDE8F88F01206161EA
:1013700009F094FCA570E56025612AE004F078F896
:10138000484605F07DFA40E0012A0CD02561E1686D
:10139000491CE16003291CD36169414528D1012121
:1013A000A1701EA220E00120616109F077FC10E02D
:1013B0002069401CC4E90350052808D00A2808D930
:1013C0001B4900224FEA070004F0B6FB1DE041462E
:1013D000E9E73B46524600214846009604F090FB60
:1013E00013E0012A04D013A2614604F01FF80CE0B8
:1013F0000321002006F002FA0D4900222031E1E726
:10140000002006F0EBF9012801D00020ACE70849E4
:10141000002210390948D7E7F001002041542B4938
:1014200050523D3932313630303B26570D0A0000DC
:1014300054A50308415445300D0A00007879002076
:1014400038B504468068174B022915D003DC41B13A
:10145000012904D10DE003290ED00A2912D0012060
:1014600038BD5168196010A241F2883103F0DEFFE7
:1014700015E003F0FDFF12E000222046196804F099
:101480005BFB0CE000200090D2E900016B4609A252
:1014900005F030FC022802D1009806F037FA00204F
:1014A00038BD0000C001002041542B4353510D0AA8
:1014B000000000002B4543363030534353513A204F
:1014C00025642C252A0D0A001CB500230093C26B4D
:1014D00052680192C06B42685168044AC2E9011324
:1014E0006A46024904F028FB00201CBDC40100200C
:1014F00010B5044606F002FA012802D12046FFF793
:10150000E3FF4FF0FF3010BD10B50446806839B1DD
:1015100001290BD002290CD003290AD0012010BDCB
:1015200009A241F2883103F081FF0BE003F0A0FF34
:1015300008E00221084606F061F90022054920462C
:1015400004F0FAFA002010BD41542B4346554E3D9D
:10155000300D0A0094A5030800B5E1B04FF4C07146
:10156000684609F0D5FD6A4604A1032005F09AF803
:10157000684604F065F961B0002000BD25730000E5
:1015800010B594B000208DF8350002208DF834009D
:1015900023480E904FF420600F90224810900420B2
:1015A0001190102012900DA9012009F0E3FA4FF0DC
:1015B000FF3408BB1B48001D05F078F9E0B91A4854
:1015C00002901A4803903520049019480590194854
:1015D00006901948079019484FF4C061CDE90801F9
:1015E00000F5C060CDE90A010E4802A9001D0C906B
:1015F000134803F069FF10B1204614B010BD01215B
:101600000F48CDE900010F4B0FA21149064804F025
:1016100035FA1049044804F06BFA0020EDE70000A9
:10162000E0620020E4010020787900208CA2030809
:10163000A12202087124020821230208E06C002084
:10164000E078002034A403084543363030530000CE
:1016500024A5030859150208044910B5086918B1F2
:10166000898A012201F0FDFF002010BD6079002071
:10167000044910B5086918B1898A002201F0F1FF08
:10168000002010BD60790020034B43F8301003EBBD
:10169000C00082800020704760790020044910B5A6
:1016A000086818B18988002201F0DBFF002010BD16
:1016B00060790020044910B5086818B189880122B2
:1016C00001F0CFFF002010BD60790020054810B563
:1016D000006805F085F90448806BBDE8104005F00E
:1016E0007FB90000E8010020E078002010B5034633
:1016F0008068154C39B101290DD002290ED0092975
:1017000019D0012010BD0021616310A241F288317F
:1017100003F08CFE16E003F0ABFE13E0606B4FF0BD
:101720000002012804D00C49184604F005FA09E02B
:1017300009493031F8E7D2E90001034B07A23433FD
:1017400005F0D8FA002010BDF001002041542B43D1
:10175000474154543F0D0A00A4A503082B434741B9
:1017600054543A20256400002DE9F04194B00C4611
:10177000064620210AA8FEF7E4FDB56824225E494A
:10178000686B076801A8FEF7B5FD06F01FF88046F4
:1017900005225AA1FEF73FFEC0B1052259A14046DD
:1017A000FEF739FE90B1052258A14046FEF733FE00
:1017B00070B1052257A14046FEF72DFE30B105223B
:1017C00056A14046FEF727FE20B108E055A202E0F0
:1017D00056A200E057A220210AA805F07EFB0022B5
:1017E000DFF8588101A8032C46D005DC5CB1012C40
:1017F00018D0022C7ED11CE0042C1AD00E2C76D0EE
:101800000F2C77D16DE0C8F82C20C8F83020DDE926
:101810000121284603F00AFED8F83000401CC8F821
:1018200030005EE0284603F023FE384605F028F835
:1018300057E0042C04D0022C14D0032C1CD039E027
:10184000D8F82C1001EB410300EB83031B7A5B07F4
:1018500050D5491CC8E90B1203291FD32649002281
:10186000543931E0D8F82C1001EB410100EB810133
:10187000097AC90709D11DE0D8F82C1001EB410104
:1018800000EB8101097A890714D5C8F83020D8F80F
:101890002C10491CC8F82C100329DFD201EB4101A0
:1018A0000AAB50F8212000EB81004168284603F084
:1018B000BDFD16E0D8F83000401CC8F83000032801
:1018C00006D30D490022F439304604F035F908E01A
:1018D0000E200090334642F210720021384604F088
:1018E0000FF9002014B0BDE8F08103E0FFE7D8F85D
:1018F0002C10D3E70120F5E718A603083436303062
:1019000030000000343630303200000034363030E1
:1019100031000000343630303600000034363030CC
:1019200033000000434D4E4554000000554E494ED3
:101930004554000043544E4554000000F00100207F
:1019400010B5826891B1012910D00F2901D0012072
:1019500010BD07490B78012B03D0104600F02EFD77
:1019600004E000220A70034904F0E6F8002010BDEC
:10197000F0010020A4A5030808B50F2925D005DC37
:10198000F9B1012908D0042904D108E01A290BD0A3
:10199000272917D0012008BD07F0B8FF15E0002265
:1019A0000B4904F0C9F810E000200090D2E90001D2
:1019B0006B4608A205F09EF9012806D1009808F0B0
:1019C000E9F802E0094901200870002008BD000084
:1019D00034A503082B51495552433A2022636C6FBA
:1019E000736564222C25640D0A000000F0010020BC
:1019F00010B5806839B1012905D00F2901D0012027
:101A000010BD00F0BDFC002010BD000010B549B1B4
:101A1000012907D0042901D0012010BD002202496C
:101A200004F08AF8002010BD34A5030810B5044660
:101A3000806839B101290BD002290CD003290AD0C2
:101A4000012010BD09A241F2883103F0EFFC0BE048
:101A500003F00EFD08E00321022005F0CFFE002276
:101A60000549204604F068F8002010BD41542B437E
:101A700046554E3D310D0A00A4A5030810B5044695
:101A800029B101291DD00F2908D0012010BDFFF771
:101A900005FE0221002005F0B1FE12E0002005F055
:101AA0009DFE012803D10221002005F0A7FE0020A1
:101AB00005F09CFE012804D100220349204604F0D1
:101AC0003BF8002010BD000054A503082DE9F843A1
:101AD00084688046254D606B0E260068814631B1D2
:101AE000012914D00E2915D00120BDE8F883002764
:101AF000E7622169204688470028FAD0E7626F70C4
:101B0000FFF7CCFD434640F6B832009622E004F0E1
:101B1000B7FE29E068784FF47A7430B1012809D013
:101B200002280FD003281FD119E001206870FFF7A9
:101B3000C1FD03E002206870FFF78EFD4346224698
:101B4000009607E003206870FFF792FD43464FF4CC
:101B5000487200960021484603F0D2FF04E00022BC
:101B60000349404603F0E8FF0020BEE7F0010020F3
:101B700064A5030808B5C9B1012917D0042903D009
:101B8000142906D0012008BD0022094903F0D4FF22
:101B90000CE000200090D2E900016B4605A205F0A0
:101BA000A9F8012802D1009807F09AFF002008BD8B
:101BB00034A503082B51495552433A2022726563DC
:101BC00076222C256400000019B1012901D00120E2
:101BD000704700207047000070B5846805460529ED
:101BE0001DD2DFE801F0030D1111110005F0F2FD27
:101BF00003460CA241F28831204603F017FC0CE0AA
:101C0000204603F035FC08E0104605F031FE074899
:101C100000224168284603F08FFF002070BD01209C
:101C200070BD000025730D0A00000000280200208E
:101C30002DE9F84FD0F808C00346DFF82881DCF81A
:101C400034000F4601260568002098F8044041F250
:101C50008831072F58D005DC6FB1012F10D0022F2B
:101C600006D114E0082F56D00E2F5ED00F2F70D063
:101C70000120BDE8F88F88F80400C8F8240058E077
:101C8000604603F0F5FB284604F0FAFD67E0354FA7
:101C90004FF00E094FF4FA6A7A6A3F6A521C14B187
:101CA000012C12D05BE088F80500012F08D0052F29
:101CB00006D0C8F82420642A1ED900222A4917E039
:101CC00088F80460C8F8240039E088F80500012F7E
:101CD00004D0052F02D0C8E909200DE0D8F828006B
:101CE000401CC8F82800032806D31F490022803171
:101CF000184603F021FF32E0524600212846CDF875
:101D0000009003F0FDFE2AE00CBBD2E90001154B68
:101D100016A2203306E0012C21D1D2E90001114B9B
:101D200016A2203304F0E6FF19E014B1012C06D00E
:101D300015E0C8F8200088F8056014A204E0C8F88F
:101D4000200088F8056014A2604603F06FFB06E0EF
:101D5000FFE798F8050010B9604600F011FB00207D
:101D600087E70000F001002034A503082B4352450B
:101D7000473A20252A2C2564000000002B434752B7
:101D800045473A20252A2C256400000041542B4366
:101D90005245473F0D0A000041542B4347524547E7
:101DA0003F0D0A0070B5054680680F4C39B1012916
:101DB0000DD002290ED003290CD0012070BD13468E
:101DC000E2600AA243F6982103F030FB0AE003F038
:101DD0004FFB07E0E06807F0DDFE002208492846D7
:101DE00003F0AAFE002070BD6002002041542B5178
:101DF00049434C4F53453D25642C31300D0A0000BA
:101E0000D4A503082DE9FE43866880460025706B43
:101E1000364C0329D0F8009037D005DC59B10129A0
:101E20002CD0022904D15FE00E2958D0162938D0D1
:101E30000120BDE8FE831046626007F003FE0746FE
:101E4000606807F0EDFD0546606807F029FE01288F
:101E500012D027A08DE8A10026A241F28831304699
:101E6000636803F0E3FA0E20009043462A4A0021FB
:101E7000484603F045FE37E028A0EBE7304603F084
:101E8000F7FA484604F0FCFC2EE0606807F0A0FE7C
:101E9000A068401CA060032821D300222049A5602F
:101EA0001FE002A8019502950090D2E9000101AB64
:101EB0001CA204F01FFF022816D160680199884215
:101EC00012D1029941B107F083FEA068401CA060C6
:101ED000032804D3A56002E0A56007F093FE16492D
:101EE0000022404603F028FE0020A2E76002002006
:101EF0005544500041542B51494F50454E3D312CD3
:101F000025642C222573222C222573222C25752C46
:101F1000302C300D0A00000020BF02005443500056
:101F200024A503082B51494F50454E3A2025642CD7
:101F300025640D0A00000000D4A503087CB5054601
:101F40008068254C02291BD003DC41B1012904D152
:101F50000DE003290ED01B2918D001207CBD1346AB
:101F600022611EA241F2883103F060FA31E003F0F1
:101F70007FFA2EE0206907F0FBFD206907F00AFEDA
:101F800000221B49284603F0D7FD22E00020154619
:101F900000900190D5E900016B4616A204F0AAFE5C
:101FA000012803D0206907F0E3FD12E00098002823
:101FB000F8D0D5E9000101AB11A204F09BFE022884
:101FC000F0D1DDE90021206907F0B4FE206907F0B7
:101FD00055FE00207CBD00006002002041542B51C2
:101FE0004952443D25642C313530300D0A00000043
:101FF000D4A503082B514952443A2025640D0A0008
:102000002B514952443A20252A0D0A25650000002B
:10201000F8B52E4C064685686069032953D005DC67
:1020200061B101291DD0022906D14AE010291ED034
:1020300018292DD0192946D00120F8BD104662611B
:1020400007F010FD18B304F0CAFFA061F8B14068B2
:1020500000901FA241F288312846636903F0E6F937
:102060002FE00020A061284603F002FA29E003F0E7
:1020700085FA012803D1A06903C803F05BFCA069BD
:1020800044F62061D0E90023284603F0F9F918E06E
:1020900007F0E8FCA8B1A16904F079FF0B49626977
:1020A000491C0120885404F031FC0E4A616942F851
:1020B00021000C3242F8210000220B49304603F087
:1020C0003BFD0020F8BD07F065FDF5E7600200204C
:1020D00041542B514953454E443D25642C25750DE3
:1020E0000A000000A8790020D4A503082DE9F041DA
:1020F0000546002404F00AFC204607F0C3FC032830
:1021000021D0204607F0BEFC042824D0204607F04A
:10211000B9FC05281BD0204607F0D2FC01281FD0AF
:10212000641C032CE8DB1F4F03208046396A491CDE
:1021300091FBF0F200FB12140026204607F0A2FCEF
:10214000062812D022E00421204607F07FFE224616
:102150001549E86B15E0144922461039E86B10E088
:10216000114922461031E86B0BE0204607F07AFC5B
:1021700060B104F034FF48B10B493C622246203183
:10218000E86B03F0D9FC0020BDE8F081641C94FBEF
:10219000F8F108FB1144761C032ECEDB4FF0FF3024
:1021A000F2E70000600200205CA60308F8B583682F
:1021B000264D0E265A6B10291468EA7829D2DFE8DA
:1021C00001F00811181D2628282828282828352835
:1021D0002D380020E8701EA241F28831184603F025
:1021E00025F92BE0184603F043F9204604F048FB9C
:1021F00024E0034640F6B832009603E003464FF46D
:102200007A7200960021204603F07AFC16E0012A3B
:1022100001D00120F8BD0022104904E0012AFAD0C3
:102220000E490022103103F087FC07E00120E8701E
:1022300004E0002005F0D2FA012801D00020F8BD0A
:102240000649002240390648EDE70000F001002071
:1022500041542B4350494E3F0D0A000084A503080A
:102260007879002010B50446022005F0B7FA01285D
:1022700002D04FF0FF3010BD084A00231360E06B1E
:102280004168516018324968C2E9011303491A468E
:10229000183103F051FC002010BD0000280200207E
:1022A000012008F013BC000004480549406888423A
:1022B00001D101207047002070470000787900208C
:1022C000D4A5030805480649406804E0884201D1C6
:1022D0000120704740680028F8D1704778790020C5
:1022E000C4A5030810B50446022005F07FFA0128B2
:1022F00002D04FF0FF3010BD084A00231360E06B9E
:102300004168516028324968C2E9011303491A46FD
:10231000283103F011FC002010BD0000280200202D
:1023200070B50D4614461146284604F0C9FC012834
:102330000CD1285D50B924B1281910F8010C0A28D5
:102340000BD0294606A000BF03F09AFA2246294680
:10235000BDE87040012008F06BBD294604A0F3E7FA
:102360005B41542053656E645D2025730D0A0000A7
:102370005B41542053656E645D20257300000000AE
:1023800010B5044600F056F8002815D02046FFF797
:10239000AFF8002810D0204600F0B0F900280BD08C
:1023A0002046FFF75FFF002806D02046FFF79AFF80
:1023B000002801D04FF0FF3010BD000070B5054679
:1023C00004F0A4FA0446284600F034F8002817D098
:1023D0002846FFF78BFE002812D02846FFF788F822
:1023E00000280DD0104842F210728168611A9142A3
:1023F00007D9846000220D490D4803F09DFB0020A1
:1024000070BD284600F07AF90028F9D02846FFF779
:1024100029FF0028F4D02846FFF764FF0028EFD0FA
:102420004FF0FF3070BD0000F0010020E4A503086C
:102430007879002010B5002005F0D8F9012803D1E3
:102440000321002005F0DAF9002005F0C7F9012882
:1024500002D04FF0FF3010BD00220349034803F0C3
:102460006BFB002010BD000044A503087879002014
:102470002DE9F04F87B04FF0000604008DF8106092
:102480004FF0FF3712D0E06880B1606A70B17D4DC7
:10249000A06A4FF00A094FF001084FF0020A28B174
:1024A000D2E0E26804A92046904718B1384607B048
:1024B000BDE8F08FE06A636A9DF81020411CE1627C
:1024C0001A54E16A606A4654E06A072818D1072264
:1024D0006DA0616AFDF789FF20B985F8008001F0E1
:1024E000C5F8E860E06A07280AD1072268A0616A97
:1024F000FDF77BFF20B985F800A001F0B7F8E86090
:10250000E06A0A280AD10A2263A0616AFDF76DFF1A
:1025100020B90320287001F0A9F8E8602878012884
:1025200003D0022801D003280ED101F09FF8E968FA
:10253000401A40F2DC51884260D8287801280DD03A
:1025400002281DD003283CD0C0B20A2857D09DF8DD
:1025500010000D2858D00A2859D05CE051A1606ABB
:10256000FDF706FF5FEA000B6ED0029602AB4EA2AB
:10257000E16A606A04F0BEFB01286BD1029816E0A4
:1025800048A1606AFDF7F4FE5FEA000B5CD0686862
:10259000401C01D068680AE0039603AB45A2E16ADB
:1025A000606A04F0A7FB012854D10398686028B33F
:1025B000626AABEB02010844801CA86085F80090B9
:1025C00042E0059637A1606AFDF7D2FE019090B314
:1025D00001A8009005AB3AA2E16A606A04F08AFBA8
:1025E000052837D1606A0199081A05990844001D29
:1025F000A86085F80090E16A814225D12AE0E06A6E
:10260000A968884220D125E084F8308007E094F85A
:102610003000012807D094F83000022805D0E06A85
:10262000012811D10CE084F830A0E06A022803D020
:1026300084F830600EE007E0E66284F8306003E082
:10264000606A00783E2805D0D4E90A01401E814224
:10265000FFF427AFE16A606A04F032FB01280BD176
:10266000E06A28B1616A084410F8010C0A2806D013
:102670001AA0616A03F004F92E70002017E71BA06E
:10268000F8E70000D40100202B514952443A2000C1
:10269000434F4E4E454354002B514D5452454356E3
:1026A0003A2000000D0A00002B514952443A2025DF
:1026B00064000000434F4E4E454354202564000003
:1026C0002B514D54524543563A20252A2C252A2C6D
:1026D000252A2C25752C2565000000005B4154201F
:1026E000526563765D2025730D0A00005B4154201E
:1026F000526563765D2025730000000010B5044626
:1027000005F0AEF8012802D04FF0FF3010BD084AA6
:1027100000231360E06B4168516008324968C2E9E8
:10272000011303491A46083103F006FA002010BDD0
:10273000280200200FB4F8B504460D4600261CB947
:10274000701EF8BC5DF814FBE06A08B90020F8E7D9
:1027500009A80090E76A29462046009B089AB847D6
:102760000646002000903046EBE7F0B504460D46E3
:102770001E46002100270023214600BF10E042F83A
:10278000331002EBC300476002EBC3075B1C6868B1
:10279000D1F804C0604502D137600020F0BD49681F
:1027A0000029ECD1481EF9E72DE9F0410546002744
:1027B00000264FF6FF7000EA1547AEB208480468DD
:1027C00009E02088B84205D100223146204603F0B6
:1027D000EFF802E06469002CF3D100BFBDE8F0819E
:1027E000BC020020094910B502460020064B497979
:1027F00006E000BF33F81040944203D0401CC0B242
:102800008842F7D310BD0000940B00202800002060
:1028100010B5274C88B00122A189A06800F021FFE3
:10282000A1880122206800F01CFF0A2000F09CFD16
:10283000A1880022206800F014FF0A2000F094FD17
:10284000A1880122206800F00CFF00208DF8010013
:102850008DF80000A4F5006001904FF48060A4F5AD
:102860008061CDE90201049002206946059008F0DC
:1028700081F9B02104F1100004F0B2F910340DA276
:102880000A21601C04F029FB20620CA20A2104F139
:102890000B0004F022FB60620AA20A2104F1150079
:1028A00004F01BFB0949A0620120887008B010BD2C
:1028B000F434002024474E47474100002447504746
:1028C0005356000024474247535600003801002069
:1028D00070B594B00C46054628210AA8FDF731FDD5
:1028E00007AA00922846214601AB15A204F002FA7D
:1028F0004FF0FF36022819D1DDE9070104F091F904
:10290000C1B201980122007803E0019B9B5C584012
:10291000521C029B9342F8D8884207D105AB0BA208
:102920002146284604F0E6F90F2802D0304614B0BC
:1029300070BD0598FDF78CFD104908700020F6E782
:102940002425702A25700D0A0000000024252A2C59
:10295000252A2C252A2C252A2C252A2C252A2C25EB
:10296000702C252A2C252A2C252A2C252A2C252A90
:102970002C252A2C252A2C252A2A00003801002063
:102980002DE9F04196B00F46804628210CA8FDF7AE
:10299000D8FC05AD09A807AE0095CDE9016003ABF1
:1029A0002D4A3946404604F0A5F92C4C15281BD079
:1029B000CDE9005603AB2AA23946404604F09AF905
:1029C000112822D003AB34A239464046009504F0CA
:1029D00091F90D2829D003AB3AA23946404604F0BC
:1029E00089F909282AD032E0E088001DE0800398A8
:1029F000FDF72EFD05460598FDF72AFD05440798CD
:102A0000FDF726FD054409980BE0E088C01CE08036
:102A10000398FDF71DFD05460598FDF719FD0544D2
:102A20000798FDF715FD28440EE0E088801CE08043
:102A30000398FDF70DFD05460598F2E7E088401C78
:102A4000E0800398FDF704FDA1880844A08016B03B
:102A50000020BDE8F0810000BCB003083801002070
:102A600024252A2C252A2C252A2C252A2C252A2CDB
:102A7000252A2C252A2C25702C252A2C252A2C2584
:102A80002A2C25702C252A2C252A2C252A2C257029
:102A90002C252A2A0000000024252A2C252A2C2552
:102AA0002A2C252A2C252A2C252A2C252A2C25704F
:102AB0002C252A2C252A2C252A2C25702C252A2A3F
:102AC0000000000024252A2C252A2C252A2C252A22
:102AD0002C252A2C252A2C252A2C25702C252A2A1F
:102AE00000000000034B43F8301003EBC00082806D
:102AF00070470000F43400202DE9FE4300250295C4
:102B00008DF8005001A92846019508F01FF81A4CCD
:102B10004FF47A78194E4FF4007719E0FEF7FCF97C
:102B2000012805D1434601226946019802F077FB4E
:102B30009DF8000000F04CF8E0689DF8001031545A
:102B4000401CE060B84200D3E56003F0DFFE206186
:102B50006946022007F0BAFF02900028DED0E06844
:102B6000002806D003F0D2FE2169401A322800D98D
:102B7000E560BDE8FE83000038010020F42A002053
:102B8000124910B54870012806D0022808D005283F
:102B90000AD00A2818D10BE00C490E2229310AE08C
:102BA0000A490E22373106E008490E22453102E07B
:102BB00006490E225331022008F03AF90349152242
:102BC0001431022008F034F9002010BD3801002033
:102BD0002DE9F0414F4C002604F12C0523789BB1E0
:102BE000224602F11508D2F8AC10012B15D0022BA9
:102BF00031D0032B0FD14855D4F8AC10491CC4F880
:102C0000AC100A2834D082E0242804D1012121709C
:102C10007055C4F8AC10BDE8F0814855D4F8AC004C
:102C2000401CC4F8AC00226A9042F4D3611C2846D0
:102C3000FDF7DBFB022760B1364928460B31626A9B
:102C4000FDF7D3FB28B141462846A26AFDF7CDFB2C
:102C5000F0BB2770DFE74855D4F8AC10491CC4F826
:102C6000AC107F2953D20D28D5D103202070D2E794
:102C7000294F2A48B978B0F8700011B9797888429C
:102C800003D0BE70C0B2FFF77BFF41462846A26A60
:102C9000FDF7ABFB20B92846D4F8AC10FFF770FE67
:102CA000611C2846226AFDF7A0FB18BB2846D4F811
:102CB000AC10FFF70DFE1748D4F8AC102A300E54B4
:102CC000284607F07BFE39781548062912D200E025
:102CD0001DE0DFE801F00303070F0B07802100F080
:102CE000BCFC07E0F978C907F8D103E00122802194
:102CF00000F0B7FC03F00AFEB968401AB0F57A7F1D
:102D000005D303F003FEB860284614F0DDF9267001
:102D100081E7000004350020380100200E0D00205E
:102D20000004024070B5374A3749002041F820209E
:102D3000401CC0B21428F9D3354C3448A18B20F87C
:102D4000751F3449098881803049052074314872E3
:102D50000A200BF0D0FE4FF47A700BF0DDFE2B4909
:102D6000002274310C200BF0A2FF00210C200BF08C
:102D7000AFFF02200BF0FCFE274D00210F200BF0CF
:102D800048FE28422063F8D0206B411C37D0400415
:102D900034D54FF4814200210F200BF05AFF00215F
:102DA00010200BF036FE00F07F0117480022C438D7
:102DB0000BF05FFE144DC43D687A05281ED1022237
:102DC0001449681DFDF711FB002817D1A87CA5F157
:102DD00044016071D1F84510216505F113014200ED
:102DE0000D4601F15100FDF785FA60792946420050
:102DF00005484838FDF77EFA0420207070BD04F0C5
:102E0000A3FD0000FFFF0100F40B00206C0A00206E
:102E1000280000200001002000D0272478B50024DD
:102E2000009490F83C20012A19D0012280F83C201F
:102E30000A6807230568092A13D9EE680A3A02EBE3
:102E4000420293409E43EE600B788A680A3B03EB94
:102E500043039A400368DD682A43DA6010E00220E9
:102E600078BD2E6902EB420293409E432E610B789F
:102E70008A6803EB43039A4003681D692A431A6179
:102E80004A681F23072A13D205686E6B521E02EB95
:102E9000820293409E436E630B790A885B1E92B256
:102EA00003EB83039A4003685D6B2A435A6327E070
:102EB00005680D2A12D22E6BD21F02EB82029340BC
:102EC0009E432E630B790A88DB1F92B203EB8303C8
:102ED0009A4003681D6B2A431A6311E0EE6A0D3AAB
:102EE00002EB820293409E43EE620B790A880D3B0F
:102EF00092B203EB83039A400368DD6A2A43DA62E5
:102F0000164B0568144A9D4206D10D68122D03D157
:102F1000556845F48005556005689D4218D10B68D9
:102F2000102B01D0112B13D1536843F400035360CD
:102F3000096810290CD10A490A4A0968B1FBF2F163
:102F400001EB8101490000E0491E00910029FBD1FD
:102F500080F83C40002078BD002301400020014063
:102F60000000002040420F0070B504004FF0000543
:102F700003D0206C002610B107E0012070BD66640C
:102F800084F83C60204600F019F8206CC00610D48C
:102F9000206C20F4885040F0020020642046FDF7A9
:102FA0005BFE6664206C20F0020040F001002064AB
:102FB00000E0012584F83C60284670BD00B500683B
:102FC0000C4987B0884212D10B480021026842F4B4
:102FD00080720260006800F480700590012000900B
:102FE0000320CDE901016946044800F06DFA07B0FD
:102FF00000BD0000002001404438024000080240AB
:1030000090F83510022903D08021416501207047D6
:10301000052180F835100068016821F00101016088
:103020000020704770B5040025D094F835000228C0
:1030300020D02068016821F001010160206800258E
:10304000056020684560206885602068C56020684C
:1030500005612168212048612046FEF753F894F865
:103060005C203F2191408160656584F8355084F88B
:103070003450002070BD012070BD00002DE9F843E0
:1030800004464FF00009CDF8009063484FF4165104
:10309000A56D0068B0FBF1F72E6894F85C1008206D
:1030A00000FA01F131420FD021680A6852070BD5AE
:1030B0000A6822F004020A6094F85C108840A86054
:1030C000606D40F00100606594F85C104FF00108FD
:1030D00008FA01F0304208D021684969090604D590
:1030E000A860606D40F00200606594F85C100420F8
:1030F0008840304208D021680968890704D5A86053
:10310000606D40F00400606594F85C101020884009
:10311000304218D021680968090714D5A8602068D2
:103120000168490304D50068000308D5A16C07E0D5
:103130000168C90503D4016821F008010160216C10
:1031400009B12046884794F85C102020884030421E
:1031500031D021680968C9062DD5A86094F83500DA
:1031600005282068016806D0490347D50068000398
:103170001DD4616C1CE021F01601016020684169DA
:1031800021F080014161206C08B9A06C20B1206859
:10319000016821F00801016094F85C103F2088402C
:1031A000A86084F8349084F83580216D1FE0E16BCD
:1031B00009B120468847606D00282BD0606DC0079C
:1031C00014D0052084F835002068016821F0010141
:1031D00001600098401C0090B84203D82068006845
:1031E000C007F6D184F8349084F83580E16C00296A
:1031F00010D001B02046BDE8F04308470168C9057A
:10320000D5D4016821F01001016084F8349084F86D
:103210003580CCE7BDE8F883000000202DE9F041BF
:10322000044600F023FA06465CB1002584F83450C9
:10323000022084F835002068016821F00101016056
:103240000DE00120BDE8F08100F010FA801B052898
:1032500005D920206065032084F83500F2E7206856
:103260000068C007F0D12268116820480140D4E905
:1032700001031843D4E90336334318436369184301
:10328000A3691843E3691843236A18430843616A32
:10329000042903D1D4E90B131943084310602068B3
:1032A0004069666A20F0070130460E430127042872
:1032B0000CD1A06A0643E06A40B12046FDF736FF14
:1032C00020B14020606584F83570BAE72068466117
:1032D0002046FDF717FF94F85C203F219140816064
:1032E000656584F835700020ACE700003F8010F081
:1032F0002DE9F0410446866D90F834000025012840
:103300000DD0012084F8340094F835700020012F8E
:1033100007D084F8340002252846BDE8F081022059
:10332000FBE7022784F8357060652046FDF728FF2B
:1033300094F85C103F208840B0602068016841F03C
:10334000160101602068416941F080014161206CF3
:1033500020B12068016841F008010160206801681F
:1033600041F001010160D7E770B5044600F07EF935
:103370000546601C02D004480078044400F076F949
:10338000401BA042FAD370BDB002002007490020C4
:103390000A68002A09DA054A054B0C3A1360054B06
:1033A00013600968002900DA01207047103C0240D0
:1033B00023016745AB89EFCD2DE9F04FDFF8ECB085
:1033C00000224FF001094FF00F0A00BF09FA02F482
:1033D00001EA0403A34264D1066857000325BD40F7
:1033E000AE430660D60800EB8607D7F820C0560724
:1033F0004FEAD6680AFA08F62CEA060CC7F820C08D
:103400008668AE4386604668A6434660C468AC439F
:10341000C46022F003055D44D5F808689407270FBF
:103420000AFA07F4DFF888C02640604502D14FF061
:10343000000C1DE0DFF87CC0604502D14FF0010CAC
:1034400016E0DFF874C0604502D14FF0020C0FE0C7
:10345000DFF868C0604502D14FF0030C08E0DFF8E8
:1034600060C0604502D14FF0040C01E04FF0070C42
:103470000CFA07FCB44514D1D5F80868A643C5F882
:103480000868104C25689D432560241D25689D43D0
:103490002560241D25689D432560241D25689D43C6
:1034A0002560521C102A91D3BDE8F08F00300140F6
:1034B000000002400004024000080240000C0240EC
:1034C00000100240003C01402DE9F84FDFF860B1E8
:1034D00000224FF001084FF0030A4FF00F090BF1E3
:1034E000040E00BF0B6808FA02F42340A3426ED119
:1034F0004D68022D01D0122D0ED1D50800EB850CA0
:10350000DCF820505607F70E09FA07F6B5430E69A6
:10351000BE402E43CCF82060066855000F790AFAA9
:1035200005FC07F0030726EA0C06AF4037430760A7
:103530004E68012E05D0022E03D0112E01D0122E7E
:103540000ED18668CF6826EA0C06AF403743876005
:103550004668A6430C79C4F3001494403443446095
:10356000C6688C6826EA0C06AC403443C4604C68DC
:10357000E40056D52F4C256845F480452560246825
:1035800022F0030504F4804400942B4C2E19D6F845
:10359000084895072F0F09FA07F5AC43274DA842B5
:1035A00001D1002515E0264DA84201D1012510E0EA
:1035B000244DA84201D102250BE0234DA84201D1A0
:1035C000032506E0214DA84202D1042501E028E0B0
:1035D0000725BD402543C6F80858DBF800405D4686
:1035E0004E689C43F60300D51C432C60DEF8004077
:1035F00075464E689C43B60300D51C432C600C4DA9
:1036000008352C684E689C43F60200D51C432C609C
:10361000074D0C352C684E689C43B60200D51C4300
:103620002C60521C102AFFF45DAFBDE8F88F00003B
:10363000003C01404438024000300140000002409C
:103640000004024000080240000C0240001002404A
:103650000069084000D00120704742694A40426139
:1036600070470AB1816170470904FBE7014880682F
:1036700070470000B00200200248816802781144BF
:1036800081607047B00200200B4810B5016841F41A
:1036900000710160016841F480610160016841F4DA
:1036A00080710160032000F08BF8002000F006F824
:1036B00000F024F8002010BD003C024070B50D4D14
:1036C00004464FF47A712878B1FBF0F00A49096892
:1036D000B1FBF0F001F0F4F848B9102C07D2002249
:1036E0002146501E00F04CF800206C6070BD012097
:1036F00070BD0000B00200200000002010B50320C3
:1037000000F05EF8002211466FF00B0000F038F870
:10371000002211466FF00A0000F032F80022114634
:103720006FF0090000F02CF800221146501F00F045
:1037300027F800221146101F00F022F8002211463F
:10374000901E00F01DF80022BDE810401146501EEA
:1037500000F016B800F01F020121914040098000DE
:1037600000F1E020C0F88011704700F01F02012135
:1037700091404009800000F1E020C0F8001170473E
:10378000F0B40E4B1B680C46C3F30223C3F10705CC
:10379000042D00D90425191D072901D2002300E0BA
:1037A000DB1E012606FA05F1491E214099409E4084
:1037B000761E16403143F0BC04F0B5B80CED00E0C5
:1037C000064900F0070208684FF6FF03184040EA78
:1037D0000220034A10430860704700000CED00E02F
:1037E0000000FA052DE9F843044600684FF001098E
:1037F000C1074FF0000601D1400727D5DFF81C8133
:10380000C8F86860FFF732FF0746454D05E000BF86
:10381000FFF72CFFC01B022857D828680001F7D4F7
:1038200060688101207A41EA00703D498431086076
:10383000C8F86890FFF71AFF074604E0FFF716FF85
:10384000C01B022841D828680001F7D520788007DE
:1038500052D533484030016841F080510160006822
:10386000304D00F080500090286840F4807028604F
:10387000FFF7FCFE074604E0FFF7F8FEC01B022836
:1038800023D82868C005F7D5254D7035286810F471
:10389000407020D0A18901F4407181421BD028687A
:1038A00020F440712048C0F8009006602960286824
:1038B000C00710D0FFF7DAFE064641F2883707E06E
:1038C000FFF7D4FE801BB84202D90320BDE8F8837D
:1038D00028688007F4D5E1681148C1F30122083057
:1038E000032A12D0016821F4F81101602868A18927
:1038F000C1F30B01084328602078000703D50B496A
:10390000207CC1F8E0010020E0E70268084B22F4C7
:10391000F81219400A430260E8E70000000047423D
:103920000038024000700040400E474200104742FD
:10393000FFFCFF0F2DE9F0470E46050065D0DFF8CC
:103940001481D8F80000F7B200F00F00B04207D29F
:1039500088F80070D8F8000000F00F00B04254D191
:1039600028683D4C810712D5400703D5206840F4F4
:10397000E05020602878000703D5206840F46040BC
:1039800020602068A96820F0F000084320602878B3
:10399000C0072DD0304968680839012812D00228A4
:1039A00013D0032811D00968890700292DDA21686E
:1039B00021F0030101432160FFF758FE814641F2E7
:1039C000883A0EE009688903EFE709688901ECE7A6
:1039D000FFF74CFEA0EB0901514502D90320BDE8D9
:1039E000F0872068696800F00C00B0EB810FEFD120
:1039F000D8F80010404601F00F01B14207D9077016
:103A0000006800F00F00B04201D00120E7E72878FD
:103A1000400705D52068E96820F4E050084320609D
:103A20002878000706D52068296920F4604040EA1C
:103A3000C100206000F03CF82168084AC1F303117E
:103A4000515CC840064908600020FFF737FE00209F
:103A5000C5E70000003C02400838024074A103089A
:103A600000000020014800687047000000000020AE
:103A70000448054900680968044AC1F38221515C81
:103A8000C8407047000000200838024084A10308A5
:103A90000448054900680968044AC1F34231515C91
:103AA000C8407047000000200838024084A1030885
:103AB000154810B5006810F00C02144813D04110DE
:103AC000042A0FD0082A0ED10F4C241F2268236825
:103AD00002F03F025B0207D52068C0F38810A0FB0C
:103AE000010106E0084610BD2168C1F38811A1FB61
:103AF00000010023FCF76AFB2168C1F30141491C66
:103B00004900B0FBF1F010BD083802400024F40079
:103B10002DE9F84F050076D02878DFF8F8B2BE4CD2
:103B2000C00749D0DBF800105846C1F381010129D4
:103B300008D00068C0F3810002280AD1201D006867
:103B4000400206D52068800336D568680028E2D098
:103B500032E06868B0F5803F10D0B0F5A02F206843
:103B600010D020F480302060206820F48020206075
:103B70006868A0B1FFF77AFD06460CE0206840F4C3
:103B80008030F4E740F480202060F7E7FFF76EFD17
:103B9000801B642873D820688003F7D50CE0FFF7FA
:103BA00065FD064605E000BFFFF760FD801B642849
:103BB000F0D820688003F7D42878DFF86082800787
:103BC0004FF000093ED5DBF80010584611F00C0FFD
:103BD00009D00068C0F3810002280BD18D48001F76
:103BE0000068400206D42068800715D5E8680128DF
:103BF00009D111E0E868B8B10120C8F80000FFF76A
:103C000035FD064605E002E1FFF730FD801B022886
:103C1000C0D820688007F7D52068296920F0F8000F
:103C200040EAC10020600DE0C8F80090FFF71EFDDB
:103C3000064604E0FFF71AFD801B02281FD8206803
:103C40008007F7D42878000722D5724E7448696936
:103C50006C3671B101210160FFF708FD074604E0F1
:103C6000FFF704FDC01B022809D830688007F7D58C
:103C70000EE0C0F80090FFF7F9FC074605E083E08E
:103C8000FFF7F4FCC01B02287ED830688007F7D409
:103C90002878400768D5DFF87CA100270AF1380AA8
:103CA000DAF80000C0000BD4DAF8001041F08051BF
:103CB000CAF80010DAF80000012700F080500090E8
:103CC000584E3068C00510D4306840F480703060C1
:103CD000FFF7CCFC009005E0FFF7C8FC0099401A04
:103CE000022851D83068C005F6D54A4EA868683613
:103CF00001280FD00528306810D020F00100306076
:103D0000306820F004003060A868B8B1FFF7AEFC5E
:103D100000900FE0306840F00100F4E740F004004C
:103D20003060F7E7FFF7A2FC0099411A41F28830B2
:103D3000814264D830688007F4D50EE0FFF796FC26
:103D4000009007E0FFF792FC0099411A41F2883099
:103D5000814254D830688007F4D42FB1DAF80010CB
:103D600021F08051CAF80010A869C0B3DBF8001038
:103D7000C1F3810102294AD00228484607D0C8F879
:103D80006000FFF773FC00E039E005463AE0474683
:103D9000C8F86000FFF76AFC064604E0FFF766FC1F
:103DA000801B02282BD820688001F7D4D5E90701B1
:103DB0000843A96A1C4A490802EB01416A6A41EAC0
:103DC0008211084395F82C1040EA01611148001F48
:103DD000016001203866FFF749FC054605E014E064
:103DE000FFF744FC401B022809D820688001F7D562
:103DF0000BE000BFFFF73AFC401B022802D903206A
:103E0000BDE8F88F20688001F4D40020F8E7012095
:103E1000F6E7000008380240003802400000474240
:103E2000800E4742007000400000FFFF00685030E5
:103E300050F8210070470068503040F8212070474A
:103E40002DE9F8478946017F9246012928D00126AD
:103E50000677022141770268CA2151620168532224
:103E60004A6201688A68324D52054FF000032D689E
:103E70004FF0FF044FF003074FF4FA4C13D5B5FB96
:103E8000FCF24FF47A7802FB08F20092B2F10108DA
:103E9000CDF8008016D3CA68520704D54246F5E72C
:103EA0000220BDE8F8878A6822F480628A60B5FB48
:103EB000FCF14FF47A72514300910168009A551E4B
:103EC000009504D24C62477703770320E9E7CA687C
:103ED0005207F3D5C1F8149001688A6822F00702EE
:103EE0008A6001688A6842EA0A028A6011490A689F
:103EF00042F480020A600F4908310A6842F48002E5
:103F00000A600168CA6802F0800262F49062CA60C6
:103F100001688A6842F480428A6001688A6842F4D3
:103F200080628A6001684C62467703770020B8E7B8
:103F300000000020003C01407047000010B504461E
:103F40000068C16849050CD58068400409D5204641
:103F5000FFF7F2FF2068C16801F0800161F4906111
:103F6000C16003494FF4800008600120607710BDF4
:103F7000143C014010B500680B4641680D480140F3
:103F8000080CD870C1F304245C7001F03F049C70ED
:103F9000C1F34231197052B904F0E8F9D870587879
:103FA00004F0E4F95870987804F0E0F99870002073
:103FB00010BD00003FFFFF0010B50B460168896A85
:103FC000596001680969C1F30E01996000680168D0
:103FD0000E480140C1F305401870C1F306245C701F
:103FE00001F07F049C70402404EA1141D97052B959
:103FF00004F0BCF91870587804F0B8F95870987843
:1040000004F0B4F99870002010BD00007F7F7F009D
:1040100070B5040002D0607F10B106E0012070BDD1
:1040200000202077204600F049F8022060772168C0
:10403000CA204862216853204862204604F0AAF949
:10404000FF25042618BB206881681B4A1140816047
:104050002168886862681043D4E904231A43104336
:1040600088602168E068086120680169228941EA66
:10407000024101612068C16821F08001C1602068AF
:104080008068800607D4204600F00CF918B120683B
:1040900045626677C2E72068016C21F480210164E3
:1040A0002068016CA2691143016420684562012007
:1040B0006077002070BD0000BFFF8FFF10B5006863
:1040C000084988420CD108490120086000221146A5
:1040D0000320FFF755FBBDE810400320FFF745BB69
:1040E00010BD0000002800403C0E47422DE9F0477B
:1040F0000446007F0B4601281FD04FF0010984F8C9
:104100001C9002206077DAB19878D97840EA0145AE
:1041100058781978000240EA413005432168CA20E6
:104120004862216853204862204604F033F9002693
:10413000FF274FF0040860BB1AE00220BDE8F087BB
:104140005878C10603D500F0EF000A305870D878CF
:1041500004F015F90204587804F011F942EA00223B
:10416000987804F00CF90243187842EA4035D5E714
:104170000F480540206845602068C16821F0800133
:10418000C1602068806880060AD4204600F08AF862
:1041900030B12068476284F81D8026770120CDE782
:1041A0002068476284F81D9026770020C6E700004B
:1041B0003FFFFF002DE9F0470446007F0D46012830
:1041C00011D04FF0010A84F81CA00220607720680B
:1041D000002680684FEA406042B100281ADA287849
:1041E00004F0C4F817E00220BDE8F087002800DBE7
:1041F000EE70287804F0C3F80204687804F0BFF881
:1042000042EA0022A87804F0BAF80243E87842EAC9
:1042100000470AE0EE70A878297840EA01476878FC
:10422000E978000240EA014007432168CA20486259
:10423000216853204862204604F0ACF84FF0FF0894
:104240004FF00409E0B9164807402068076020686D
:10425000816821F480218160D5E903010843216848
:104260008A68104388602068C16821F08001C160BD
:104270002068806880060BD4204600F013F838B11F
:104280002168C1F8248084F81D9026770120ABE7CF
:104290002168C1F8248084F81DA026770020A3E7B8
:1042A0007F7F7F0070B504460068C16821F0A001DF
:1042B000C160FFF7DBF905464FF47A7607E000BFEF
:1042C000FFF7D4F9401BB04201D9032070BD20682C
:1042D000C0688006F4D5002070BD70B5040005D01C
:1042E0000025A56294F8510010B106E0012070BDD0
:1042F00084F85050204600F031F8022084F8510034
:104300002068016821F040010160D4E901010843FF
:10431000D4E903121143084361690843218B01F476
:1043200000710843E1690843216A0843A16A084310
:1043300021680860A069042101EA1040616A08430D
:10434000216848602068C16921F40061C161656528
:10435000012084F85100002070BD000000B5006805
:104360000E4987B0884216D10D480021026842F4F8
:1043700080520260006800F480500590E0200090B8
:104380000220CDE901010320039005200490694635
:104390000448FFF799F807B000BD00000030014065
:1043A00044380240000002402DE9F84F04464068BE
:1043B0000026984617460D464FF00409B0F5827F57
:1043C00001D1A06890B194F85000012819D04FF0A5
:1043D000010B84F850B0FFF749F9009094F85100B0
:1043E0004FF0000A01280ED002267FE084F8519099
:1043F00013460A462046CDF8008000F031F9BDE8AA
:10440000F88F0220FBE7002D6FD0002F6DD084F8CD
:104410005190C4F854A0A563A787E787C4F830A0DB
:10442000A4F834A0A4F836A0C4F840A0C4F844A06E
:10443000A0684FF40047B84204D12068016821F415
:104440008041016020680168490603D4016841F099
:1044500040010160E068B8B133E020688168C907B5
:1044600006D0007B05F8010BE08F401EE0870BE0D3
:10447000B8F1000F23D0B8F1FF3F05D0FFF7F6F8F1
:104480000099411A41451AD2E08F0028E5D11BE07E
:1044900020688168C90706D0C06825F8020BE08F44
:1044A000401EE0870DE0B8F1000F08D0B8F1FF3FE3
:1044B00007D0FFF7DBF80099411A414501D30326E5
:1044C00014E0E08F0028E3D16068B0F5827F0AD164
:1044D000A068B84202D0B0F5806F04D120680168AE
:1044E00021F040010160606D00B1012684F851B0F7
:1044F00084F850A0304682E72DE9F84F044690F842
:1045000050000026994617460D4601280DD04FF061
:10451000010B84F850B0FFF7A9F8804694F85100D9
:10452000B246012804D0022694E00220BDE8F88FAC
:10453000002D7BD0002F79D0032084F85100C4F8DF
:1045400054A02563A786E786C4F838A0A4F83CA049
:10455000A4F83EA0C4F844A0C4F840A0A068B0F5F8
:10456000004F04D12068016841F480410160206857
:104570000168490603D4016841F040010160E06828
:10458000B0F5006F606804D030B3E08E012823D00E
:104590003EE010B1E08E01281AD135F8021B2068E8
:1045A00005E020688168890706D535F8021BC160DF
:1045B000E08E401EE0860BE0B9F1000F34D0B9F177
:1045C000FF3F05D0FFF752F8A0EB080149452BD279
:1045D000E08E0028E5D11EE0216815F8010B087374
:1045E00006E020688168890706D515F8011B01736C
:1045F000E08E401EE0860BE0B9F1000F14D0B9F157
:10460000FF3F05D0FFF732F8A0EB080149450BD278
:10461000E08E0028E5D14B46012202212046CDF84C
:10462000008004F0C5FA10B1032613E011E0424601
:104630004946204604F08AFA18B101262020606518
:1046400008E0A06818B92068C16880680090606DB3
:1046500000B1012684F851B084F850A0304665E7D7
:104660002DE9F84F044690F8500000260A9F9A461C
:1046700093460D464FF0010801280ED0012084F822
:104680005000FEF7F3FF814694F85100616801285D
:104690000CD0B1F5827F07D102E00220BDE8F88F8F
:1046A000A16809B9042801D00226BDE055B1BBF1CB
:1046B000000F07D0BAF1000F04D094F85100012880
:1046C00002D004E00126AFE0052084F8510000206C
:1046D0006065C4F838B0A4F83EA0A4F83CA02563F7
:1046E000A4F836A0A4F834A02064606420680168AF
:1046F000490603D4016841F040010160E068B0F56B
:10470000006F606804D0E8B3E08E01283BD06AE017
:1047100010B1E08E01282ED1216835F8020BC86057
:10472000E08E401EE08626E0B8F1000F0DD0E08E4E
:1047300058B120688168890707D535F8021BC16028
:10474000E08E401EE0864FF00008E08F58B12068F0
:104750008168C90707D0C0682BF8020BE08F401EA4
:10476000E0874FF00108781C05D0FEF77FFFA0EB33
:104770000900B84246D2E08E0028D5D1E08F00284B
:10478000D2D136E0FFE7216815F8010B0873E08EFF
:10479000401EE08627E000BFB8F1000F0DD0E08E8C
:1047A00058B120688168890707D515F8011B017386
:1047B000E08E401EE0864FF00008E08F58B1206880
:1047C0008168C90707D0C0680BF8010BE08F401E55
:1047D000E0874FF00108781C05D0FEF747FFA0EBFB
:1047E0000900B8420ED2E08E0028D5D1E08F002813
:1047F000D2D13B46012202212046CDF8009004F0A0
:10480000D7F908B103260FE04A463946204604F09E
:104810009DF918B101262020606505E0A06818B94F
:104820002068C16880680090012084F85100002051
:1048300084F85000304631E74FF0E0210428086941
:1048400003D020F004000861704740F00400FAE74C
:104850001648174A0189491C89B2018113685B1CFB
:104860001360B1F57A7F1FD3002101814189114A7C
:10487000491C89B2418192ED000AF7EE000A30EE40
:10488000200A82ED000A012242710A290CD9BFF3E5
:104890004F8F09480168094A01F4E0611143016042
:1048A000BFF34F8F00BFFDE77047000004000020FA
:1048B00084020020AC0200200CED00E00400FA05A8
:1048C00010B5401EB0F1807F01D3012010BD4FF024
:1048D000E02460610F21601703F025F80020A0613B
:1048E00007202061002010BD10B5FFF7B1FF10BDFB
:1048F0007047704730B590F83820012A20D0012247
:1049000080F83820022380F8393003685C6824F08E
:1049100070045C6003685C680D682C435C6003682D
:104920009C6824F080049C6003689C6849680C4380
:104930009C6080F83920002180F83810084630BD8E
:10494000022030BD10B5040003D094F8390010B136
:1049500007E0012010BD002084F83800204600F058
:104960000DF8022084F83900211D206805F016FB9F
:10497000012084F83900002010BD000008B500684F
:104980000B49884212D10B48016841F002010160D5
:104990000068002200F00200009011461D20FEF782
:1049A000EFFEBDE808401D20FEF7DFBE08BD000099
:1049B00000040040403802400168CA6842F0010229
:1049C000CA600068016841F0010101600020704781
:1049D00070B5044690F83800012817D0012584F8F6
:1049E0003850022084F839002068826822F077026B
:1049F00022F47F4282600868502837D00DDC2028DE
:104A000059D005DC88B3102841D151E0022070BD97
:104A1000302853D040283AD13FE060282ED070286B
:104A20000BD0B0F5805F03D0B0F5005F2FD110E060
:104A30002068816821F0070115E0CB68D1E90121E8
:104A4000206805F0F3FA2168886840F077008860F4
:104A50001DE0CB68D1E90121206805F0E7FA206864
:104A6000816841F48041816011E01EE0CA684968B4
:104A7000206805F0EDFA5021206806E0CA68496810
:104A8000206805F0F6FA6021206805F0D9FA84F86C
:104A90003950002084F8380070BDCA684968206821
:104AA00005F0D6FA40212068EFE700212068ECE706
:104AB00010212068E9E720212068E6E730212068FE
:104AC000E3E7704770B50446006801694FF00005E0
:104AD000C943890715D4C168C943890711D4E91EA0
:104AE000016101202076206880698007204602D07D
:104AF000FFF7E7FF04E000F098F8204600F096F892
:104B0000257620680169C943490717D4C168C9439C
:104B1000490713D46FF00401016102202076206858
:104B2000806910F4407F204602D0FFF7CAFF04E0FE
:104B300000F07BF8204600F079F8257620680169BE
:104B4000C943090716D4C168C943090712D46FF0D5
:104B500008010161042020762068C0698007204692
:104B600002D0FFF7AEFF04E000F05FF8204600F04F
:104B70005DF8257620680169C943C90617D4C16864
:104B8000C943C90613D46FF01001016108202076D3
:104B90002068C06910F4407F204602D0FFF791FFE3
:104BA00004E000F042F8204600F040F82576206846
:104BB0000169C943C90708D1C168C943C90704D1FC
:104BC000891E0161204600F033F820680169C9435D
:104BD000090609D4C168C943090605D46FF08001EC
:104BE00001612046FFF784FE20680169C943490638
:104BF00009D4C168C943490605D46FF04001016179
:104C0000204600F02DF820680169C94389060BD4BD
:104C1000C168C943890607D46FF0200101612046AD
:104C2000BDE87040FFF765BE70BD7047704700007B
:104C300009490868401C0860B0F57A7F01D300205C
:104C400008606421B0FBF1F201FB1200002802D1E0
:104C5000024901200870704784020020E300002010
:104C6000704710B504000ED0242084F83900204687
:104C700000F0C8F80020E06384F8390084F83A00B6
:104C800084F8380010BD012010BD06F077B8000090
:104C900070B5026804461068D168536910F00F0FB0
:104CA00050D003F0010501F4907635435DD0C20782
:104CB00005D0CA0503D5E26B42F00102E263420768
:104CC00005D5DA0703D0E26B42F00202E263820705
:104CD00005D5DA0703D0E26B42F00402E263020773
:104CE00005D5DA0703D0E26B42F00802E263E26B1B
:104CF000002A33D0800604D5880602D5204605F068
:104D00007AFA20684069E16BC0F38010090700D48B
:104D100028B3204605F058FA2068416949061AD59B
:104D2000416921F040014161606BA0B11B490165FF
:104D3000606BFEF765F9002810D0606B016DBDE86F
:104D400070400847830610D58B060ED52046BDE877
:104D5000704005F050BA2046FFF797FF70BD20461F
:104D6000FFF793FF0020E06370BD030606D50B0636
:104D700004D52046BDE8704005F0DABB4006F3D507
:104D80004806F1D5D168204621F04001D1602021AC
:104D900084F8391000F0FFFA70BD0000F1A002089D
:104DA00070B5040004D094F83900002510B106E075
:104DB000012070BD84F83850204600F073F824209C
:104DC00084F839002068C16821F40051C160204690
:104DD00005F058FA2068016921F4904101612068CA
:104DE000416921F02A0141612068C16841F4005104
:104DF000C160E563202084F8390084F83A0000207F
:104E000070BD000010B50446214B01682148224ABC
:104E1000994210D1016821F0100101604FF4C06186
:104E20001046FEF7C9FA606BFEF7FCF8206BFEF740
:104E3000F9F8252027E0194B994211D11548001F98
:104E4000016821F4003101600C211046FEF7B4FA2C
:104E5000606BFEF7E7F8206BFEF7E4F8262012E01F
:104E60000F4B994213D1016821F0200101604FF4EA
:104E7000C0511046FEF7A0FA606BFEF7D3F8206B26
:104E8000FEF7D0F84720BDE81040FEF763BC10BD28
:104E9000001001404438024000000240004400403D
:104EA000001401402DE9F04F0446D0F800C0022064
:104EB000DFF834828D4B01210322DFF834A2C701D1
:104EC0000025460287B04FF0070B4FF04009C4455C
:104ED00051D1D3F800C04CF0100CC3F800C01B68CF
:104EE0000DF1040803F0100305935302009388E8C2
:104EF000070869465046FEF7E7FADFF8FCA17D494E
:104F000050464FF00068CAF80010C0E90185C0E9BA
:104F10000356CAF81450C0E90657CAF82050CAF818
:104F20002450FEF77BF920B140F2391173A006F04E
:104F3000C1F8794FC4F834A0CAF83840C7E903561D
:104F40007D61BD616B48FD613D6278307D6287E8BF
:104F500001033846FEF762F920B140F24B1167A019
:104F600006F0A8F82763002211462520BC63FEF74F
:104F700007FC252056E0DFF8A481C44557D15B4BE0
:104F80001B1FD3F800C04CF4003CC3F800C01B68E2
:104F90000DF1040803F4003305930C23009388E813
:104FA000070869465046FEF78FFADFF878A15C499A
:104FB00050464FF00068CAF80010C0E90185C0E90A
:104FC0000356CAF81450C0E90657CAF82050CAF868
:104FD0002450FEF723F920B14FF4BC7147A006F02E
:104FE00069F8514FC4F834A0CAF83840C7E90356ED
:104FF0007D61BD614A48FD613D6218307D6287E890
:1050000001033846FEF70AF920B14FF4C5713BA001
:1050100006F050F82763002211462620BC63FEF7F5
:10502000AFFB2620FEF7A1FB07B0BDE8F08FDFF84D
:10503000FC80C445F8D1D3F800C04CF0200CC3F874
:1050400000C01B680DF1040803F0200305934FF422
:10505000C053009388E80700082004906946504632
:10506000FEF732FA2349DFF8C880183940464FF07E
:10507000206AC8F80010C0E901A5C0E90356C8F8C5
:105080001450C0E90657C8F82050C8F82450FEF75D
:10509000C5F820B140F2B71118A006F00BF8254F63
:1050A000C4F83480C8F83840C7F80890C7E90356F8
:1050B0007D61BD610F48FD613D6260307D62C7E981
:1050C000000A3846FEF7AAF820B140F2C9110BA039
:1050D00005F0F0FF2763002211464720BC63FEF76E
:1050E0004FFB47209EE7000000100140443802407B
:1050F0000000024040640240147D00202E2E2F53F9
:1051000072632F73746D3332663478785F68616CC4
:105110005F6D73702E630000747D002000440040BA
:1051200088600240D47D0020347E002000140140BD
:10513000947E0020F47E0020F8B5044690F83A00F2
:1051400020283CD1C1B3BAB394F83800012836D036
:10515000012084F83800A162A2850025E5632220A1
:1051600084F83A00636B1748D863636B1648186479
:10517000636B1648D864606B134605650846666B1A
:10518000216802463046091DFEF7B2F82068016822
:105190004168009184F83850C16841F48071C16061
:1051A0002068416941F0010141612068416941F095
:1051B000400141610020F8BDFFE70120FBE702202C
:1051C000F9E700004BA1020887A1020801A102082B
:1051D00090F83A30202B1DD1D1B1CAB190F83830B7
:1051E000012B17D081628285C2850021C1632222F2
:1051F00080F83A2080F8381001684A6942F00102CC
:105200004A610068C16841F49071C1600020704734
:10521000012070470220704705F0D4BD70472DE98A
:10522000F843044690F839001F4616460D462028DC
:1052300050D1A5B19EB194F8380001284AD0012080
:1052400084F838004FF00008C4F83C80212084F82E
:105250003900FEF70BFAA6848146E68426E0012099
:10526000BDE8F883E08C401EE084A0684B46B0F5B2
:10527000805F4FF000024FF080012046009703D07E
:1052800005F087F9E8B90DE005F083F9C8B9288879
:105290002168C0F308004860206908B16D1C05E072
:1052A000AD1C03E0216815F8010B4860E08C002874
:1052B000D8D14B46002240212046009705F069F9DD
:1052C00008B10320CCE7202084F8390084F8388026
:1052D0000020C5E70220C3E770B5044690F8390006
:1052E000202830D169B362B394F8380001282AD05D
:1052F000012084F838002162A284E2840025E5635D
:10530000212084F83900236B1048D863236B1048A0
:105310001864236B0F48D864206B13460565266814
:10532000206B321DFDF7E4FF21686FF0400008603C
:1053300084F838502068416941F0800141610020C3
:1053400070BD012070BD022070BD000091A1020857
:10535000BFA1020801A1020890F83930202B18D112
:10536000A9B1A2B190F83830012B12D00162828429
:10537000C2840021C163212280F8392080F83810CE
:105380000068C16841F08001C160002070470120C1
:1053900070470220704705F0BFBD70472DE9FE43FE
:1053A00004460025A84600260020029000270CB1E4
:1053B000606808B9BDE8FE83A068402800D9F9E715
:1053C00000252CE0204600F0DFF82E464FF00008C4
:1053D0001DE0606A825D02AB4146204600F07DF927
:1053E0000746022F0DD1606A0090E06A0190606864
:1053F000029A00EBC2006A464168204600F0A2F81B
:1054000008E007B906E000BF761C08F10108E06A71
:10541000B042DED800BF022F00D103E06D1CE06A6D
:10542000A842CFD800BF00BFC4E700000FB438B512
:1054300004460D4607A80090D4E90601009B069A91
:1054400005F066FE206200200090084800780128E0
:1054500003D1216AA06900F09FFA29462046236AF9
:10546000A26900F00DF838BC5DF814FBDC020020E6
:1054700010B50446A06B01F003FA002010BD000037
:10548000F8B504460D4616461F463A4631462046B4
:105490006369984750B92046FFF7EAFF0094084B2C
:1054A0002A460021A06B01F0EFFA06E00094054BBC
:1054B00001220021A06B01F0E7FA0020F8BD0000F6
:1054C00009560208F955020870B504460D468021B8
:1054D000204601F085FB2868E06368686060A86882
:1054E000A060E868E0602869206168696061A86977
:1054F000A061E869E06100202062286A6062686A51
:10550000A0620020E06284F83000A86A606304F1C1
:10551000380001F0CBF910B14FF0FF3070BD2046DC
:1055200000F002F8FAE70000014611B94FF0FF3031
:105530007047034800680860014801600020F7E7F1
:10554000D802002070B504460D461646022D06D03E
:10555000032D05D0042D04D0052D07D102E000BF96
:1055600000BF00BF2046FFF783FF00E000BF00BF81
:1055700032462946E06B00F01BFA70BD0148007806
:1055800070470000DC02002010B5044601224021D3
:1055900004F14000FAF7CEFE10BD000010B5002463
:1055A000124804681EE0204621698847C8B910489F
:1055B0000078012810D1E16A606A01F081FB0128BE
:1055C00003D1606A00F03CF906E0E16A606A00F02D
:1055D000B1F908A000F034F92046FFF7DFFE002003
:1055E000E0622468002CDED110BD0000D80200204B
:1055F000DC0200200D0A000010B50446002205213F
:105600002046FFF79FFF10BD10B50446002204217D
:105610002046FFF797FF10BD70B504460D462046A3
:1056200000F02FF8012801D1801E70BD2068401CB9
:10563000E168B0FBF1F201FB1200206026692368EB
:10564000A16803FB061032462946FAF753FE0020F4
:10565000EBE710B58160C26003610124446000245F
:10566000046010BD01460868401CCA68B0FBF2F334
:1056700002FB13004A68904201D1012070470020CC
:10568000FCE701460868801CCA68B0FBF2F302FB25
:1056900013004A68904201D1012070470020FCE7C6
:1056A00070B504460D462046FFF7DCFF012801D106
:1056B000801E70BD2669D4E9013003FB0601324625
:1056C0002846FAF717FE6068401CE168B0FBF1F26B
:1056D00001FB120060600020EBE7F0B504460D46C8
:1056E000002600211BE004F14000405C012815D198
:1056F000606850F83100405D904204D0002704F10A
:10570000400047540AE0761C606850F83170681C0D
:10571000385C18B903B119600220F0BD491CA068BB
:105720008842E0D80EB90020F7E70120F5E710B570
:10573000024612B94FF0FF3010BD00BF106888421A
:10574000FCD31068401A106050680844D368B0FB5E
:10575000F3F403FB140050600020EDE710B502469F
:1057600012B94FF0FF3010BD10680844106000BF40
:10577000D36810689842FBD890680844D368B0FB9F
:10578000F3F403FB140090600020ECE7F0B504464E
:10579000002522B11BB1E6682068B04202D34FF069
:1057A000FF30F0BD2668E068801B884202D24FF0CF
:1057B000FF30F6E7A0680844E668B0420BD9D4E9A8
:1057C0000260851B2668E068801B4E19B04202D239
:1057D0004FF0FF30E5E7A0682844E668B0FBF6F735
:1057E00006FB17001060681818600020D9E7014612
:1057F00048687047014688687047024612B94FF002
:10580000FF3070470020506090601060D16000BF92
:10581000F7E7014609B901207047086808B9012077
:10582000FAE70020F8E7014609B9012070470A6845
:10583000C868904201D10120F8E70020F6E7000097
:105840000FB40E4810B54078ADF5007D28B10DF5C8
:10585000007D002010BC5DF814FB4FF4007483AB96
:1058600021466846829A05F053FC0246A04200D3C6
:10587000621E6946002005F0DBFAE8E728010020F7
:105880000FB4224810B54078ADF5087D28B10DF56C
:10589000087D002010BC5DF814FB86A802F098FD7E
:1058A000FDF7E4FE4FF47A71B0FBF1F201FB120058
:1058B0009DF81D329DF81C229DF81E12CDE90410A2
:1058C0009DF81B129DF81A02CDE90223CDE90001D3
:1058D0004FF40074BDF818320DA2214606A801F05D
:1058E000FCFA024606A9002005F0A2FA8BAB21467D
:1058F00006A88A9A05F00CFC0246A04200D3621E5C
:1059000006A9002005F094FAC1E700002801002054
:10591000253034752D253032752D253032752025F2
:105920003032753A253032753A253032752E2530B1
:1059300033752000F0B5064615480C4691B0417805
:1059400011BB007801281FD10127102C01D9102587
:1059500000E02546402101A8FAF7F3FC402301AA04
:1059600029463046009701F0EFF80AA101A8FAF79E
:10597000F3FC01A8FAF724FD024601A9002005F076
:1059800057FA641B2E44E0D111B00020F0BD000096
:10599000280100200D0A0000044A52780AB10020B4
:1059A00070470A460146002005F042BA280100204F
:1059B0002DE9FC4104460D4617464FF0000800262D
:1059C000608801281FD1206950B960680068CDE95E
:1059D00000051AA200212046E368FCF7ABFE12E0A6
:1059E000206950F8250000782D280CD0206950F847
:1059F000250061680968CDE9001018A20021204641
:105A0000E368FCF797FE66683A4629462046F36845
:105A1000984780460BE0706840B170683A46294666
:105A2000C368204698478046766800E002E0B8F1F7
:105A3000010FF0D000BFBDE8FC81000046534D3A95
:105A4000252D38732053544154453A252D3238734F
:105A5000204556454E543A25750D0A0046534D3A99
:105A6000252D38732053544154453A252D3238732F
:105A7000204556454E543A25730D0A002DE9F0474E
:105A800004460E4617469846DDE9089A00250CB9EB
:105A9000BDE8F08730212046FAF753FCC4F808909F
:105AA000C4F810806660E7600021A16261620E4860
:105AB00000882080A4F802A00C48006860610B48B0
:105AC000046009480088401C07490880656806E0B2
:105AD0006560002211462046FFF76AFFAD68002D81
:105AE000F6D100BFD4E70000C0020020BC020020B5
:105AF000024612B94FF0FF307047D1620020FBE739
:105B00002DE9F84305460E4617461C46DDF8209061
:105B10004FF000082188484661F31F408046054B3E
:105B20003A4631462846CDF8008000F0ADFFBDE88A
:105B3000F8830000A92702082DE9F04196B0054638
:105B40000E461746D5F804800024002015904446E0
:105B500029E06C60002201212846FFF729FFA642B8
:105B600005D13A4600212846FFF722FF1DE05021CB
:105B700001A8FAF7E6FB15AB01AA21463046FCF76F
:105B8000F4FD78B90AE01598006868603A4600218B
:105B90002846FFF70DFF15984068159015980028C6
:105BA000F1D102E06468002CD3D100BFB46806E0F4
:105BB0006C603A4600212846FFF7FAFEA468002CE4
:105BC000F6D116B0BDE8F081016E05E000F17C026F
:105BD0004B1CD35C5354491CC26D8A42F6D87047A3
:105BE00010B5C26D511E05E000F17C02545C4B1CE7
:105BF000D454491E026E8A42F6DD10BD70B50546CA
:105C00000C46A87910B101282ED100E000BF432C2A
:105C10001BD004DC412C0CD0422C22D10FE0442CB0
:105C200019D07E2C1DD100220821284600F028FB27
:105C300018E000220321284600F022FB12E0002297
:105C40000421284600F01CFB0CE000220621284617
:105C500000F016FB06E000220521284600F010FBAC
:105C600000E000BF00BF2CE0432C1BD004DC412C23
:105C70000CD0422C22D10FE0442C19D07E2C1DD107
:105C800000220821284600F07FF818E000220321B6
:105C9000284600F079F812E000220421284600F09E
:105CA00073F80CE000220621284600F06DF806E0AB
:105CB00000220521284600F067F800E000BF00BF81
:105CC00000BF00BF70BD70B504460D46432D45D0E2
:105CD00008DC1B2D0DD0332D24D0412D3CD0422D7E
:105CE0004CD13AE0442D3AD05B2D10D07E2D45D1D9
:105CF00023E0207910B1042804D100E000BF012086
:105D0000207102E00020207100BF00BF39E020793F
:105D1000012802D10220207102E00020207100BF82
:105D200000BF2EE02079022802D10320207102E07A
:105D30000020207100BF00BF23E02079032806D196
:105D400029462046FFF75AFF0420207102E0002078
:105D5000207100BF00BF14E000BF00BF00BF20796A
:105D6000022806D129462046FFF748FF042020716B
:105D700002E00020207100BF00BF02E0002020717F
:105D800000BF00BF207970BD2DE9F04104460D46EB
:105D90001746092D02D00020A066E0660A2D6FD2BA
:105DA000DFE805F06E0540CDFDFCFBFAF9F86079FF
:105DB00010B1012833D100E000BFE06D63282BD281
:105DC0003846D4F8981588472046FFF709FF04F1B4
:105DD0007C00216E4754206E401C2066E06D401C04
:105DE000E065266E4FF0000808E004F17C02905D4B
:105DF000D4F898158847761C08F10108E06DB04288
:105E0000F3D803E00820D4F898158847B8F10000CB
:105E1000A8F10108F6D100BF0020607100E000BFCA
:105E200000BF28E2E06D20B9FEA0D4F894158847A1
:105E300021E2607910B1012866D122E0002104F14D
:105E40007C00E26D8154616F01EBC10202EB011233
:105E500004F5A27101EB8200C839FAF7D3FA606F3A
:105E6000401C6067606F0A2801DB00206067A06F3C
:105E7000401CA067A06F0A2801D30A20A06744E055
:105E8000F8E100BF00BF206F00EBC00202EB001280
:105E900004F5A27000EB8201642204F22C50FAF7A0
:105EA00029FA266F19E0701C0A21B0FBF1F201FB00
:105EB000120808EBC80202EB081304F5A27202EB09
:105EC000830106EBC60202EB061304F5A27202EB95
:105ED00083006422FAF70EFA4646606F09300A2101
:105EE00090FBF1F201FB1200B042DCD106EBC601DF
:105EF00001EB061204F5A27101EB8200642204F2A8
:105F00002C51FAF7F7F900E000BF00BFC6A0D4F8A3
:105F100094158847204600F0ADFC04F17C0000F0A9
:105F20000BFC002000F0A6FC00202066E065606FFE
:105F30000A302067BDA0D4F8941588479BE16079AA
:105F400010B1012853D100E000BFA06F00B94FE0AD
:105F5000A06F0A2803D1D4E91C0188420ED1A06F9A
:105F60000A2841D0606F0A30A16F401A0A21B0FBA5
:105F7000F1F201FB1200216F884235D0206F093009
:105F80000A21B0FBF1F201FB12002067206F00EB49
:105F9000C00205E008E1CCE08EE07EE072E029E09E
:105FA00002EB001204F5A27000EB8201C838FAF788
:105FB00029FA04F17C00FAF703FAE065E06D206647
:105FC0009BA0D4F894158847226F02EBC20303EB21
:105FD000021304F5A27202EB8300D4F894158847EB
:105FE00094A0D4F8941588470120607100E000BFA8
:105FF00000BF40E1607910B1012840D100E000BF4E
:10600000A06F00B93CE0606F09300A2190FBF1F20B
:1060100001FB1200216F88422ED0206F401C0A2104
:10602000B0FBF1F201FB12002067206F00EBC00211
:1060300002EB001204F5A27000EB8201C838FAF7F7
:10604000E1F904F17C00FAF7BBF9E065E06D206648
:1060500077A0D4F894158847226F02EBC20303EBB4
:10606000021304F5A27202EB8300D4F8941588475A
:1060700070A0D4F8941588470120607100E000BF3B
:1060800000BFF8E0206E002806DD206E401E20666E
:106090000820D4F898158847EDE0D4E91710884215
:1060A00009D204F17C02236ED05CD4F8981588479D
:1060B000206E401C2066DEE0607910B1012835D1E9
:1060C00000E000BFE06D70B3206E00282BDD0820DB
:1060D000D4F898158847266E4FF0010808E004F1BF
:1060E0007C02905DD4F898158847761C08F1010869
:1060F000E06DB042F3D82020D4F89815884703E02B
:106100000820D4F898158847B8F10000A8F10108D4
:10611000F6D1206E401E20662046FFF755FDE06D4B
:10612000401EE06500BF0020607100E000BF00BFBE
:10613000A1E0607910B1012833D100E000BFE06D2B
:1061400060B3206E002829DDD4E91701884225D0EC
:10615000206E461C4FF0010808E004F17C02905DBF
:10616000D4F898158847761C08F10108E06DB04214
:10617000F3D82020D4F89815884703E00820D4F8F5
:1061800098158847B8F10000A8F10108F6D120461B
:10619000FFF71AFDE06D401EE06500BF0020607152
:1061A00000E000BF00BF66E0607910B101285ED159
:1061B00000E000BFE06D98B3E06E50B90120E066EA
:1061C00004F17C0104F1E000E26DFAF793F8E06D70
:1061D00060663CE0A06E00F0F5FA064604F1E001CE
:1061E000626EFAF718F9E0B913A0D4F8941588474D
:1061F000A06E00F0E7FA0646D4F894158847A06E22
:1062000000F0E0FA0646314604F17C00FAF7FAF8AD
:1062100004F17C00FAF7D4F8E065E06D20660FE049
:1062200022E011E00D0A3E000D0A00003E000000D1
:106230000D3E00001B5B4A000D1B5B4A3E00000048
:10624000A06E401CA06607E0A06E401CA06600F097
:10625000B3FAA16E8842BDD800BF00F0ADFAA16EBE
:10626000884201D80020A0660020607100E000BFD5
:1062700000BF00E000BF00BFBDE8F0810020704714
:106280002DE9F04104460E461746092E7DD2DFE87F
:1062900006F07C05457C7C9BA6BDF800E06D63287C
:1062A0003BD2A079012804D12A20D4F89815884738
:1062B00003E03846D4F8981588472046FFF790FC4D
:1062C00004F17C00216E4754206E401C2066E06D76
:1062D000401CE065256E4FF0000810E0A079012811
:1062E00004D12A20D4F89815884705E004F17C02EF
:1062F000505DD4F8981588476D1C08F10108E06DD1
:10630000A842EBD803E00820D4F898158847B8F1E4
:106310000000A8F10108F6D1ECE0EBE0E06D30B947
:10632000A07920B975A0D4F894158847E2E0A07947
:1063300010B1012845D115E0002104F17C00E26D87
:10634000815472A0D4F8941588470120A0710020D0
:106350002066E06504F17C02102104F10C0000F0DD
:10636000BCFD2FE0002104F17C00E26D815400208F
:10637000E06504F17C02402104F11C0000F0ADFD59
:1063800004F11C0104F10C0000E0B2E000F070F92F
:1063900050B962A0D4F8941588470220A07100205B
:1063A0002066E06560710BE060A0D4F89415884722
:1063B00052A0D4F8941588470020A0712066E065AB
:1063C00000E000BF00BF95E0206E002806DD206ED3
:1063D000401E20660820D4F8981588478AE0D4E942
:1063E0001710884211D2A079012804D12A20D4F8AC
:1063F0009815884706E004F17C02236ED05CD4F83F
:1064000098158847206E401C206673E0E06DB0B39D
:10641000206E002833DD0820D4F898158847256EB3
:106420004FF0010810E0A079012804D12A20D4F807
:106430009815884705E004F17C02505DD4F8981562
:1064400088476D1C08F10108E06DA842EBD82020B8
:10645000D4F89815884703E00820D4F898158847A1
:10646000B8F10000A8F10108F6D1206E401E2066A8
:106470002046FFF7A9FBE06D401EE06500BF39E054
:10648000FFE7E06DA0B3206E002831DDD4E91701ED
:1064900088422DD0206E451C4FF0010810E0A079F5
:1064A000012804D12A20D4F89815884705E004F182
:1064B0007C02505DD4F8981588476D1C08F10108DE
:1064C000E06DA842EBD82020D4F89815884703E067
:1064D0000820D4F898158847B8F10000A8F1010801
:1064E000F6D12046FFF770FBE06D401EE06500BF6F
:1064F00000E000BF00BFBDE8F08100000D0A757329
:1065000065726E616D653A20000000000D0A7061D1
:106510007373776F72643A20000000000D0A5765AC
:106520006C636F6D65210D0A3E0000000D0A557306
:10653000657220766572696679206661696C65644A
:106540002E00000038B50020009000244248046866
:106550007EE076E000F0DAF905469DF8001020466E
:10656000FFF7B1FB00B16CE0FFF788FE01280AD10C
:10657000A068281A3949884207D9A5600020A0716F
:10658000E065206601E00220A071A07910B1012829
:106590002BD100E000BF9DF800000D2806D19DF82A
:1065A000002002212046FFF76BFE1DE09DF8000051
:1065B0000A2819D09DF80000082805D100220721DB
:1065C0002046FFF75DFE0FE09DF80000092805D189
:1065D000002209212046FFF753FE05E09DF8002028
:1065E00001212046FFF74CFE29E09DF800000D2810
:1065F00006D19DF8002002212046FFF7C5FB1DE0D3
:106600009DF800000A2819D09DF80000082805D13F
:10661000002207212046FFF7B7FB0FE09DF800009E
:10662000092805D1002209212046FFF7ADFB05E02E
:106630009DF8002001212046FFF7A6FB00BF00BF08
:1066400000BF6846D4F89C158847002882D024688B
:10665000002C7FF47EAF38BDE002002040771B00A5
:10666000024909680160014908607047E0020020A2
:10667000024600207047000000BFEFF3058000B124
:1066800070470748006820B9012080F3108800BFD8
:1066900000BF03480068401C0149086000BFEFE7E5
:1066A000C402002010B50446002010BD70B5044699
:1066B0000D4600F099F850B100F096F8D0F890052A
:1066C00028B100F091F8D0F8901502A0884700207A
:1066D00070BD00001B5B481B5B4A000030B50246E2
:1066E0000C460021002302B114B94FF0FF3030BD39
:1066F0000021002315E00E4850F8310080B952F80F
:1067000033000B4D45F8310002EBC300406805EB48
:10671000C105686007480068401C064D28605B1C86
:10672000491C502901D2A342E5D30020DFE7000035
:10673000EC020020E8020020F0B595B004460026E7
:1067400000E0641C20782028FBD02046F9F738FEB2
:1067500010B9002015B0F0BD2046F9F731FE2044F5
:10676000461E02E000203070761E30782028F9D0D6
:10677000142301AA2021204600F0C6FB074600256D
:1067800011E00C4951F835002146F9F720FE48B9CF
:10679000084800EBC50001A942683846904700B997
:1067A00005E004E06D1C00F007F8A842E9D800BF3E
:1067B0000020CFE7EC02002001480068704700008D
:1067C000E8020020014605480068814201D304A088
:1067D0007047044850F83100FAE70000E802002052
:1067E00000000000EC020020014800687047000033
:1067F000E40200202DE9F04106460F4600252AE07C
:10680000002412E0FFF7F0FF70B1FFF7EDFFD0F8C2
:10681000900548B1FFF7E8FFD0F890252819114BF3
:1068200053F8301010A09047641C052C04DAFFF7D1
:10683000C3FF29198842E5D8FFF7D6FF50B1FFF70B
:10684000D3FFD0F8900528B1FFF7CEFFD0F8901510
:1068500007A088476D1DFFF7AFFFA842D0D80020E2
:10686000BDE8F081EC020020252D313673000000D8
:106870000D0A00000149086070470000E402002092
:106880000146202902D34FF0FF3070470120C1EBB1
:10689000C102054B43F822000020C1EBC10203EB0B
:1068A0008202D06000BFF0E7547F002070B505463B
:1068B00000240DB9601E70BD00240DE0C4EBC400BF
:1068C0000C4951F8200030B90120C4EBC401094A39
:1068D00042F8210002E0641C202CEFD300BF202CE2
:1068E00005D105A0FEF7ACFF4FF0FF30E3E72C60C9
:1068F0000020E0E7547F002074696D6572204944F0
:106900002069732066756C6C0D0A000001480068F0
:1069100070470000C802002070B5FFF7ADFE0448C4
:106920000468456800F0F6F82046294670BD00006E
:10693000D002002010B5002400BF4AE0C4EBC40020
:10694000254951F82000022842D1C4EBC40001EBD4
:106950008000C06821490968081AC4EBC4011E4AB6
:1069600002EB81010969884232D9C4EBC4001146A7
:1069700001EB8000806928B3C4EBC40001EB800008
:10698000007928B90120C4EBC40142F821000CE0D1
:106990000220C4EBC401104A42F821000F480068ED
:1069A000C4EBC40102EB8101C860C4EBC4020A4B12
:1069B00003EB82025069C4EBC40203EB82029169CB
:1069C000884705E00120C4EBC401034A42F82100D6
:1069D000641C202CB2D310BD547F0020C8020020BC
:1069E00010B50446202C49D2C4EBC400244951F808
:1069F0002000022842D1C4EBC40001EB8000C06833
:106A000020490968081AC4EBC4011D4A02EB810140
:106A10000969884232D9C4EBC400114601EB8000F9
:106A2000806928B3C4EBC40001EB8000007928B969
:106A30000120C4EBC40142F821000CE00220C4EBA9
:106A4000C4010F4A42F821000E480068C4EBC4019B
:106A500002EB8101C860C4EBC402094B03EB820264
:106A60005069C4EBC40203EB82029169884705E0D8
:106A70000120C4EBC401024A42F8210010BD00000D
:106A8000547F0020C8020020F0B50446059D202C4C
:106A900002D34FF0FF30F0BD0220C4EBC406114F0B
:106AA00047F82600C4EBC4003E4606EB80000171A7
:106AB0000D480068C4EBC40607EB8606F060C4EB23
:106AC000C4003E4606EB80000261C4EBC40006EB46
:106AD00080008361C4EBC40006EB800045610020A8
:106AE000D9E70000547F0020C80200200748006852
:106AF000401C06490860064802684068521C40F184
:106B0000000003490A60486070470000C802002086
:106B1000D002002000BFEFF3058000B170470948A4
:106B2000006820B107480068401E06490860054813
:106B3000006820B9002080F3108800BF00BF00BFAC
:106B4000ECE70000C40200202DE9F04305460C46A6
:106B50009846079F0026002399460DB102B114B94B
:106B60000020BDE8F083012F01D1032000E00220C6
:106B70006043401C404501D90020F2E7002618E0A0
:106B800015F806904FEA191000F019F819465B1C29
:106B9000505409F00F0000F012F819465B1C5054D5
:106BA000012F05D14FF0200C18465B1C02F800C0E5
:106BB000761CA642E4D30020D0541846D1E7014603
:106BC000092903DC01F13000C0B270470A2905DB56
:106BD0000F2903DC01F13700C0B2F6E73020F4E7FB
:106BE00070B504460D4629462046F9F7AAFB70BD4C
:106BF0000146302904DB392902DCA1F130000EE026
:106C0000412904DB462902DCA1F1370007E06129B4
:106C100004DB662902DCA1F1570000E00020C0B2CD
:106C2000704710B502460B46002406E01078FFF7C7
:106C3000DFFF00EB0414521C5B1E002BF6D1204634
:106C400010BD00B50246002305E01078FFF7D0FF25
:106C500000EB0313521C10780028F6D1184600BD33
:106C600070B588B005460C46002007900690059048
:106C700004902846F9F7A4FB064604A805A906AA2D
:106C800007ABCDE9002102900AA23146284600F068
:106C900031F8042803D04FF0FF3008B070BD0798DA
:106CA0002070069860700598A0700498E07000202D
:106CB000F3E7000025642E25642E25642E2564004C
:106CC00002460B46002100BF10E0505C202803DB89
:106CD000505C7E2800DC08E0505C0D2802D0505C3F
:106CE0000A2800D101E000207047491C9942ECD3EA
:106CF0000120F9E70FB42DE9F84704460020009081
:106D00000022202600270CB10B9820B90020BDE8F6
:106D1000F8075DF814FB0CA80090D4E041B90B987B
:106D20000078252803D10B984078652800D0CFE063
:106D30000B980078252874D10B98401C0B900B9869
:106D400010F8016B0B90652E6CD004DC2A2E07D056
:106D5000642E68D113E0702E7AD0782EF9D144E0F9
:106D600008E020780B9B1B78984202D0641C491ED7
:106D700000E001E00029F4D100BF521C92E04FF086
:106D8000000CE046002300252020DDF8009059F893
:106D9000045BCDF800901AE02078B8F1000F06D11E
:106DA0002D2804D14FF0010C4FF001080DE03028E0
:106DB0000ADB392808DC4FF00108A0F1300903EBA9
:106DC000830A09EB4A0300E003E0641C491E002922
:106DD000E2D100BFBCF1010F03D16FEA030909F151
:106DE000010305B12B60521C5CE000230025DDF897
:106DF00000C05CF8045BCDF800C022E020783028A9
:106E000006DB392804DCA0F1300C0CEB031316E090
:106E1000612809DB662807DCA0F1570C0CEB031393
:106E20000DE043E033E03AE0412807DB462805DC8B
:106E3000A0F1370C0CEB031301E009E003E0641C44
:106E4000491E0029DAD100BF05B12B60521C29E090
:106E5000DDF800C05CF8040BCDF800C0002500236D
:106E600025460CE094F800C0DDF82C8098F80080EE
:106E7000C44501D05B1C00E003E0641C491E0029EE
:106E8000F0D100BF08B105604360521C0AE0009BCE
:106E900001CB009300B10460521C012702E00127DE
:106EA000002200BF00BF012F0DD111E020780B9B05
:106EB0001B78984205D1641C0B98401C0B90491E0E
:106EC00001E0002204E00B98007800287FF426AF50
:106ED00000BF00200090104619E70FB4F8B5064631
:106EE0000C46002509A8009021463046009B089AD0
:106EF00004F00EF9054600200090A54200D3651E5F
:106F00002846F8BC5DF814FBF0B504460E461D4655
:106F1000214600230DB104B10AB90020F0BD184686
:106F20005B1C42F820100AE00878B04206D100202D
:106F30000870481C1F465B1C42F82700491C087853
:106F400008B1AB42F0D31846E8E770B50646002515
:106F5000002478213046F9F729FA044624B958214B
:106F60003046F9F723FA04465CB1641C05E020784A
:106F7000FFF73EFE00EB0515641C20780028F6D1D3
:106F800003E03046F9F764FA0546284670BD70B54F
:106F900004460D4604B115B94FF0FF3070BD012114
:106FA00004F11000FEF7C3FB04F12000A968FEF70E
:106FB000BEFB0020F2E770B504460D4604B115B9DA
:106FC0004FF0FF3070BD012104F11000FEF7C6FB49
:106FD00004F12000A968FEF7C1FB0020F2E710B51C
:106FE00004460CB9002010BD04F11000FEF711FC9E
:106FF000012801D10020F6E704F12000FEF709FC8A
:10700000012801D10020EEE704F11000FEF7EFFBAC
:1070100000EB4000216801EB8000E4E77CB504460A
:107020000E46002500200190009004B97CBD04F1BB
:107030001000FEF7F8FB08B10020F7E76B4601AA45
:10704000314604F12000FEF7A1FB08B10020EDE776
:1070500004F11000FEF7CEFB00EB4000216801EBCD
:107060008005A0680199084428606E600098A860B7
:107070002846DBE72DE9F04104460E4617461D463B
:107080004FF0000805EB4500B7EB800F03D84FF039
:10709000FF30BDE8F08105EB45004FEA800826602F
:1070A000C4F8048060683044A060A7EB0801E16088
:1070B000294604F11000FEF7A0FB04F12000E1686E
:1070C000FEF79BFB0020E4E703F0D4FCFCE70000A4
:1070D00070B50F4D4FF48044002221462846FCF73E
:1070E000C0FA002261102846FCF7BBFA0A2007F01C
:1070F00060FA012221462846FCF7B3FA0A2007F07D
:1071000058FA21462846BDE870400022FCF7A9BA8B
:107110000004024070B50F4D4FF480440022214618
:107120002846FCF79EFA012251032846FCF799FAFB
:107130000A2007F03EFA012221462846FCF791FA80
:107140000A2007F036FA21462846BDE870400022A2
:10715000FCF787BA000402402DE9F0470024174FDE
:10716000804625464FF480464FF4005900223146B0
:107170003846FCF776FA0A2007F01BFA012231465E
:107180003846FCF76EFA6006040E49463846FCF7AE
:107190005FFA08B1641CE4B2052007F00AFA6D1C1E
:1071A000EDB2082DE2D3B8F1000F04D0FFF790FF45
:1071B0002046BDE8F087FFF7ADFFF9E70004024085
:1071C0002DE9F041174F05464FF480460022314625
:1071D0003846FCF746FA00244FF40058280601D53B
:1071E000012200E0002241463846FCF73AFA6806E0
:1071F000050E0A2007F0DDF9012231463846FCF77A
:1072000030FA0A2007F0D5F9002231463846FCF75B
:1072100028FA0A2007F0CDF9641CE4B2082CDDD36B
:10722000BDE8F0810004024070B501220D4D540309
:1072300021462846FCF715FA0122960331462846D6
:10724000FCF70FFA002221462846FCF70AFA0A202A
:1072500007F0AFF931462846BDE870400022FCF740
:1072600000BA00000004024070B5104D4FF4804495
:10727000002221462846FCF7F4F966100022314628
:107280002846FCF7EEF90A2007F093F9012221467F
:107290002846FCF7E6F9012231462846FCF7E1F9D9
:1072A000BDE870400A2007F084B9000000040240E5
:1072B0002DE9F0410122154D5603002431462846A0
:1072C000FCF7CFF9062007F074F90122970339463D
:1072D0002846FCF7C6F9062007F06BF908E0641CA5
:1072E000E4B2FA2C04D9FFF7BFFF0120BDE8F0811A
:1072F00031462846FCF7ACF90028F0D10022394687
:107300002846FCF7AEF90020F0E700000004024038
:1073100010B5F9F733FD0B4CB4F86000012804D127
:107320000020A4F8600003F0A5FB2088A0F5AA4186
:10733000AA3902D1E088002803D1BDE8104003F04B
:1073400099BB10BD0E0D002010B5FAF719F90028F1
:1073500001D04FF0FF3010BDFAF7B4BF10B50022D6
:107360000F210248FEF724FB002010BD7879002091
:1073700010B5FFF7F1FF0649012806D0054800784F
:1073800008B14FF40840086010BD4FF40800FAE758
:107390009C020020E100002008B55721202000F0C9
:1073A0006BF80321212000F067F84021222000F033
:1073B00063F80821232000F05FF8AA21302000F0B4
:1073C0005BF8084801210187322000F055F80221BE
:1073D000332000F051F8684600F006F80A2007F064
:1073E000E8F808BD0E0D002010B501460F2000F092
:1073F00021F8002800D0012010BD10B50446FFF789
:1074000013FF3220FFF7DCFEFFF752FFE0B2FFF779
:10741000D7FEFFF74DFFFFF707FF3320FFF7D0FE42
:10742000FFF746FF0020FFF797FE0446FFF71CFF1B
:10743000204610BD10B50C46FFF7DFFF207001207D
:1074400010BD70B50D460446FFF7EEFE3220FFF783
:10745000B7FEFFF72DFFE0B2FFF7B2FEFFF728FF00
:107460002846FFF7ADFEFFF723FFFFF7FDFEBDE85F
:1074700070400A2007F09DB810B5FFF7E2FF012029
:1074800010BD00007FB512481049002401604FF480
:107490008031C0E90114046184610E490462C0E9CD
:1074A0000A140125C460C56145610463FBF75CFDF6
:1074B00000B1FEE70A20CDE90005694602940448C0
:1074C000FBF7ACFC002800D0FEE77FBD00200140A8
:1074D000587B00200100000F214808B5016841F4E5
:1074E00080010160016801F480010091016841F4AC
:1074F000001101600068002200F4001000901146A5
:107500001020FCF73DF91020FCF72FF9002211465E
:107510001120FCF735F91120FCF727F9002211465C
:107520003920FCF72DF93920FCF71FF9002211460C
:107530003A20FCF725F93A20FCF717F9002211460A
:107540004520FCF71DF94520FCF70FF900221146F4
:107550004620FCF715F9BDE808404620FCF705B9C0
:10756000303802402DE9F041434886B000240168DC
:1075700041F004010160016801F004010591016816
:1075800041F080010160016801F08001059101680E
:1075900041F001010160016801F0010105910168FC
:1075A00041F0020101600068344E00F002000590D5
:1075B000012212213046FCF754F8314F01221021EC
:1075C0003846FCF74EF8DFF8BC80002240F2A521D7
:1075D0004046FCF746F8012246F20A014046FCF715
:1075E00040F80022B1143846FCF73BF84FF4005045
:1075F000CDE90004694638460294FBF765FF012592
:1076000021480095CDE9010469463046FBF75CFF4F
:1076100012200090CDE90154694630460394FBF7EF
:1076200053FF41F210000090CDE9015469463846FD
:107630000394FBF749FF40F2AF200090CDE90154DD
:10764000694640460394FBF73FFF4FF4C04000906B
:107650001120CDE901040320039069464046FBF761
:1076600033FF5020CDE90004694640460294FBF701
:107670002BFF06B0BDE8F081303802400000024028
:1076800000080240000402400000111070B5244DB3
:1076900086B02248286000212846FCF7C7FB43F249
:1076A000F226B04238D000247F20C5E90140FF20F7
:1076B000C5E903046C612846AC61FCF7A9FC00B184
:1076C000FEE78DF800408DF801408DF802400394EC
:1076D0000122694612480494FCF76CFD00B1FEE7F4
:1076E00001208DF814008DF815008DF81600024663
:1076F0008DF8174005A90A48FCF7F8FC00B1FEE731
:10770000002211460648FCF79BFB00B1FEE732461B
:1077100000210348FCF78FFB06B070BD0028004035
:10772000A07B00200E4810B50C4901604FF4827117
:10773000416000218160C1604FF400720161C0E9C5
:1077400005120822C0E90721416281620A21C16253
:10775000FCF7C3FD002800D0FEE710BD003001405B
:10776000C07B002010B5134886B0114901604F213D
:107770000024C0E901144FF47A71C0E90314FDF745
:10778000E1F800B1FEE74FF48050009069460948E7
:10779000FDF71EF900B1FEE7049404A9054805941D
:1077A000FDF7A8F8002800D0FEE706B010BD0000E5
:1077B00000040040187C0020FEE7000000487047ED
:1077C000FC35002000487047DC3500200048704739
:1077D000EC35002000487047113600200249002394
:1077E0000A5C0B5410467047A40100200249002394
:1077F0000A5C0B5410467047A7010020034A10B5DD
:10780000D3690BB1126A9847002010BD9C0100207B
:10781000034A012111540021D21C1154084670471B
:10782000A4010020034A012111540021D21E115449
:1078300008467047A701002010B548B1064A01214B
:107840005170024680210548FFF747FB002010BD1C
:107850004FF0FF3010BD00009C01002011360020C9
:107860000249002248784A70704700009C010020BD
:107870000020704710B50C46152907D20A4601466C
:107880000348F8F737FD024900200855002010BDD5
:10789000FC35002010B5022902D24FF0FF3010BD98
:1078A0008C1E102C07D2014622460448F8F722FD10
:1078B000024900200855002010BD0000DC350020E2
:1078C00010B5022902D24FF0FF3010BD8C1E102CD3
:1078D00007D2014622460448F8F70CFD0249002071
:1078E0000855002010BD0000EC350020024AC2E916
:1078F00007010020704700009C010020024900227F
:1079000008780A70704700009C01002070B5044C94
:107910000546A2690AB1616990470020256170BDE2
:107920009C01002070470907090E002806DA00F0C4
:107930000F0000F1E02080F8141D704700F1E020F6
:1079400080F8001470470000BFF34F8F05480168AE
:10795000054A01F4E06111430160BFF34F8F00BF9E
:10796000FDE700000CED00E00400FA052DE9F04F02
:1079700085B00A2007F0BFF8FE4CA08F80B207F058
:10798000CBF80025A570FC48E065E07B0C2801D30E
:107990000B20E073F948FA4EE57000783071F94831
:1079A000F9490078097840EA4100217D40EA8100E8
:1079B000F071E06AF070010A3172401CE062607997
:1079C000B074420006F1B401A1F1A1008046F8F7BD
:1079D00091FC6079042101EB800206EB400006F582
:1079E0008A711330F8F786FC6079022707EB4002B2
:1079F00000EB400006EB400006F506711730F8F783
:107A000079FCB4F92600DFF884B318B1BBF8501044
:107A10000844E0846079E28C06EBC001B246A1F82C
:107A20001920D749B0744200B4314046F8F762FCDF
:107A300006207072D6484FF01C0800220078B07201
:107A4000A07E3073CE48A18B7438A0F87510617990
:107A500008EBC100CA4907F02AF9617908EBC100B7
:107A6000002107F035F9022007F082F8F5716574FE
:107A700025730126A6736573E5706079F8F78EFEAD
:107A80009FEDC41B53EC112BF8F796FD41EC100B46
:107A900003F09EFB9FEDC11B51EC100B53EC112B1F
:107AA000F8F7E3FCF8F7B2FEE18BC0B201EB40104F
:107AB00080B22084B0F5004F02D3A0F500402084AE
:107AC000B848A0642079401C2071FEF71FFFA06316
:107AD000B7E100BFFEF71AFFA16B401A052802D9D3
:107AE00009E0DFF8C49200210F2006F092FF10EAAF
:107AF000090F2063EED0206B411C22D0A046400429
:107B00007ED54FF4814200210F2007F0A2F84FF4F8
:107B10007A7007F001F8002006F0C0FF0021102065
:107B200006F077FF00F07F01954800225030C8F83A
:107B3000541006F09EFF92485030417A0729C7D171
:107B400001E0FFF701FF02229849401DF8F74DFCC4
:107B50000028BDD107F01EFAC8E91A0107F007FA9C
:107B6000C8E91C0198F80300401C88F80300844809
:107B70000C30B0F84500ADF800000090B8F81C10CB
:107B8000884278D17E48DFF828820C3030F8522FB6
:107B9000A8F800204088208306F0FEFED4E91C01EE
:107BA000844A821841F10000010641EA122929F0B5
:107BB0000100010E0002C4E91E017148D4E91A2334
:107BC0000A3007F0FAF86079D4E91C230AEB800048
:107BD000163007F0F2F86A48D4E91E23123007F095
:107BE000ECF86748082150308AF80910C17C09096F
:107BF000E17415D002226D49401DF8F7F6FB00E054
:107C000010E168B966748AF8076094F854005C491A
:107C10001638C2B26631A27401F1EA00F8F76AFBC5
:107C200061794FF01C0A0AEB81000022544907F0E9
:107C30003EF861790AEB8100002107F049F84846D7
:107C400006F054FF012006F093FFA07202215A486B
:107C5000FBF7FEFC80B100214A48017048490C3115
:107C600001F58472D1F84E006064A0641060626D0A
:107C70001C2A03D015E04CE00121EDE731F85A2F22
:107C80004E4B228549889981904209DD002807DD05
:107C900032B1E27D511CE175052A02D9277000E05E
:107CA000E5754749884200D0257126736673208B9D
:107CB0004FF47A7100F5E17080B2208388420CD3D2
:107CC000A0F2E7302083B8F80020521C92B2A8F846
:107CD00000208A4201D3A8F80050B8F8000000EB59
:107CE0004001C1EBC010218B01EBC000E06400F04B
:107CF00027F9A07A30B1ABE0FEF708FEA16B401A7D
:107D0000052805D800210F2006F083FE0006F3D5D4
:107D10009EE0FAF767FD294A8146C83A0321A2F599
:107D20009C7302F80910D3F84E00C8F84400D8F844
:107D300054101C2905D1D43202EB4902B3F85C106F
:107D400051800F49E43101EB8902B3F858101180DA
:107D50001A49F83901EB89014860D8E91C230AEB7C
:107D60008900163007F029F8D8F85C10D8F84400DC
:107D7000884227E0280000203F420F000801002031
:107D8000E00A00200A000020080000200E0D00205C
:107D9000F0000020B81E85EB51B8CE3F0000000077
:107DA00000000040A086010000D027240001002030
:107DB0000401002000008E0300040240EC0C0020AF
:107DC000FFFF010008DA5B4951F82910012903D1AE
:107DD000C8F85C0000990491BBF82230009A9342E5
:107DE0000CD1BBF814104246814205DD1572D179E1
:107DF000491C88F8071001E088F807504D4951F8F0
:107E0000291081421DDD01291BDD002819DD88F8BC
:107E100006500098A8F81C0088F80B50032088F83A
:107E200000000EE04A4600210F2006F012FF98F8ED
:107E3000050098F80310401C814202D0002006F093
:107E40002DFEFEF763FDA16B401A0528FFF449AE35
:107E5000207B012800D0277306F09EFD364A0021C2
:107E60000F2006F0F6FE207960B1052800D92770B2
:107E7000607C58B32F496C310B7848788A78022B94
:107E800014D023E0A06CE16D323881420CDAA17984
:107E90002046491CC9B2A1710229E9D904998183FC
:107EA000C57203212170E3E7A571E1E7182815D019
:107EB00010280BD0C82809D2602822D05844C91CE9
:107EC000F8F718FA11F044FB02F0D4FD194B00202A
:107ED000303B2178627903F118051EE0C878174E0F
:107EE0000D46012804D130780028EFD100F076F853
:107EF000E8780028EAD130780128E7D1F8F7F6FFD2
:107F0000E4E72670E2E700BF33F8106035F8107040
:107F1000BE4200D00221401CC0B29042F4D3217076
:107F200005B0054ABDE8F04F803200210F2006F071
:107F300090BE0000C40B002000D02724E1000020E8
:107F40002DE9F04F1F4900224FF47A7C8A751E4AB2
:107F5000DFF87890DFF87CA015680A464FF0640BD4
:107F6000548B1B4A17881C4A16881EE002FB0743E5
:107F70009BB2AAF8003003EB43080BEB08134FF059
:107F8000640803FB08F30B66A3F51C53103B9842EF
:107F900009D20A6E101A4866B0FBFCF04119C9F804
:107FA0000010BDE8F08F521C8A758A7DB242DDD97F
:107FB00004EB440242F2747303EB021264235A434B
:107FC0000A66E7E728000020840200201C00002049
:107FD000FA00002006010020F0000020064910B53C
:107FE0000120487000F0ACF90122BDE810401103F7
:107FF0000248FBF736BB0000E00000200000024012
:10800000704700002DE9F05F4FF000080A2006F0ED
:1080100072FD4FF47A7006F07FFDB44CC146B4494E
:1080200084F802906163E26A4FF0030B521CE26233
:1080300084F81590AF4DB04E8A462DE1AF4984F8D3
:1080400005B0B04A09782971AD49127858460978C7
:1080500041EA4201227D41EA8201E971A18DE97084
:10806000090A2972A849A8740622A1F28D10F8F70E
:1080700041F9A0481022193000F2AF11F8F73AF98F
:10808000B6F85000E18C00220844E0849948E18C65
:10809000A0F825109C490A20687228319B4841F8B5
:1080A00027A094490078A872A07E28736F701C27BF
:1080B0002E2006F0FCFD6079002100EB400007EB6C
:1080C000400006F005FE022006F052FD904F002110
:1080D0000F2006F09EFC38422063F8D0206B411C34
:1080E00018D040047ED54FF4814200210F2006F0C5
:1080F000B0FD0021102006F08CFC00F07F017D48CF
:108100000022503006F0B5FC7A485030417A0229FE
:1081100002D0B9E0FFF718FC02227E49401DF8F7B3
:1081200064F900287DD106F035FFC4E91A0106F094
:108130001EFFB8F1000FC4E91C013BD16D49764820
:108140000C314FF0010831F8522F0280498801F5B7
:10815000E17189B22183B1F57A7F0CD3A1F2E731C5
:108160002183018840F2F232491C89B20180914298
:1081700001D3A0F800900088238B00EB4002C2EBF3
:10818000C01203EBC202E264644A01460A38138853
:1081900000B2DAB22274A084002802DA00F57A7004
:1081A000A084521E934201D1012060736184608BD0
:1081B00000F09AFD4F48627D0C3005EB420130F82B
:1081C000453FA1F813304B4BD0F80910743B0768BA
:1081D000C3F8237003F50F7343F82210283B03EB19
:1081E000420200E07BE000881080626B914202D284
:1081F0006163A4F85800D4E91C01494A801841F190
:108200000001070A47EA0167384606F06FFC27F0CD
:108210000100010E0002C4E91E0136484F464838ED
:1082200000E031E0D4E91A2306F0C7FD3148D4E973
:108230001C23443806F0C1FD2E48D4E91E234038E3
:1082400006F0BBFD2B49002252393C2006F02FFDE1
:1082500000213C2006F03CFD012006F089FC10F0D6
:10826000FF00A072A17801F10101A17005D10021E8
:108270000F2006F0CEFB0006F9D5802200210F204A
:1082800006F0E7FC677001E001206070012006F055
:108290008BF9607D401C60753089677DB8423FF680
:1082A000CDAE616B514506D084F80B9084F800B0D8
:1082B000B4F85800A083B8F1000F0ED1608B1949B3
:1082C00010B10A88904201D908886083164980B2AB
:1082D000401E0988484315490880BDE8F09F144AAC
:1082E00000210F2006F0B5FCCEE70000280000209A
:1082F000FFFF0100E00A00200E0D0020DC0000203E
:108300000A00002008000020800C0020F00000205F
:1083100000D027240001002004010020F8000020E4
:1083200000008E03EC000020EA000020E80000209E
:108330000090272410B50020FFF76AFA002010BD36
:1083400010B50020FFF76EFA002010BD10B5002117
:108350000248FFF7CBFA002010BD0000618302083D
:108360000148026070470000B4000020010901EBE1
:10837000810100F00F0000EB4100C0B27047002106
:1083800002E00A38C0B2491C0A28FAD2090740EABA
:108390001160704770B504460068C168490614D47E
:1083A0004FF0FF31C160FBF761F905464FF47A7673
:1083B00007E000BFFBF75AF9401BB04201D9032088
:1083C00070BD2068C0684006F4D5002070BD000074
:1083D00070B5154D86B00446002269462868FBF743
:1083E000EBFD4FF0FF3628B9002205A92868FBF7FE
:1083F000C1FD10B1304606B070BD9DF8170000F504
:10840000FA6020809DF81500A0709DF81600E070BD
:108410009DF8000020719DF8010060719DF8020038
:10842000A0710020E7E70000340100200149086046
:1084300070470000340100200148FBF77FBD0000B9
:10844000A07B002008B540B10246074800210091FA
:10845000044B0068FEF718FB08BDBDE8084000208B
:1084600000F004B86D84020894020020044972B63A
:1084700002480860BFF34F8F704700000400FA0500
:108480000CED00E02DE9F84F0120C827B7FBF0F113
:10849000DFF8DCA1DFF8DCB1774CAAF80000ABF81C
:1084A0000010607A401C6072C00705D0608B411ECE
:1084B0006183022800D26783608B00F015FC0A20DC
:1084C00006F019FB4FF47A75284606F025FB0221C9
:1084D0006A48FBF7BDF878B30020694980006B4E0D
:1084E0000978A94640EA4101664800780143664898
:1084F000817210214172F288B5FBF2F14173644937
:1085000000220978817374387188A0F87F1000F117
:1085100080084046318F20F8031F718F41805A49EF
:10852000152006F0C4FB0021152006F0D1FB022027
:1085300006F01EFB574D05E0FFE70120CDE700BF29
:10854000FEF7E6FE00210F2006F063FA28422063C2
:10855000F6D0208E40047DD54FF4814200210F20BB
:1085600006F077FB0021102006F053FA00F07F019F
:10857000454800225030616506F07BFA424D503587
:10858000687A11286AD102224349681DF7F72DFF46
:10859000002863D1B8F84510ADF80010AA7AAAF8FF
:1085A0000020B7FBF2F3B9FBF2F2ABF800302B7B03
:1085B00063834046394BF280B0F852601E80B0F8B9
:1085C0005400CC4600F5E17080B25146D846208375
:1085D00060450CD3A0F2E7302083188840F2F236D1
:1085E000401C80B21880B04201D300201880188847
:1085F000BCFBF2F200EB4003C3EBC010238B03EB98
:10860000C000E0640A80B7FBF2F1A8F80010FFF7A1
:1086100097FCBDF80000A083A87C1B496071633102
:1086200042000D4601F15100F7F764FE60792946DA
:1086300042001548CC30F7F75DFE608BFF2808D16B
:108640001748B8F800100068B0FBF1F201FB120007
:10865000608301E004E001E003202070BDE8F88FB2
:108660002A46BDE8F84F00210F2006F0F2BA0000BC
:10867000F0000020FA000020280000200004024042
:10868000E4000020E5000020E00A00200E0D00209C
:10869000A002002000D027240001002004010020B7
:1086A000840200202DE9F05F06460F4614461D4661
:1086B000324620462946F7F7FAFD80468946402093
:1086C000821B20462946F7F7E3FD82468B4648EA9F
:1086D0000A0049EA0B01BDE8F09F70B5054600F0BD
:1086E00026FA4FF0FF34C0B9284600F025F80022E2
:1086F000C721284600F0ACF90028284602D000F037
:108700000FF80AE000F00CF8284600F001FA20B952
:10871000284600F0ABF9002800D0204670BD0000CC
:1087200000EB80010348012200EBC1000189406891
:10873000FAF797BFB435002000EB80010348002210
:1087400000EBC10001894068FAF78BBFB435002007
:108750002DE9F0470C46804600EB880116480025BD
:1087600000EBC1001F46406A1646A0420BD956B125
:10877000A119814207D8114A52F82710491E2142F7
:1087800001D1032F03D34FF0FF30BDE8F08774B958
:10879000B0420CD84046FFF7A0FF0BE061193A4603
:1087A000404600F011F959F82700054400E09146D1
:1087B000B542F3D30020E8E7B435002080A20308D7
:1087C00038B504460322694600F0D1F84FF0FF3572
:1087D00088B99DF80000FF280FD19DF80100FF28FF
:1087E0000BD19DF80200FF2807D1032269462046DD
:1087F00000F0BDF808B1284638BD9DF802300C4A9B
:1088000004EB84004FF4800102EBC000152B05D06F
:10881000162B03D0172B04D0182B05D04162002053
:1088200038BD4FF40001F9E74FF08071F6E7000022
:10883000B43500202DE9F0478246C8B20025C0F5C6
:108840008074089F90460E469C4200D91C465046B4
:1088500000F00CF94FF0FF3960BB504600F067F9AB
:1088600040BB5046FFF768FF00220221504600F04F
:10887000EFF8E0B90022C6F30741504600F0E8F8EF
:10888000A8B90022C6F30721504600F0E1F870B9FC
:10889000F1B20022504600F0DBF840B90CE000BF16
:1088A00018F805100022504600F0D2F818B15046D2
:1088B000FFF736FF0DE06D1CA542F1D35046FFF7E0
:1088C0002FFF504600F024F918B9504600F0CEF8BA
:1088D00010B14846BDE8F08707B13C600020F9E7D9
:1088E00010B500EB8004044800EBC40000EBC100AD
:1088F0004260038110BD0000B43500202DE9F04135
:108900001E4615460F4680460024FFF715FF00223D
:108910000321404600F09CF8D0B90022C5F307417E
:10892000404600F095F898B90022C5F3072140466B
:1089300000F08EF860B9E9B20022404600F088F8F5
:1089400030B90DE03A19FF21404600F081F830B10E
:108950004046FFF7E5FE4FF0FF30BDE8F081641CB4
:10896000B442EFD34046FFF7DBFE0020F5E72DE9E8
:10897000F04115460E4607460024FFF7DDFE0022B3
:108980009F21384600F064F830B90DE03219FF211C
:10899000384600F05DF830B13846FFF7C1FE4FF0C1
:1089A000FF30BDE8F081641CAC42EFD33846FFF7DE
:1089B000B7FE0020F5E70000024A00EB800002F855
:1089C00030107047B43500202DE9F04107461F48AC
:1089D000154650F82500401E21EA0004384600F0F4
:1089E000A6F84FF0FF3608BB3846FFF7A5FE17483C
:1089F0000022001F415D384600F02AF898B9002295
:108A0000C4F30741384600F023F860B90022C4F3EC
:108A10000721384600F01CF828B9E1B20022384698
:108A200000F016F818B13846FFF77AFE0BE038462A
:108A3000FFF776FE384600F06BF820B9384600F0B4
:108A400015F8002800D03046BDE8F08180A2030868
:108A500007B51146044A00EB8000012312F83000EC
:108A600001AA00F083F80EBDB4350020F8B5054624
:108A700000208DF800006E462846FFF75DFE0022BC
:108A800005212846FFF7E4FF040005D13246FF2107
:108A90002846FFF7DDFF04462846FFF741FE200089
:108AA00003D19DF80010C907E5D1F8BD2DE9FC41BF
:108AB0008046002001900D46144808EB880100EB29
:108AC000C1001C46406A16464FF0FF37A84212D933
:108AD0008EB184B10146401E2840081AA04201D23E
:108AE00004460FE001A8009023463246294640463E
:108AF000FFF7A0FE10B13846BDE8FC81019805449F
:108B00000644241A002CEDD10020F5E7B4350020EE
:108B100070B50546FFF710FE002204212846FFF736
:108B200097FF04462846FFF7FBFD204670BD70B551
:108B30000546FFF701FE002206212846FFF788FFC1
:108B400004462846FFF7ECFD204670BD38B50B46BD
:108B5000009204460022802100F02AF8002804D068
:108B6000606D40F020006065032038BD38B51446C4
:108B700069B1642503FB05F20092084A9BB252F8E2
:108B800020000A462146FBF76BFD002038BD1A463F
:108B90002146BDE8384000F057B800008C020020A4
:108BA000024A42F820100020704700008C0200208A
:108BB0002DE9F0411D4617460E460446DDF81880A3
:108BC00035E0681C33D02DB1FAF750FDA0EB08005A
:108BD000A8422CD32068416821F0E0014160606820
:108BE000B0F5827F0BD1A068B0F5004F02D0B0F590
:108BF000806F04D12068016821F040010160A06A03
:108C0000B0F5005F0AD1206801684DF6FF7211408F
:108C100001602068016841F400510160012084F87E
:108C20005100002084F850000320BDE8F081206846
:108C3000806836EA000004D00020B842C1D100208C
:108C4000F3E70120F9E7000010B5054C6423534316
:108C500092B254F82000FBF74FFC002010BD00003A
:108C60008C02002070470000F8B5044600201B4D20
:108C7000ADF8000055222A70AA226A700322AA7059
:108C8000661DEE702A716971154AAC7102EB4101E3
:108C90002246E81DF7F72EFB002007E02918BDF853
:108CA00000208978401C1144ADF80010B042F5DB7B
:108CB000611DA81CF8F70DF9ADF800002819BDF8E2
:108CC0000010A0F8071001B004F10902BDE8F0405F
:108CD0004FF47A7301490348FCF7A1BA72110020DE
:108CE0000E0D0020547C00207047000010B50228B3
:108CF0000FD0FDF779FD50B1FDF776FDD0F8900566
:108D000028B1FDF771FDD0F8901504A08847002028
:108D100010BD4868FEF790FDF9E700004552524F3C
:108D2000520D0A0010B50220FEF772FDFDF75CFD42
:108D300050B1FDF759FDD0F8900528B1FDF754FD6D
:108D4000D0F8901501A08847002010BD4F4B0D0AA8
:108D50000000000010B50C4602280DD0FDF744FDC0
:108D600050B1FDF741FDD0F8900528B1FDF73CFD6D
:108D7000D0F8901527A088476068F7F769FB98B18D
:108D8000012824D0022832D0FDF72EFD50B1FDF786
:108D90002BFDD0F8900528B1FDF726FDD0F89015F1
:108DA0001DA08847002010BD0020F8F781F9FDF7CD
:108DB0001BFD0028F6D0FDF717FDD0F89005002820
:108DC000F0D0FDF711FDD0F8901515A0E9E7FDF7FB
:108DD0000BFD50B1FDF708FDD0F8900528B1FDF767
:108DE00003FDD0F890150EA0884701200EE0FDF796
:108DF000FBFC50B1FDF7F8FCD0F8900528B1FDF769
:108E0000F3FCD0F8901506A088470220F8F750F937
:108E1000C8E70000417267204552524F520D0A00C8
:108E20004F4B0D0A0000000010B54868F7F710FB23
:108E30004FF47A71B0FBF1F10A036421B0FBF1F356
:108E40000A21B3FBF1F401FB143302EB0322B0FB64
:108E5000F1F3B3FBF1F401FB143302EB0312B0FBAB
:108E6000F1F301FB13000C49104480B288800B49D8
:108E7000086010F06DFBFDF7B7FC50B1FDF7B4FCD6
:108E8000D0F8900528B1FDF7AFFCD0F8901504A0FC
:108E90008847002010BD00000E0D002000010020BA
:108EA0004F4B0D0A0000000010B5022810DAFDF744
:108EB0009BFC50B1FDF798FCD0F8900528B1FDF768
:108EC00093FCD0F8901503A088474FF0FF3010BDF9
:108ED000002010BD64656275675F6F666620666C12
:108EE00061670D0A0000000010B5022810DAFDF7D6
:108EF0007BFC50B1FDF778FCD0F8900528B1FDF768
:108F000073FCD0F8901503A088474FF0FF3010BDD8
:108F1000002010BD64656275675F6F6E20666C61CE
:108F2000670D0A0010B50C4602280DD0FDF75CFC59
:108F300050B1FDF759FCD0F8900528B1FDF754FC6D
:108F4000D0F890150CA088476068F7F781FA0146C1
:108F5000022001F0A3FEFDF747FC50B1FDF744FCF1
:108F6000D0F8900528B1FDF73FFCD0F8901505A08A
:108F70008847002010BD0000417267204552524FC3
:108F8000520D0A004F4B0D0A0000000010B5FDF70E
:108F90002BFC58B1FDF728FCD0F8900530B1FDF757
:108FA00023FCD0F8902525A126A09047FDF71CFCB6
:108FB00058B1FDF719FCD0F8900530B1FDF714FC5D
:108FC000D0F8902525A128A09047FDF70DFC70B1A1
:108FD000FDF70AFCD0F8900548B1FEF7F3FB044614
:108FE000FDF702FCD0F89025214625A09047FDF71B
:108FF000FBFB70B1FDF7F8FBD0F8900548B1FEF728
:10900000DDFB0446FDF7F0FBD0F89025214622A0B9
:109010009047FDF7E9FB70B1FDF7E6FBD0F890054E
:1090200048B1FEF7D3FB0446FDF7DEFBD0F89025F0
:1090300021461FA09047002010BD00007178777A6C
:109040000000000041707020547079653A202020A3
:10905000202020202025730D0A00000056323032D7
:10906000313035313030300056657273696F6E3A89
:1090700020202020202020202025730D0A00000021
:10908000494D45493A202020202020202020202022
:109090002025730D0A000000434349443A20202054
:1090A00020202020202020202025730D0A000000F1
:1090B000494D53493A2020202020202020202020E4
:1090C0002025730D0A00000010B51E210248FDF78F
:1090D00005FB002010BD00008CA1030810B502287C
:1090E00010D0FDF781FB50B1FDF77EFBD0F8900565
:1090F00028B1FDF779FBD0F890150AA088474FF00A
:10910000FF3010BDFDF770FB50B1FDF76DFBD0F8DF
:10911000900528B1FDF768FBD0F8901506A08847A8
:10912000002010BD75736167653A206C6F6720730E
:109130007472696E670D0A004F4B0D0A0000000043
:1091400010B5FDF751FB50B1FDF74EFBD0F890057F
:1091500028B1FDF749FBD0F8901502A08847002000
:1091600010BD00004F4B0D0A0000000010B5032891
:1091700010D0FDF739FB50B1FDF736FBD0F8900564
:1091800028B1FDF731FBD0F8901503A088474FF0C8
:10919000FF3010BD002010BD75736167653A206C0B
:1091A0006F675F7072696E74206173635B302D311D
:1091B0005D20636E740D0A000020704738B50C46C0
:1091C000022810D0FDF710FB50B1FDF70DFBD0F8D1
:1091D000900528B1FDF708FBD0F8901519A0884735
:1091E0004FF0FF3038BD4CF6CC40ADF800001AA06F
:1091F000FCF726FB00234FF4883502222946184647
:10920000FFF7A6FA02236A4629460020FFF74EFC24
:1092100000234FF490354FF4807229461846FFF72B
:1092200097FA6068F7F7CCF8431C2946002062687B
:10923000FFF73CFC0A2005F0B7F90020FFF702F920
:10924000002038BD75736167653A206F74612075C1
:10925000726C0D0A00000000676F746F206F7461FC
:10926000206170706C69636174696F6E0D0A000033
:1092700010B50220FEF7D6FAFDF7B6FA50B1FDF7A9
:10928000B3FAD0F8900528B1FDF7AEFAD0F89015F2
:1092900001A08847002010BD4F4B0D0A00000000C0
:1092A00010B50020FEF7B4FAFDF79EFA50B1FDF7B5
:1092B0009BFAD0F8900528B1FDF796FAD0F89015F2
:1092C00001A08847002010BD4F4B0D0A0000000090
:1092D00010B50020FEF7A6FAFDF786FA50B1FDF7AB
:1092E00083FAD0F8900528B1FDF77EFAD0F89015F2
:1092F00001A08847002010BD4F4B0D0A0000000060
:1093000010B5022810D0FDF76FFA50B1FDF76CFAD6
:10931000D0F8900528B1FDF767FAD0F890150AA0AB
:1093200088474FF0FF3010BDFDF75EFA50B1FDF7F2
:109330005BFAD0F8900528B1FDF756FAD0F89015F1
:1093400008A08847002010BD75736167653A2072D8
:1093500074635F7365745F616C61726D20736563C4
:109360000D0A00004F4B0D0A00000000002070475E
:1093700010B5072810D0FDF737FA50B1FDF734FAD1
:10938000D0F8900528B1FDF72FFAD0F8901503A07A
:1093900088474FF0FF3010BD002010BD7573616726
:1093A000653A207274635F736574207979797920E6
:1093B0006D6D206464206868206D6D2073730D0AE4
:1093C0000000000010B50020FFF73CF8002010BDA1
:1093D00010B50C46052810DAFDF706FA50B1FDF776
:1093E00003FAD0F8900528B1FDF7FEF9D0F89015F2
:1093F0001BA088474FF0FF3010BD1BA220211B4847
:10940000636801F059FE194817A220212030A36893
:1094100001F052FE154814A220214030E36801F00B
:109420004BFE124810A220216030236901F044FE57
:1094300010F08EF8FDF7D8F950B1FDF7D5F9D0F856
:10944000900528B1FDF7D0F9D0F8901508A088470D
:10945000064901207C39A1F86000002010BD000001
:109460004552524F520D0A00257300008A0D00200C
:109470004F4B0D0A0000000038B50D46032810DAE6
:10948000FDF7B2F950B1FDF7AFF9D0F8900528B16A
:10949000FDF7AAF9D0F8901528A088474FF0FF30C3
:1094A00038BD69466868FDF7DBFB264C9DF8000077
:1094B000B4F87210884211D19DF80110B4F87420EC
:1094C00091420BD19DF80210B4F87620914205D15B
:1094D0009DF80310B4F8782091420DD0A4F87200E2
:1094E0009DF80100A4F874009DF80200A4F876002D
:1094F0009DF80300A4F87800A868FDF726FDB4F8ED
:109500007A10884204D0A868FDF71FFDA4F87A00FD
:1095100010F01EF8FDF768F950B1FDF765F9D0F8C5
:10952000900528B1FDF760F9D0F8901506A088479E
:109530000120A4F86000002038BD00004552524FC1
:10954000520D0A000E0D00204F4B0D0A00000000C6
:1095500038B50D46032810DAFDF746F950B1FDF78E
:1095600043F9D0F8900528B1FDF73EF9D0F89015F1
:1095700028A088474FF0FF3038BD69466868FDF77E
:109580006FFB264C9DF80000B4F86610884211D19C
:109590009DF80110B4F8682091420BD19DF802109B
:1095A000B4F86A20914205D19DF80310B4F86C20FC
:1095B00091420DD0A4F866009DF80100A4F868005F
:1095C0009DF80200A4F86A009DF80300A4F86C005E
:1095D000A868FDF7BAFCB4F86E10884204D0A868F9
:1095E000FDF7B3FCA4F86E000FF0B2FFFDF7FCF836
:1095F00050B1FDF7F9F8D0F8900528B1FDF7F4F86F
:10960000D0F8901506A088470120A4F8600000203B
:1096100038BD00004552524F520D0A000E0D002079
:109620004F4B0D0A000000000020704701A0FCF71E
:1096300007B900004576656E743A25750D0A00007D
:1096400010B50C4602280DD0FDF7CEF850B1FDF74D
:10965000CBF8D0F8900528B1FDF7C6F8D0F89015F2
:1096600013A088476068F6F7F3FE00F037F978B189
:10967000FDF7BAF850B1FDF7B7F8D0F8900528B16A
:10968000FDF7B2F8D0F890150AA08847002010BD69
:10969000FDF7AAF80028F9D0FDF7A6F8D0F8900554
:1096A0000028F3D0FDF7A0F8D0F8901503A0ECE760
:1096B000417267204552524F520D0A004F4B0D0A1E
:1096C0000000000070B50C4604280DD0FDF78CF8A2
:1096D00050B1FDF789F8D0F8900528B1FDF784F86E
:1096E000D0F8901517A088476068F6F7B1FE0646D7
:1096F000D4E90250F6F7ACFE82B22946304600F0BB
:1097000029F978B1FDF770F850B1FDF76DF8D0F890
:10971000900528B1FDF768F8D0F890150AA08847A1
:10972000002070BDFDF760F80028F9D0FDF75CF867
:10973000D0F890050028F3D0FDF756F8D0F8901532
:1097400003A0ECE7417267204552524F520D0A00C8
:109750004F4B0D0A0000000008B5002003460090A2
:109760001A4A0121684600F015F978B1FDF73CF876
:1097700050B1FDF739F8D0F8900528B1FDF734F86D
:10978000D0F8901512A08847002008BDFDF72CF8EE
:1097900058B1FDF729F8D0F8900530B1FDF724F85D
:1097A000D0F890250CA000999047FDF71DF80028EF
:1097B000EAD0FDF719F8D0F890050028E4D0FDF7BD
:1097C00013F8D0F8901507A0DDE700002D960208E9
:1097D0004552524F520D0A00536F636B49443A256C
:1097E000750D0A004F4B0D0A0000000070B50C46C5
:1097F00003280DD0FCF7F8FF50B1FCF7F5FFD0F8C7
:10980000900528B1FCF7F0FFD0F8901517A0884715
:109810006068F6F71DFEA46805462046F6F7D0FD01
:1098200002462146284600F0D5FA78B1FCF7DCFF65
:1098300050B1FCF7D9FFD0F8900528B1FCF7D4FF60
:10984000D0F890150AA08847002070BDFCF7CCFF27
:109850000028F9D0FCF7C8FFD0F890050028F3D015
:10986000FCF7C2FFD0F8901503A0ECE74172672027
:109870004552524F520D0A004F4B0D0A0000000096
:109880000020704738B54AF6AA20ADF80000FCF772
:10989000ABFF50B1FCF7A8FFD0F8900528B1FCF75A
:1098A000A3FFD0F890150AA0884700234FF488340E
:1098B000022221461846FEF74BFF02236A46214644
:1098C0000020FFF7F3F80A2004F06EFE002038BDF8
:1098D000757064617465204F4B0D0A00C0EB8011F8
:1098E000094AC1EB011102EB8101032808D239B109
:1098F000087818B1012801D00520087000207047B1
:109900004FF0FF3070470000943600202DE9F04101
:1099100000240F4D26460127C4EB8410C0EB001035
:1099200005EB80000178032903D0042901D0062922
:1099300007D18670077083681BB1C2680221204678
:109940009847641C032CE7DB0020BDE8F081000091
:109950009436002070B51546C0EB80120B4BC2EB5D
:10996000021203EB820403280CD25CB10B4608A25E
:109970002A2104F11000FDF7B0FA6587032020705A
:10998000002070BD4FF0FF3070BD00009436002005
:10999000257300002DE9F047814620481F46904678
:1099A0000E460025C5EB8511C1EB011110EB8104BA
:1099B00001D0217831B16D1C032DF3DB4FF0FF3066
:1099C000BDE8F08740F6C4612046FDF709F96560FF
:1099D000667002202070C4E9028710234FF4C06231
:1099E00004F1C40104F13C00FDF744FB4FF40062B4
:1099F000012E0AD0102304F2C46104F16C00FDF7BB
:109A000039FB0020C9F80050DAE7012304F2C461F1
:109A100004F1B000FBF71DFEF3E7000094360020D0
:109A2000032808DAC0EB80100449C0EB001001EBFA
:109A300080001030704702A070470000943600206C
:109A400000000000032808DAC0EB80100449C0EBD6
:109A5000001001EB8000408F70470020704700002D
:109A600094360020032808DAC0EB80100449C0EBCC
:109A7000001001EB80003C30704700207047000070
:109A800094360020032807DAC0EB80100349C0EBAE
:109A9000001011F820007047002070479436002015
:109AA000032808DAC0EB80100449C0EB001001EB7A
:109AB00080004078704700207047000094360020F6
:109AC000032808DAC0EB80100449C0EB001001EB5A
:109AD0008000807870470020704700009436002096
:109AE00003280ADAC0EB8010054AC0EB001002EB35
:109AF000800001218170002070474FF0FF307047D7
:109B000094360020C0EB80120C4BC2EB021203EB28
:109B1000820203280CD259B1107801280BD050B121
:109B2000072808D0022806D00020087000207047BF
:109B30004FF0FF3070470120F7E700009436002017
:109B4000C0EB8012094BC2EB021203EB8202032826
:109B500007D231B11078062806D000200870002006
:109B600070474FF0FF3070470120F7E79436002030
:109B700003280ADAC0EB8010054AC0EB001002EBA4
:109B8000800000218170084670474FF0FF30704719
:109B900094360020C0EB80110C4AC1EB011110B5C6
:109BA00002EB81014FF0FF3203280CD259B10B7840
:109BB000042B08D001220A708B6813B1CA680221F5
:109BC0009847002010BD104610BD000094360020BC
:109BD000C0EB80110A4A10B5C1EB011102EB810103
:109BE000032809D241B107220A708B6813B1CA68F1
:109BF00000219847002010BD4FF0FF3010BD00003D
:109C00009436002070B50546C0EB85101A49C0EBAC
:109C1000001001EB8004032D25D224B30620207010
:109C20000202102304F1C40104F13C00FDF722FA02
:109C3000C5EB8511104B6078C1EB011103EB81017D
:109C40004FF4006201F2C46101280FD0102304F127
:109C50006C00FDF70FFAA3681BB101212846E268EA
:109C60009847002070BD4FF0FF3070BD012304F114
:109C7000B000FBF7EEFCEEE794360020C0EB80115D
:109C8000094A10B5C1EB011102EB8101032807D28B
:109C900031B18B6813B1CA6803219847002010BD09
:109CA0004FF0FF3010BD0000943600202DE9F04742
:109CB000894601461746C0EB81101D4AC0EB0010D3
:109CC0001E464FF0FF3402EB8000032918D2B8B1D2
:109CD000B6B14178012916D06C308046FDF77FF986
:109CE00005000DD06A68BA4206D248462968F6F7E0
:109CF00001FB68680024306029464046FDF747F9BB
:109D00002046BDE8F0870024254600F1B0080AE0AF
:109D100009EB04014046FBF7C3FC10B1002035609D
:109D2000EFE7641C6D1CBC42F2D300243560E7E70A
:109D3000943600202DE9F04706468946C0EB861090
:109D4000C0EB00111A480025174600EB81004FF0C8
:109D5000FF38032E1ED2E8B14178012910D06C30B3
:109D600004461146FDF75AF905001AD03A4649460D
:109D70002868F6F7BFFA20462946FDF71CF914E0DB
:109D800000F1B0040AE000BF09EB05012046FBF733
:109D900043FC10B14046BDE8F0876D1CBD42F3D3D3
:109DA00003E0314603A0FBF74BFD0020F3E7000082
:109DB00094360020536F636B65745B25755D20528C
:109DC000656376204275666665722046756C6C0D1B
:109DD0000A0000002DE9F04705468846C0EB8510D3
:109DE0001249C0EB0010174601EB80004FF0FF3620
:109DF000032D13D290B13C3011468146FDF70EF988
:109E000004000DD03A4641462068F6F773FA214621
:109E10004846FDF7D0F80020BDE8F0873046FBE764
:109E2000294603A0FBF70CFDF8E70000943600205C
:109E3000736F636B65745B25645D2073656E64206E
:109E40006275662066756C6C0D0A0000032808DADE
:109E5000C0EB8010044AC0EB001002F82010002074
:109E600070474FF0FF3070479436002010B5FCF774
:109E70003DFEF9F701FCBDE81040FAF735BD0000E2
:109E800030B52B4897B00025016841F08051016042
:109E9000006800F0805016902648016821F4404187
:109EA00041F4004101600068022400F44040169033
:109EB000052000904FF48030019001200290800531
:109EC000CDE9064008200890A020CDE9090404202F
:109ED0000B906846F9F71CFE00B1FEE70CA90F20B5
:109EE00081E831004FF48050CDE90F0502210CA824
:109EF000F9F720FD00B1FEE74FF480701490119443
:109F000011A8F9F76FFC00B1FEE7F9F7ABFD4FF4CC
:109F10007A71B0FBF1F0FAF7D3FC0420FAF78CFC6D
:109F200000221146501EF9F72BFC17B030BD00007F
:109F300040380240007000401048016841F4700150
:109F400001600F48016841F0010101600C4A0021E5
:109F50000832116002680B4B1A400260031D0A4A66
:109F60001A60026822F48022026005480C30016009
:109F700002490648803908607047000088ED00E01B
:109F800000380240FFFFF6FE1030002400000208F7
:109F90000148FAF797BD0000187C0020F0B5026870
:109FA0001B4B1C4C9F031C4D1C4E984207D0B842C3
:109FB00005D0A04203D0A84201D0B04204D122F083
:109FC000700C4A6842EA0C02984210D0B8420ED097
:109FD000A0420CD0A8420AD0B04208D0104CA042F7
:109FE00005D0104CA04202D00F4CA04203D122F465
:109FF0004074CA68224302608A68C2620A68826248
:10A00000984201D10969016301214161F0BD00005D
:10A01000000001400004004000080040000C004027
:10A0200000400140004401400048014010B58468F0
:10A0300042EA032224F47F440A432243826010BD93
:10A04000826822F070020A4342F007018160704783
:10A0500010B5036A046A24F001040462846924F0E0
:10A06000F00444EA021423F00A020A438461026203
:10A0700010BD10B5036A23F0100303628369046AFC
:10A0800023F4704343EA023224F0A00343EA0111AF
:10A090008261016210BD000070B520211148F9F7FE
:10A0A000DCFA114C002525642078062817D2DFE859
:10A0B00000F0160306091406FEF7E4F90FE0FDF7B9
:10A0C000A1FF0CE0E07A401CE072F8F72BFEE07A8A
:10A0D000052804D90220207001E0FDF747FC034861
:10A0E000057070BD00040240280000200A00002016
:10A0F00010B5806B0021C185C184FAF7C6FD10BD83
:10A1000070B5846B2068406994F83910C0F3C010B2
:10A110000025212904D118B1E584204600F062F819
:10A120002068406994F83A10C0F38010222904D1C5
:10A1300018B1E585204600F047F8E06B40F01000CC
:10A14000E0632046FAF7A1FD70BD10B50146806BB3
:10A1500009680968C90513D40021C1850168CA6866
:10A1600022F48072CA6001684A6922F001024A61E1
:10A1700001684A6922F040024A61202180F83A10C1
:10A18000FBF74AF810BD10B5806BFBF747F810BD20
:10A1900010B50146806B09680968C9050CD4002117
:10A1A000C18401684A6922F080024A610068C1687E
:10A1B00041F04001C16010BDFBF7EDF810BD10B5D6
:10A1C000806BFBF7EAF810BD0168CA6822F4907250
:10A1D000CA6001684A6922F001024A61202180F8C0
:10A1E0003A1070470168CA6822F0C002CA60202194
:10A1F00080F83910704710B590F83A10222901D034
:10A20000022010BD8168B1F5805F11D0016900297D
:10A2100001681FD0496801F07F03816A4A1C82628D
:10A220000B70C18D491E0904090CC18518D026E0A8
:10A230000269816A002A0268526805D0D2B20A8097
:10A24000816A491C8162ECE7C2F308020A80816AD4
:10A25000891CF7E74A68816A4B1C83620A70E0E751
:10A260000168CA6822F49072CA6001684A6922F0E3
:10A2700001024A61202180F83A10FAF7CDFF002050
:10A2800010BD00002DE9F04104460068016921F489
:10A290004052E168114301612168C86849F20C62CB
:10A2A00090432369A268E5691A4363692B431A4303
:10A2B0000243CA602168486920F44072A0691043D3
:10A2C0004861E1696425B1F5004F9748974A2168D4
:10A2D0004FF032083FD0914201D081427CD1F9F752
:10A2E000D7FB00EBC00101EB001061688900B0FBF7
:10A2F000F1F6F9F7CDFB00EBC00101EB001061684E
:10A300008900B0FBF1F0B0FBF5F06FF018014843A5
:10A3100006EB800108EB0110B0FBF5F000F0F00651
:10A32000F9F7B6FB00EBC00101EB00106168890092
:10A33000B0FBF1F0B0FBF5F006EB0016F9F7A8FB67
:10A3400000EBC00101EB001061688900B0FBF1F780
:10A35000F9F79EFBD2E0914201D081423DD1F9F75D
:10A3600097FB00EBC00101EB001061684900B0FBF6
:10A37000F1F0B0FBF5F00601F9F78AFB00EBC00144
:10A3800001EB001061684900B0FBF1F7F9F780FBC1
:10A3900000EBC00101EB001061684900B0FBF1F077
:10A3A000B0FBF5F06FF01801484307EB800108EBB4
:10A3B000C100B0FBF5F000F0F80006EB4006F9F73D
:10A3C00067FB00EBC00101EB001061684900B0FBC6
:10A3D000F1F7F9F75DFB3CE055E0F9F749FB00EBDD
:10A3E000C00101EB001061684900B0FBF1F0B0FB67
:10A3F000F5F00601F9F73CFB00EBC00101EB0010A2
:10A4000061684900B0FBF1F7F9F732FB00EBC001DE
:10A4100001EB001061684900B0FBF1F0B0FBF5F012
:10A420006FF01801484307EB800108EBC100B0FB57
:10A43000F5F000F0F80006EB4006F9F719FB00EB29
:10A44000C00101EB001061684900B0FBF1F7F9F7BA
:10A450000FFB00EBC00101EB001061684900B0FB8D
:10A46000F1F0B0FBF5F06FF01801484307EB800105
:10A4700008EBC100B0FBF5F000F0070021683044A4
:10A480008860BDE8F081F9F7F3FA00EBC00101EB59
:10A49000001061688900B0FBF1F6F9F7E9FA00EB0A
:10A4A000C00101EB001061688900B0FBF1F0B0FB66
:10A4B000F5F06FF01801484306EB800108EB01103E
:10A4C000B0FBF5F000F0F006F9F7D2FA00EBC001AE
:10A4D00001EB001061688900B0FBF1F0B0FBF5F012
:10A4E00006EB0016F9F7C4FA00EBC00101EB00100F
:10A4F00061688900B0FBF1F7F9F7BAFA00EBC00127
:10A5000001EB001061688900B0FBF1F0B0FBF5F0E1
:10A510006FF01801484307EB800108EB0110B0FB16
:10A52000F5F000F00F00A9E7001401400010014011
:10A5300090F83910212901D0022070478168B1F5C7
:10A54000805F016A0BD04A1C026202680978516080
:10A55000C18C491E0904090CC1840ED017E009887A
:10A560000268C1F30801516001690029016A02D043
:10A57000491C0162ECE7891CFBE70168CA6822F00C
:10A580008002CA600068C16841F04001C1600020DB
:10A5900070472DE9F041984617460E460446069D41
:10A5A0001DE0681C1BD02DB1F9F760F8A0EB080086
:10A5B000A84214D92068C16821F4D071C160206814
:10A5C000416921F001014161202084F8390084F8BB
:10A5D0003A00002084F838000320BDE8F0812068AC
:10A5E000006836EA000004D00020B842D9D000202C
:10A5F000F3E70120F9E7000070B506468EB0744914
:10A6000074A0FBF71DF9082274A13046F5F703FF8B
:10A61000754C4FF0FF35A8B1082274A13046F5F70C
:10A62000FAFE00286AD0082273A13046F5F7F3FE3F
:10A6300000287CD0092273A13046F5F7ECFE0028F3
:10A6400076D0C2E00C236A462C213046FCF75CFC35
:10A6500005286ED30198FCF7F4FAA1888842F0D15E
:10A6600000250298FCF771FCB4F87010814202D00A
:10A67000A4F8700001250CA90398FCF7F1FA9DF8E5
:10A680003000B4F86610884211D19DF83110B4F84A
:10A69000682091420BD19DF83210B4F86A209142A3
:10A6A00005D19DF83310B4F86C20914211D0A4F874
:10A6B00066009DF83100A4F868009DF83200A4F807
:10A6C0006A009DF8330052490125A4F86C0000206F
:10A6D00008700498FCF739FCB4F86E10884205D075
:10A6E0000498FCF732FCA4F86E0001E0002D6CD059
:10A6F0000EF02EFF0120A4F8600066E00C236A46ED
:10A700002C213046FCF700FC042851D30198FCF7BB
:10A7100098FAA188884258D13EA10398F5F757FED0
:10A72000002852DD4CF6CC40ADF8300002E02BE0C2
:10A7300036E03DE03AA0FBF783F800234FF488347D
:10A74000022221461846FEF703F802230CAA2146EE
:10A750000020FEF7ABF900234FF490344FF48072E1
:10A7600021461846FDF7F4FF0298F5F729FE431C31
:10A7700021460020029AFEF799F90A2003F014FFFF
:10A780000020FDF75FFE20E00C236A462C213046B6
:10A79000FCF7BAFB03280BD30198FCF752FA14E03C
:10A7A0000C236A462C213046FCF7AEFB032802D26C
:10A7B00028460EB070BD0198FCF743FAA188884284
:10A7C00003D11DA10298F5F702FE0020F1E7000079
:10A7D000D619002025730D0A0000000024636F6E57
:10A7E0006669672C000000000E0D0020247570645F
:10A7F0006174652C00000000246765746C6F672C21
:10A800000000000024636F6E74726F6C2C000000F7
:10A81000C000002056323032313035313030300017
:10A82000676F746F204F5441204170706C69636191
:10A8300074696F6E0D0A00006265657065720000D4
:10A8400010B5134C88B0207802281ED1FCF7B6FF53
:10A850001049A37801F18002CDE90521CDE9030378
:10A860000D490E4B48881B78C2B2000ACDE9003072
:10A8700002928B880AA24FF480611248FCF72DFBEC
:10A88000024610496068FFF7A5FA08B0002010BD25
:10A89000C0000020412300200E0D002008010020F0
:10A8A000245854422C25582C2530327525252C252A
:10A8B000642E25642C25732C25642C3225732025C9
:10A8C00073000000D619002010B50023034A0221AE
:10A8D0000348FFF75FF8002010BD00006DA90208D3
:10A8E000C40000203EB5FCF737FD0025194C0128B7
:10A8F00002D0257000203EBD207890B10228F9D109
:10A90000FCF704F8A1684EF66022411A914202D287
:10A9100061780029EED06570A060FFF791FFA57007
:10A92000E8E70D4D01202070B5F86800B5F86C20FF
:10A93000B5F86A108DE8070035F8663F07A24FF4B6
:10A9400080610948FCF7C9FA2A8907496068FFF75E
:10A9500001F8CFE7C00000200E0D002025752E2540
:10A96000752E25752E257500D619002038B511488D
:10A9700000240278A9B1012917D0022913D0032994
:10A980000ED100946B4640F2FF320B494068FFF74E
:10A990008DF9002804D1084800994454FFF72CFE93
:10A9A00038BD012AFCD1047038BD012AFCD1022136
:10A9B000017038BDC0000020D619002070B51F4BB3
:10A9C0001F4A86B0198814880025B1FBF4F11D4C8C
:10A9D000C9B2E1701D8015802278022A2AD1CDE902
:10A9E00002151949049505950A78184903461F4828
:10A9F0008988CDE9001216A24FF48061FCF76DFA48
:10AA000006461B48E168324608441849F5F772FCCF
:10AA1000E0683044E060FBF779FF2169401AC828FC
:10AA200008D3FBF773FF20611149E2686068FFF704
:10AA3000D1F9E56006B0002070BD00003C010020A7
:10AA40003E010020C0000020080100200E0D002063
:10AA500025732C25582C253032782C25642C256420
:10AA60002C25642C2564250D0A000000D619002031
:10AA7000D611002010B5F8F789FC00224FF41041E0
:10AA80000748F8F7EEFD002204210648F8F7E9FD33
:10AA9000642003F089FDBDE810400020FDF7D2BC22
:10AAA00000000240000402400148FAF7F1B800003B
:10AAB000547C00200148FAF7EBB80000947C002099
:10AAC0000148FAF7E5B80000D47C00202DE9F041F8
:10AAD0004FF0FF3471B3032832D200EB4002C2EBD7
:10AAE0004012194800EB8200827812B1012A22D06C
:10AAF00026E04568D0E902326E6B1344366876680A
:10AB00009B1BD6180369F61AB6FBF2F702FB176215
:10AB1000012A04D814D12A681268920610D41A782F
:10AB20000A70D0E90412914201D1816800E0491C09
:10AB30000161002404E01830FAF7B2FD0028F8D0D3
:10AB40002046BDE8F0810000C079002009B103284B
:10AB500002D34FF0FF30704700EB4002C2EB4010D1
:10AB6000034A02EB80004068086000207047000044
:10AB7000C079002070B50C00064601D0032E02D328
:10AB80004FF0FF3070BD06EB4600C0EB4611204889
:10AB900000EB810500F8216022786A706078A87067
:10ABA0006068A860A168E960627812B1012A05D0E6
:10ABB0000BE028610844401E686106E0D4E90112F8
:10ABC00005F118000123FAF744FDE068E862206906
:10ABD0002863A069286760696863207808B1012844
:10ABE00006D104F10C0105F138000EC9FCF742FA58
:10ABF000607820B1012806D0022804D006E0304653
:10AC000000F008F802E0304600F028F8002070BD9F
:10AC1000C0790020104900EB4002C2EB401018B48C
:10AC200001EB80025068016809E04B68ADF8003024
:10AC3000BDF80030ADF800300B684B6800930B682E
:10AC40001B07F2D491681161D368CC18641E54615B
:10AC50009AB218BCFAF770BAC07900200E4900EB1E
:10AC60004002C2EB401001EB800182B048680268EC
:10AC700009E05368ADF80030BDF80030ADF80030A1
:10AC800013685368009313681B07F2D401226831DC
:10AC900002B0FAF79DBA0000C079002070B50646F0
:10ACA0000D4600EB4600C0EB46110A4800EB81045C
:10ACB0006068F9F7D6FF606845606068FAF770F879
:10ACC00010B14FF0FF3070BD304600F005F80020A5
:10ACD00070BD0000C079002070B5054600EB45004E
:10ACE000C0EB4511184800EB8104A07810B1012891
:10ACF00007D00DE0A0682061E1680844401E606153
:10AD000006E0D4E9021204F118000123FAF7A1FCCD
:10AD1000607808B1012806D104F12C0104F1380053
:10AD20000EC9FCF7A7F9A07820B1012806D00228A7
:10AD300004D006E02846FFF76DFF02E02846FFF743
:10AD40008DFF002070BD0000C079002070B50C00A0
:10AD500001D0032802D34FF0FF3070BD00EB40015B
:10AD6000C1EB4011044800EB810005467421FBF75C
:10AD700037FF00206C6070BDC0790020024610498A
:10AD8000002000BF00EB4003C3EB401301EB830343
:10AD90005B6893420FD100EB4002C2EB401201EB23
:10ADA0008201897829B1012901D0022907D1FFF751
:10ADB00055BFFFF72FBF401CC0B20328E2D3704736
:10ADC000C079002038B501461848002404EB44023D
:10ADD000C2EB441200EB820252688A4220D104EB9B
:10ADE0004401C1EB441100EB8100817801290BD0B3
:10ADF000022914D1016F11B190F8680088472046EC
:10AE0000BDE83840FFF72ABF90F868108DF80010B1
:10AE100069461830FAF700FC2046FFF71FFF38BDDF
:10AE2000641CE4B2032CD1D338BD0000C0790020EB
:10AE30002DE9F04715465FEA010A4FF000084FF090
:10AE4000FF391AD0CDB1032817D200EB4001C1EB76
:10AE50004012304901EB82077E6876B100EB400278
:10AE6000C2EB40102B4A797802EB8004383439B1B8
:10AE7000012923D0022943D04AE04846BDE8F087A3
:10AE8000FBF7FAFB29462046FCF7C8F8060033D04A
:10AE900020463146FCF78FF82A4651463068F5F7D0
:10AEA00029FA2046FCF79BF80446FBF733FEA088FE
:10AEB000216882B27868FAF70FFA29E0FBF7DCFB29
:10AEC00020462946FCF7AAF8060015D02046314650
:10AED000FCF771F82A4651463068F5F70BFA204620
:10AEE000FCF77DF80446FBF715FEA088216882B2C6
:10AEF0007868FAF731FA0BE0FBF70CFEC84607E07A
:10AF0000642005FB00F3AAB251463046FAF787F9F0
:10AF10004046B3E7C079002070B5234A002100BF46
:10AF200001EB4103C3EB411302EB83035B688342F4
:10AF300035D101EB4100C0EB411002EB8004607899
:10AF4000B8B101282FD104F138000546FCF747F8C5
:10AF500001462846FCF71BF82846FCF740F8002875
:10AF600021D081888AB201686068BDE87040FAF734
:10AF7000F3B904F138000546FCF731F801462846DC
:10AF8000FCF705F82846FCF72AF800280BD0818842
:10AF90008AB201686068BDE87040FAF79DB9491C43
:10AFA000C9B20329BCD370BDC0790020FEE7000000
:10AFB0002DE9F0413C4C0027012621783B4A3D46D3
:10AFC00008290FD0072944D006294DD005294FD094
:10AFD000042950D0032951D079B3012956D0022930
:10AFE00058D059E0A1780023A1F1050C05E000BF7D
:10AFF00012F803E05B1C7744BFB26345F8DB63796A
:10B0000094F803C0FA181144627861442779114416
:10B0100039440844C04310F0FF0F14D1012B0DD068
:10B02000022B10D1224F214907EB0C00F5F762F9F2
:10B030000EF08EFAA7F8606005E023E04FEA5C01AD
:10B040001046FDF711FE2570E570A570A571BDE8ED
:10B05000F081A1795054491CC8B2A071A178491F50
:10B060008842F4D1082001E0607007202070EEE7EC
:10B07000E0700620FAE760710520F7E7A070E57040
:10B080000420F3E7552807D12670E0E7AA2803D16A
:10B090000220EBE7032803D02570E570A570D6E702
:10B0A000032020702071D2E7B80000200E1100208C
:10B0B0000E0D0020FEE700000FB41CB50246002074
:10B0C00007AC00290BD0491ECDE90021054B6A468B
:10B0D0002146069801F0A0F9009A002111701CBCCD
:10B0E0005DF814FB47CB02080FB4084B10B504A958
:10B0F00002AA039801F090F9044602A9002001F089
:10B100002DFD204610BC5DF814FB00005DCB02084D
:10B110007CB5044600201D46164600290BD0491E6A
:10B12000CDE90041044B6A462946304601F074F9E6
:10B13000009A002111707CBD47CB020803B401982E
:10B140004100009850EAC12018BF04204A0D18BFE2
:10B1500040F0010040F2FF72B2EB515F08BF40F0D7
:10B160000200012808BF052002B070470048704760
:10B17000680A002030B528B1144C031F0020216854
:10B180000A4605E0084630BD9A4203D81046526888
:10B19000002AF9D1002800D041680BD00468A3EB45
:10B1A0000005A54204D11B681C440346046002E06C
:10B1B000436000E023603AB11C68D51AA54203D170
:10B1C00015682C441C6052685A6030BD600A00202B
:10B1D0002DE9F0412DED020B9FED3D0B2DED028B86
:10B1E0009FED3D8BDDE90254C4F30A50A0F2FF3617
:10B1F000142E37DA002E18DA53EC102B9DED020BCB
:10B2000051EC100BF5F731F953EC182BF5F748FB1F
:10B2100057D2002CBCBF4FF00044002551DB54EA4C
:10B22000050018BF2E4C1BD14BE02E4820FA06F724
:10B2300004EA070028431FD053EC102B9DED020BAE
:10B2400051EC100BF5F711F953EC182BF5F728FB1F
:10B2500037D2002C03DD4FF48010F0400444BC438F
:10B2600000252EE0332E07DCA6F114004FF0FF314D
:10B2700021FA00F73D4206D19DED020BBDEC028B99
:10B2800002B0BDE8F08153EC102B9DED020B51ECA8
:10B29000100BF5F78EF953EC182BF5F701FB10D2D4
:10B2A000002C0DDD142E08BF641C09D0C6F134003B
:10B2B000012101FA00F02844A84238BF641C054669
:10B2C000BD43CDE902549DED020BD7E7000000001D
:10B2D0009C7500883CE4377E000000000000000000
:10B2E0000000F03FFFFF0F002DED020B019820F052
:10B2F000004001909DED000B02B07047000000007F
:10B300002DE9F0412DED020B9FED3D0B2DED028B54
:10B310009FED3D8BDDE90254C4F30A50A0F2FF36E5
:10B32000142E37DA002E18DA53EC102B9DED020B99
:10B3300051EC100BF5F799F853EC182BF5F7B0FA20
:10B3400057D2002CA4BF0024254652DA24F0004036
:10B35000284318BF2E4C4CD01AE02E4820FA06F78E
:10B3600004EA070028431FD053EC102B9DED020B7D
:10B3700051EC100BF5F779F853EC182BF5F790FA20
:10B3800037D2002C03DA4FF48010F0400444BC4361
:10B3900000252EE0332E07DCA6F114004FF0FF311C
:10B3A00021FA00F73D4206D19DED020BBDEC028B68
:10B3B00002B0BDE8F08153EC102B9DED020B51EC77
:10B3C000100BF5F7F6F853EC182BF5F769FA10D2D5
:10B3D000002C0DDA142E08BF641C09D0C6F134000D
:10B3E000012101FA00F02844A84238BF641C054638
:10B3F000BD43CDE902549DED020BD7E700000000EC
:10B400009C7500883CE4377E0000000000000000CE
:10B410000000F0BFFFFF0F002DE9F04D2DED040BF4
:10B420002DED0E8B96B0DDE92550279CDDF890A020
:10B4300025F0004624F00048BAF1000F14BF0121A6
:10B44000002101EB4502FC4953184A1093422AD3CC
:10B45000002814BF0123002303EB44030B44F749E6
:10B460008B4220D358EA00019FEDF59B76D0DFF8A0
:10B47000D8B35D4503D1BAF1000F05D188E0BAF128
:10B48000000F08BF002100D0012101EB450111F59B
:10B49000001F08D8002814BF0121002101EB44013E
:10B4A00011F5001F0BD99DED261B9DED240B16B049
:10B4B000BDEC0E8B04B0BDE8F04D00F099BE002746
:10B4C000002DBCBFE149884521DAE1498845A8BF84
:10B4D00002271CDAC3451ADCDE4901EB2851142986
:10B4E00008DDC1F1340220FA02F101FA02F28242CF
:10B4F0000DD108E058B9C1F1140228FA02F101FA9D
:10B5000002F2424503D101F00101C1F1020756EAFE
:10B510000A0124D1002C22DA002D18BF022F01D0FD
:10B52000012F0AD0022000F0AFFE16B0BDEC0E8B4A
:10B5300004B0BDE8F04D00F043BE022000F0A4FED0
:10B5400000F03EFE51EC100B81F0004141EC100B7D
:10B5500016B0BDEC0E8B04B0BDE8F08D18E09FED89
:10B56000BEAB9FEDBF8B002871D1B848804522D17A
:10B5700005F1804010F5801008BFBAF1000F07D028
:10B58000B3450ADC002CA8BF9DED260BE0DA0DE0E8
:10B59000B0EE490AF0EE690ADAE7002C06DA9DED12
:10B5A000260B51EC100B81F000416FE0AE4878445F
:10B5B00090ED000BCCE7D8454DD1002C48DA2EB1E8
:10B5C00086423AD1BAF1000F42D126E0BAF1000F1B
:10B5D00013D0022000F058FE00F026FE8DED020B85
:10B5E0009DED240B8DED000B10EE900A039961F395
:10B5F0001E0003909DED020BAAE78DED02AB9DEDC1
:10B60000240B1AEE901A10EE900A8DED000B61F3E8
:10B610001E0003909DED020B9AE78DED028B9DEDD0
:10B62000240B18EE901A10EE900A8DED000B61F3CA
:10B630001E0003909DED020B8AE709DA9DED240BB5
:10B6400051EC190B53EC102BF5F728F81EE020E015
:10B650009DED240B7CE786421BDAB4F1804F0DD0C0
:10B66000A4F10050B0F1FF5013D1002D11DB9DED7E
:10B67000240B51EC100B0EF019FB07E09DED240B91
:10B6800053EC102B51EC100B00F0C2BC41EC100B32
:10B690005EE79DED240B51EC100B03F082FBBAF139
:10B6A000000FCDE90E0142D19FED710B46B3A6F11B
:10B6B000E040B0F17F600CD05E4538D1002D00DA5B
:10B6C000A7B3022F0CBF01204FF0FF30F5F755F85C
:10B6D000DCE7002D01DD002C0DDA002D01DD002C52
:10B6E0001FDB002D16DA002C14DB012F08BF9FEDA5
:10B6F000620B3FF42DAFB0EE4A0AF0EE6A0A27E77C
:10B70000022F18BF002D0CD0012F0AD1002DFFF6FB
:10B710001FAF06E0002DB8BF002C08DA012F3FF460
:10B7200017AFB0EE480AF0EE680A11E71BE00120FF
:10B7300000EBE57050EA070115D0791EB0EE498A9A
:10B74000F0EE698A084308BF9FED4D8B4E480025F7
:10B75000804570DD4D494E48884514DDB0420DDB13
:10B76000002C19DB2FE0012000F08EFD16B0BDEC9F
:10B770000E8B04B0BDE8F04D00F046BDB34502DCD1
:10B78000002C09DC1FE0864202DA002C1BDA03E001
:10B790005E452BDD002C16DD022000F075FD00F06B
:10B7A00043FD8DED020B53EC1A2B51EC180BF4F703
:10B7B00003FFCDE900010399019861F31E00039096
:10B7C0009DED020BC4E6022000F05EFD00F03CFDA2
:10B7D00010EE901A18EE900A8DED020B8DED008B95
:10B7E00061F31E0003909DED020BB1E69DED0E0B83
:10B7F00053EC192B51EC100BF4F7D8FE9FED260BF0
:10B80000CDE9080153EC102B9DED080B51EC100B0A
:10B81000F4F7D2FE9FED221B53EC112BF4F7C9FE77
:10B820009DED081B53EC112BF4F7C6FE9FED1E1B7C
:10B8300053EC112B3CE08CE0FFFF1F00FFFF0F00DB
:10B84000000000000000F03F0000F03F0000F07F2B
:10B850000000404301FCFFFF000000000000F07FFB
:10B860000000000000000000E6F8000000000000FA
:10B870000000000000000080000000000000F0FF59
:10B88000000000000000F0BF0000E0410000F043B5
:10B89000FFFFEF3F00000000000000000000D03F6D
:10B8A000555555555555D53F000000000000E03F67
:10B8B000F4F77FFE9DED080B41EC1A0B53EC102BB7
:10B8C00051EC100BF4F778FE53EC1A2BF4F774FEDE
:10B8D00041EC1A0B9FEDFE0B53EC102B9DED080B6A
:10B8E00051EC100BF4F768FE41EC1B0B9FEDFA0BCB
:10B8F00051EC1A0B53EC102BF4F75EFE41EC1A0BD3
:10B900009FEDF70B53EC102B9DED080B51EC100B3A
:10B91000F4F752FE53EC1A2BF4F748FE41EC1A0BE5
:10B9200051EC1B0B53EC1A2BF4F79FFD0690CDE95D
:10B9300006519DED060B53EC1B2B51EC100BF4F74D
:10B9400035FE53EC1A2BF4F734FE41EC100B00F0EB
:10B95000A1B90020B6F5801F0EDA9FEDE30B53EC82
:10B96000102B9DED0E0B51EC100BF4F725FECDE9DD
:10B970000E016FF034000E4600EB2650A0F2FF37A8
:10B98000C6F31300DA4940F07F6646F0405688421D
:10B99000D8BF002408DDD7498142C8BF012403DC99
:10B9A0000024A6F580167F1CD348784400EBC40021
:10B9B0000F9690ED00CB9DED0E0B53EC1C2B51EC34
:10B9C000100BF4F7F3FD9DED0E0B41EC1B0B53EC4C
:10B9D0001C2B51EC100BF4F748FD41EC100B51EC13
:10B9E000190B53EC102BF4F759FE41EC1D0B51ECE5
:10B9F0001B0B53EC1D2BF4F7DFFD41EC1A0BBF487A
:10BA00008DED10AB7844109590ED000B4FF0005089
:10BA100040EA660000EB84408DED080B00F5002045
:10BA200009909DED080B53EC1C2B51EC100BF4F717
:10BA3000BDFD9DED0E1B53EC112BF4F7BAFD41EC4F
:10BA4000100B53EC102B9DED100B51EC100BF4F779
:10BA5000B3FD9DED080B41EC1C0B53EC102B9DED41
:10BA6000100B51EC100BF4F7A7FD53EC1B2BF4F764
:10BA7000A0FD53EC1C2BF4F799FD53EC1D2BF4F7B0
:10BA80009BFD41EC1C0B53EC1A2B51EC1A0BF4F7F9
:10BA900093FD41EC1B0B9A480621B0EE4B0AF0EEE9
:10BAA0006B0A784400F0E0FAB0EE401AF0EE601A4B
:10BAB000B0EE41DAF0EE61DA53EC1B2B51EC1B0BCC
:10BAC000F4F77AFD53EC1D2BF4F776FD9DED100B8A
:10BAD00041EC1B0B53EC1A2B51EC100BF4F7C5FC8B
:10BAE00053EC1C2BF4F768FD53EC1B2BF4F7BDFC57
:10BAF0009DED100B41EC1B0B53EC102B51EC100B7C
:10BB0000F4F75AFD41EC1D0B9FED7FEB53EC1E2B20
:10BB1000F4F7ABFC53EC1B2BF4F7A7FC0890CDE932
:10BB200008519DED080B53EC1E2B51EC100BF4F754
:10BB30003DFD53EC1D2BF4F739FD53EC1B2BF4F7B3
:10BB400038FD9DED080B41EC1D0B53EC102B9DEDCA
:10BB5000100B51EC100BF4F72FFD41EC1B0B53ECC9
:10BB60001A2B51EC1D0BF4F727FD9DED080B41EC52
:10BB70001A0B53EC102B51EC1C0BF4F71DFD53EC7E
:10BB80001A2BF4F772FC41EC1A0B51EC1B0B53EC23
:10BB90001A2BF4F76AFC0C90CDE90C519DED0C0BBF
:10BBA00053EC1B2B51EC100BF4F700FD53EC1A2B4C
:10BBB000F4F7FFFC41EC1B0B9FED550B53EC102BE6
:10BBC0009DED0C0B51EC100BF4F7F6FC41EC1A0B4D
:10BBD0009FED510B51EC1B0B53EC102BF4F7ECFCCD
:10BBE00041EC1B0B9FED4E0B53EC102B9DED0C0B02
:10BBF00051EC100BF4F7E0FC53EC1B2BF4F735FC85
:10BC000041EC100B4848784400EBC40090ED001B59
:10BC100051EC100B53EC112BF4F727FC41EC1B0BF0
:10BC20003846F4F7AAFDCDE9080153EC1B2B51EC83
:10BC30001A0BF4F71AFC41EC100B3C48784400EB6B
:10BC4000C40090ED00CB51EC100B53EC1C2BF4F71F
:10BC50000CFC9DED081B53EC112BF4F706FC069031
:10BC6000CDE906519DED080B53EC102B9DED060B15
:10BC700051EC100BF4F79AFC53EC1C2BF4F796FCE8
:10BC800053EC1A2BF4F792FC53EC1B2BF4F791FCBA
:10BC900041EC100B9DED261B53EC102B8DED001B82
:10BCA00000959DED260B51EC100BF4F785FC9DEDF6
:10BCB000000B41EC1A0B53EC102B9DED260B51ECB5
:10BCC000100BF4F773FC9DED061B53EC112B2FE0CA
:10BCD000000000604715F73FFE822B654715F73FD0
:10BCE00044DF5DF80BAE543E00000000000040430E
:10BCF0008E9803007AB60B0062F4000090F4000006
:10BD00009AF300000000000000000000000008405E
:10BD1000000000E009C7EE3FFD033ADC09C7EE3F33
:10BD2000F5015B14E02F3EBE26F20000E0F10000BA
:10BD3000F4F742FC53EC1A2BF4F797FB9DED060B3E
:10BD400041EC1A0B53EC102B9DED000B51EC100B3A
:10BD5000F4F732FCCDE90C019DED0C0B51EC1A0B04
:10BD600053EC102BF4F781FBCDE902010C46AA49F4
:10BD70008C422FDB611A084318D19DED0C0B53EC5C
:10BD8000102B9DED020B51EC100BF4F70FFC41EC66
:10BD90001B0B9FEDA30B51EC1A0B53EC102BF4F77C
:10BDA00064FB53EC1B2BF4F77BFD2DD2022000F03B
:10BDB0006BFA00F039FA10EE901A18EE900A8DED39
:10BDC000020B8DED008B61F31E0003909DED020BC5
:10BDD000FFF7BEBB944A24F00041914214D393492B
:10BDE000214408437FF4EFAC9DED0C0B53EC102B7A
:10BDF0009DED020B51EC100BF4F7D8FB53EC1A2B12
:10BE0000F4F74EFD7FF6DFAC24F000408849894A04
:10BE1000002601EB205182422BDA481C4FF480119E
:10BE200021FA00F02044844AC0F30A517A44A1F276
:10BE3000FF3192ED000B814A8DED080BCA4020EADC
:10BE40000202C0F3130040F48010C1F1140120FA83
:10BE500001F60992002CB8BF76429DED080B53EC19
:10BE6000102B9DED0C0B51EC100BF4F79FFBCDE963
:10BE70000C019DED0C0B51EC1A0B53EC102BF4F74D
:10BE8000F4FA9FED6F0B0890CDE9085153EC102B9D
:10BE90009DED080B51EC100BF4F78EFB41EC1B0BE6
:10BEA0009FED690B53EC102B9DED080B51EC100B23
:10BEB000F4F782FB9DED0C0B41EC1C0B53EC102BAB
:10BEC0009DED080B51EC100BF4F770FB53EC1A2BA3
:10BED000F4F76FFB9FED5E1B53EC112BF4F76CFB3B
:10BEE00053EC1C2BF4F7C1FA41EC1A0B51EC1B0B71
:10BEF00053EC1A2BF4F7B9FACDE902019DED020BD0
:10BF000053EC1B2B51EC100BF4F750FB53EC1A2B9A
:10BF1000F4F74FFB9DED020B41EC1A0B53EC102B89
:10BF200051EC100BF4F748FBCDE908014A489DEDB0
:10BF3000080B0521784400F097F89DED081B51ECA3
:10BF4000100B53EC112BF4F737FB9DED021B53EC58
:10BF5000112BF4F72EFBCDE906019DED020B53ECFE
:10BF60001A2B51EC100BF4F727FB53EC1A2BF4F7B8
:10BF70007CFA9FED3B0B41EC1A0B53EC102B9DED23
:10BF8000060B51EC100BF4F711FB9DED060B41EC89
:10BF90001B0B53EC102B9DED020B51EC100BF4F727
:10BFA0000BFB53EC1B2BF4F779FB53EC1A2BF4F738
:10BFB000FDFA9DED021B53EC112BF4F7F7FA53EC4D
:10BFC000192BF4F7F6FACDE9020101EB0650011541
:10BFD0000029C8BF039015DC9DED020B324651ECE1
:10BFE000100BF4F732FDFFF7A9F8042808BF00F0A2
:10BFF0002BF932469DED020B51EC100BF4F725FDA9
:10C00000CDE902019DED020B51EC180B53EC102B06
:10C01000F4F7D2FAFFF73ABB0000904000000000AE
:10C02000FE822B654715973C00CC904000346F3F53
:10C0300001FCFFFF0000E03F68F00000FFFF0F0081
:10C0400000000000432EE63F396CA80C615C20BE66
:10C05000EF39FAFE422EE63F38EF00000000000004
:10C06000000000000000004070B504462DED028B7A
:10C070004D1E00EBC500B0EE408AF0EE608A90EDF8
:10C08000000B35F0060017D053EC182B51EC100BB9
:10C09000F4F792FA41EC100B6D1E04EBC50090ED25
:10C0A000001B51EC100B53EC112BF4F7DEF941ECB3
:10C0B000100B35F00600E7D1022D36D0042D1CD030
:10C0C000062D1CBFBDEC028B70BD53EC182B51EC40
:10C0D000100BF4F771FA94ED0A1B53EC112BF4F7E3
:10C0E000C4F953EC182BF4F767FA94ED081B53ECE2
:10C0F000112BF4F7BAF941EC100B53EC182B51EC5F
:10C10000100BF4F759FA94ED061B53EC112BF4F7CE
:10C11000ACF953EC182BF4F74FFA94ED040B53ECF5
:10C12000102BF4F7A2F941EC100B53EC182B51EC47
:10C13000100BF4F741FA94ED021B53EC112BF4F7BA
:10C1400094F953EC182BF4F737FA94ED001B53ECE9
:10C15000112BF4F78AF9BDEC028B41EC100B70BD8A
:10C160005060026041600860704700002DE9F047B0
:10C1700082460F4C10480D4E0E4F001B4FF000082A
:10C1800020F007054FF0010900221146504603F048
:10C190005FFC002802D1306810B10020BDE8F087B4
:10C1A0003C60C4E90058C6F80090EDE7640A00203E
:10C1B00004E80020600A002000F8002000000000D1
:10C1C0009FED070B10B553EC102B9FED070B51ECB7
:10C1D000100BF4F763FA41EC100B10BD00000000E7
:10C1E0000000000000000000000000000000F03F20
:10C1F00010B553EC112B51EC100BF4F736F941EC60
:10C20000100B10BD000000009FED050B10B553ECA6
:10C21000102B51EC100BF4F741FA41EC100B10BD50
:10C2200000000000000000009FED050B10B553EC6E
:10C23000102B51EC100BF4F7BFF941EC100B10BDB3
:10C2400000000000000000709FED050B10B553ECDE
:10C25000102B51EC100BF4F7AFF941EC100B10BDA3
:10C26000000000000000001002E008C8121F08C112
:10C27000002AFAD170477047002001E001C1121F67
:10C28000002AFBD170470000014908607047000098
:10C29000680A00202DE9FF5F82B00021DDE904304B
:10C2A000020DDDF840B0034318D044F61050A2F25E
:10C2B000FF3242431514119801281FD0A5EB0B0043
:10C2C000401C5FEA000A4FF000064E4FDFF838913D
:10C2D000B046504615D5CAF1000413E01198012468
:10C2E0004AA3012801D16FEA0B010298119AC0E913
:10C2F0000031C0E9024206B0BDE8F09FCBF100007A
:10C30000DFE704460021404A491842EB0450CDE9DA
:10C31000001012E0E00707D032463B46404649464F
:10C32000F4F74AF98046894632463B46104619469C
:10C33000F4F742F906460F466410002CEAD1DDE915
:10C340000401DDE90023BAF1000F06DAF4F734F94D
:10C3500042464B46F4F730F905E0F4F79FF94246C0
:10C360004B46F4F79BF904460E460022284BF4F79F
:10C3700097FA03D84FF0FF30014607E00022254B23
:10C3800020463146F4F771F8F4F759FA102409E021
:10C39000002C0ADB0A220023F3F718FF039B30323C
:10C3A0001A55641E50EA0102F2D1641C039AC4F1CA
:10C3B00011031444119A012A03D0012208430DD11C
:10C3C0000AE0084304D000204FF0110B119072E7EF
:10C3D000A3EB0B056D1E0DE05B4504DD4FF0000285
:10C3E00005F1010504E003DA4FF00002A5F10105B3
:10C3F000002AECD002981199C0E90231C0E9004549
:10C4000079E70000000014400000F03F3000000019
:10C410000000F0430000E03F2DE9FF4F95B09B4640
:10C420008946064600250FE2252877D100242746B5
:10C43000F84A0121059400E0044316F8013F203B2F
:10C4400001FA03F01042F7D130782A2811D06FF0AA
:10C450002F033078A0F13002092A16D8059A44F04B
:10C46000020402EB820203EB42021044761C0590A8
:10C47000EFE759F8042B0592002A03DA504244F4FE
:10C480000054059044F00204761C30782E2816D112
:10C4900016F8010F44F004042A280DD06FF02F0283
:10C4A0003078A0F13003092B09D807EB870302EBA2
:10C4B0004303C718761CF3E759F8047B761C3078E1
:10C4C0006C280FD006DC4C2817D068280DD06A28BD
:10C4D00014D104E0742810D07A280FD10DE044F470
:10C4E00000140AE044F4801401E044F4401472782B
:10C4F000824202D104F58014761C761C30786628BE
:10C500000BD013DC582877D009DC002875D04528DB
:10C51000F6D04628F4D047281AD19DE118E06328C8
:10C5200035D0642879D0652812D195E1702873D070
:10C5300008DC6728F1D069286FD06E280DD06F28ED
:10C5400006D1B5E073282CD0752875D0782874D022
:10C550005A46179990476D1C75E1C4F302500228A2
:10C5600009D003280DD0D9F8001004280DD00D6093
:10C5700009F1040967E1D9F80010EA17C1E900528E
:10C58000F6E7D9F800100D80F2E70D70F0E719F822
:10C59000041B8DF8001000208DF80100EA460120F0
:10C5A00003E059F804AB4FF0FF3061074FF0000192
:10C5B00002D40DE008F101018846B9420FDA804546
:10C5C000F8DB1AF808100029F4D108E008F101019D
:10C5D00088468142FADB1AF808100029F6D105983E
:10C5E0005B46A0EB080721463846179A00F094FAFC
:10C5F000284400EB080507E04DE029E10DE01AF8BA
:10C60000010B5A4617999047B8F10108F7D25B46DB
:10C6100021463846179A13E142E00A220092C4F3F9
:10C6200002524FF0000A022A08D059F804CB032A1C
:10C630004FEAEC710AD00DE029E02AE009F1070188
:10C6400021F00702F2E802C1914609E00FFA8CFCE2
:10C650004FEAEC71042A03D14FFA8CFC4FEAEC71DB
:10C66000002907DA0A460021DCF1000C61EB020127
:10C670002D2202E0220504D52B228DF80420012270
:10C6800003E0E20701D02022F7E7904659E00A21B3
:10C6900002E010220DE010214FF0000A00910BE0A3
:10C6A00010224FF0000A44F004040827009203E02F
:10C6B00008224FF0000A0092C4F30252022A05D069
:10C6C00059F804CB0021032A08D009E009F1070139
:10C6D00021F00702F2E802C1914605E01FFA8CFC46
:10C6E000042A01D10CF0FF0C4FF00008220728D5D6
:10C6F000702806D0009B83F0100353EA0A0305D08C
:10C700000EE040228DF80420012208E05CEA0102DC
:10C7100006D030228DF804208DF8050002229046C4
:10C72000009B83F0080353EA0A030AD15CEA010282
:10C7300001D1620705D530228DF804204FF00108A1
:10C740007F1E582804D034A003900EA802900DE05C
:10C7500036A0F9E753466046009AF3F737FD844662
:10C760000398825C0298401E029002705CEA01000D
:10C77000F0D1029806A9081A00F1200A600702D534
:10C7800024F4803400E00127574502DDA7EB0A00BE
:10C7900000E0002000EB0A01009005984144401A97
:10C7A0000590E00306D45B462146179A059800F0F1
:10C7B000B3F90544002706E001A85A46C05D179961
:10C7C00090476D1C7F1C4745F6DBE0030CD55B46AC
:10C7D0002146179A059800F09FF9054404E030209F
:10C7E0005A46179990476D1C0099481E00900029E1
:10C7F000F5DC08E0029802995A460078491C02913B
:10C80000179990476D1CBAF10001AAF1010AF1DCF9
:10C8100065E1000009280100303132333435363704
:10C82000383961626364656600000000303132337C
:10C83000343536373839414243444546000000001C
:10C8400000F058F90544761C307800287FF4ECADF0
:10C8500019B02846BDE8F08F620700D4062709F119
:10C86000070222F0070CFCE80223E14603F000482F
:10C870005FEA080C02D00FF2702C0DE05FEA045C56
:10C8800002D50FF2682C07E05FEAC47C02D00FF2F9
:10C89000602C01E0AFF2700C4FF0FF3823F0004342
:10C8A000CDF850C065280CD006DC452809D04628B4
:10C8B0001DD047283DD13DE0662818D067287ED19D
:10C8C00038E00021112F01DB112000E0781CCDE9B8
:10C8D000000106A90EA8FFF7DDFCDDE90F010E9AA5
:10C8E00003910021009207F1010A04914DE04FF0FD
:10C8F00000400097CDE9011006A90EA8FFF7CAFC79
:10C90000DDE90F0203920E9B11990022DDF80CA0C5
:10C910000093049211B9791C00EB010AB7EB0A00ED
:10C9200004D4C0F1FF3007F1010A0490AAEB07001C
:10C93000019044E0012F00DA01270021112F01DDD1
:10C94000112000E03846CDE9000106A90EA8FFF746
:10C95000A1FCDDE90F010E9A0391002104910092E0
:10C96000BA4621070CD40399514500DA8A46BAF138
:10C97000010F05DD009AAAF10101515C302908D0B0
:10C98000B84202DA10F1040F06DA0121CDE90110F4
:10C9900015E0AAF10101E9E7002805DC049901444A
:10C9A0000491AAEB000102E0411C514500DD8A46DA
:10C9B0000499401A401C01904FF00040029020075B
:10C9C00004D40198504501DBCDF8048000208DF897
:10C9D0004F0002980DF14F07B0F1004F25D02B20EA
:10C9E0000E9002984FF0020800280CDA40420290A4
:10C9F0002D200E9007E00A210298F3F769FF3031ED
:10CA0000029007F8011DB8F10001A8F10108F2DC5D
:10CA100002980028EFD1791E0E980870307800F047
:10CA2000200040F0450007F8020D12A8C01B00F1DD
:10CA300007081498007800B1012000EB0A01019862
:10CA400001EBE07105984144401A401E0590E00357
:10CA500006D45B462146179A059800F05DF8054418
:10CA60001498007818B15A46179990476D1CE00346
:10CA700024D55B462146179A059800F04DF80544E9
:10CA80001CE00498002807DBDDE90301884203DD90
:10CA90000098405C179901E0179930205A4690475A
:10CAA000049805F10105401C04900198401E019076
:10CAB00004D12E205A46179990476D1CBAF10001F7
:10CAC000AAF1010ADDDC05E017F8010B5A461799B7
:10CAD00090476D1CB8F10001A8F10108F4DC5B4639
:10CAE0002146179A0598ABE62D0000002B000000A8
:10CAF000200000002DE9F041044600251E4617469F
:10CB0000880404D405E039462020B0476D1C641E1B
:10CB1000F9D52846BDE8F0812DE9F041044600250D
:10CB20001E469046C80301D5302700E02027880420
:10CB300004D505E041463846B0476D1C641EF9D562
:10CB40002846BDE8F0814A68002A06D00A68531CCE
:10CB50000B6010704868401E486070470A68531C9C
:10CB60000B601070704770B505460C4605F10C015E
:10CB7000204605F077F970BD10B5044602492046FD
:10CB800005F070F910BD0000A00500202DE9F0416E
:10CB900005460E461746002420200BF053F90446A4
:10CBA0000CB9BDE8F0812560676026720AF088FF45
:10CBB000C4E90401034904F1180005F05AF900BF63
:10CBC000EFE70000AC0800202DE9F04780468946D9
:10CBD00015464FF0000A00260024002718200BF00D
:10CBE00031F90446002C2DD0002020726072E560DF
:10CBF00000BF04F110002061606100BF00BF12E0BF
:10CC000006EB460108EB810005F01BFA074637B139
:10CC10007D6104F11001384605F032F902E06FF44D
:10CC2000FA7A02E0761C4E45EAD300BFBAF1000F53
:10CC300003D0204601F089FC06E00549204605F0B6
:10CC40001FF901E06FF4FA7A5046BDE8F087000062
:10CC5000A4D9002070B505464FF0FF360024A5B1D9
:10CC600000BF0FE00A4800EB0410006848B1084913
:10CC700001EB041108682946F3F7A9FB08B9264619
:10CC800002E0641C0D2CEDD300BF304670BD0000E7
:10CC9000B80700202DE9F04706460D460027B946A3
:10CCA000002430200BF0CEF80446002C30D0266053
:10CCB00028682061A868A06168686061E868E06130
:10CCC000286920620020A0606869C8B1686900789E
:10CCD000B0B16869F3F774FB00F1010840460BF04E
:10CCE000B1F86062606A20B16969606AF3F78AFB33
:10CCF00008E020460AF068FD0024601EBDE8F087C9
:10CD000000206062044904F1280005F0B2F801E057
:10CD10004FF0FF373846F1E748C1002070B50024D6
:10CD2000002500260948006970B108480469256893
:10CD300006E0A4F12806306800F024F82C462568A7
:10CD4000024810308442F4D170BD000038C1002088
:10CD500070B50024002500260948006970B1084814
:10CD60000469256806E0A4F12806306800F0E6F8BA
:10CD70002C462568024810308442F4D170BD000072
:10CD800038C100203EB5044600200090019002907A
:10CD90008DF80000204600F0FCFB0190204600F0DA
:10CDA000D7FB0290204600F0E9FB05462A46012108
:10CDB00068460BF001FA3EBD2DE9F0472DED028BE0
:10CDC00082B0074600250026002402F009F88146BB
:10CDD00000F03FFF06462EB9601E02B0BDEC028B8C
:10CDE000BDE8F0874846F3F7D9FC41EC180BB0EEEC
:10CDF000480AF0EE680A00F014FF8046424617A188
:10CE0000304600F0EDFE304601F008F8044614B953
:10CE10004FF0FF351CE02046F3F7D2FA8046384643
:10CE200000F0A1FB824600204346224640210090AC
:10CE300050460BF093F9054620460AF0C5FC002D3C
:10CE400000DA05E04A4603213846FFF79FFE00BF9F
:10CE5000304600F01DFF2846BFE7000073657100F3
:10CE60002DE9F04F2DED028B83B080460E4614461F
:10CE70004FF0000A0027002501F0B2FF029000F0F9
:10CE8000E8FE07462FB9681E03B0BDEC028BBDE873
:10CE9000F08F0298F3F782FC41EC180BB0EE480AD1
:10CEA000F0EE680A00F0BDFE81464A4620A13846F1
:10CEB00000F096FE3046F3F771FC41EC180BB0EE33
:10CEC000480AF0EE680A00F0ACFE81464A4619A115
:10CED000384600F085FE44B1204600F0C3FE81468E
:10CEE0004A4615A1384600F07BFE384600F096FF12
:10CEF000054615B94FF0FF3A14E02846F3F760FAFB
:10CF00008146404600F02FFB834600204B462A46D0
:10CF10004121009058460BF021F9824628460AF03C
:10CF200053FC00BF384600F0B3FE5046ACE70000AB
:10CF30007365710061636B006D73670070B50546C2
:10CF40000024284600F018F808B1E01E70BD002348
:10CF500008A208A128460CF097FC28460AF026FAF9
:10CF60000446002C01DA2046F0E7284600F0BCFA1F
:10CF70002046EBE76F66660010B5024600210123EC
:10CF800000BF09E001EB8100064C54F820009042FC
:10CF900001D1002010BD491C9942F3DB4FF0FF3056
:10CFA000F8E70000C80800202DE9F04F2DED028BB6
:10CFB00085B082460E4617461C464FF0000BD846F9
:10CFC00000250020049001F00BFF039050460AF06A
:10CFD0008DFA0490049828B9681E05B0BDEC028B48
:10CFE000BDE8F08F00F035FE8046B8F1000F02D1A9
:10CFF0004FF0FF30F1E70398F3F7D0FB41EC180B4B
:10D00000B0EE480AF0EE680A00F00BFE81464A4690
:10D0100028A1404600F0E4FD3046F3F7BFFB41ECA9
:10D02000180BB0EE480AF0EE680A00F0FAFD8146EF
:10D030004A4621A1404600F0D3FD3846F3F79DFB58
:10D0400041EC180BB0EE480AF0EE680A00F0E9FD7A
:10D0500081464A4619A1404600F0C2FD44B120462F
:10D0600000F000FE81464A4616A1404600F0B8FD99
:10D07000404600F0D3FE054615B94FF0FF3B14E0E3
:10D080002846F3F79DF98146504600F06CFA02906D
:10D0900000204B462A467E21009002980BF05EF855
:10D0A000834628460AF090FB00BF404600F0F0FDA2
:10D0B000584692E77365710061636B00636F646546
:10D0C000000000006D7367002DE9F04107468846B7
:10D0D00015461C46069E412D29D006DC012D09D09F
:10D0E000072D19D0402D28D11BE07C2D08D07F2D95
:10D0F00023D10BE032462146384600F035F91DE0D9
:10D1000032462146384600F0D1F817E03246214633
:10D11000384600F0F8F811E03146204601F04EFFA5
:10D120000CE032462146384600F063F906E032460C
:10D130002146384600F07DF900E000BF00BFBDE8A1
:10D14000F08100002DE9F04F2DED028B83B00746F2
:10D15000884614464FF00009CA460025AB4601F048
:10D160003FFE064638460AF0C1F98346BBF1000F80
:10D1700005D1681E03B0BDEC028BBDE8F08F00F056
:10D1800068FD8246BAF1000F02D14FF0FF30F1E79F
:10D190003046F3F703FB41EC180BB0EE480AF0EE13
:10D1A000680A00F03EFD024627A10290504600F0BA
:10D1B00017FD584600F056FD024624A10290504645
:10D1C00000F00EFD84B1012F05D1224620A150466A
:10D1D00000F006FD08E0204600F044FD02461CA1D8
:10D1E0000290504600F0FCFC504600F017FE054649
:10D1F00015B94FF0FF3921E02846F3F7E1F8029026
:10D20000384600F0B0F90190002000902A467D21B8
:10D21000DDE901030AF0A2FF814628460AF0D4FAAC
:10D22000B9F1000F00DA09E0B146B8F1010F04D1FD
:10D23000324663213846FFF7A9FC00BF504600F094
:10D2400027FD484696E70000736571006361700032
:10D25000636F6E74656E7400FEB506460D4600245D
:10D2600000200090019002909DB98DF8000030469A
:10D2700000F0BBF90190304600F096F9029030467C
:10D2800000F0A8F907463A46012168460AF094FFE3
:10D290000BE0304600F03EF9044634B1206920B17D
:10D2A00000221146501E23699847FEBD2DE9FC411E
:10D2B00007460D4616460020009001900024804647
:10D2C000384600F027F904460CB1606908B9BDE89A
:10D2D000FC816A463146284600F0C6F9002800DA8B
:10D2E000F5E7019818B10198F3F76AF88046DDE98F
:10D2F0000001424663699847019810B101980AF00D
:10D3000063FA00BFE3E72DE9FF4107460D461646E5
:10D31000002000900190029003900024804638463F
:10D3200000F0F8F804460CB1A06908B9BDE8FF8127
:10D330006A463146284600F0DDF9002800DAF5E7B4
:10D34000039818B10398F3F73BF88046DDE9021221
:10D3500000984346D4F818C0E047039810B10398EA
:10D360000AF032FA00BFE1E72DE9FC4707460D4617
:10D3700016464FF00008C14600240020009001909E
:10D38000384600F0C7F804460CB1206908B9BDE87A
:10D39000FC876A463146284600F01AFA8046B8F102
:10D3A000000F05DA00221146501E2369984715E048
:10D3B000009801280DD1019818B10198F3F700F8F1
:10D3C000814601994A460020236998470120606000
:10D3D00004E000221146501E236998470121384677
:10D3E00001F090FE019810B101980AF0EDF900BF2C
:10D3F000CDE72DE9FC4106460C461546002000907D
:10D40000019000276A462946204600F02FFA00289E
:10D4100000DA05E03046DDE90012FFF721FD00BF2C
:10D42000019820B10198FDF7A5FE00200190BDE80C
:10D43000FC812DE9F04105460E461746002428469A
:10D4400000F068F804460CB10020A06003212846D3
:10D4500001F058FEBDE8F0812DE9F0470746894606
:10D4600015461E46DDF820800024384600F052F8AC
:10D47000044634B1E06920B1424631462846E369AA
:10D480009847BDE8F08700002DE9F04106460D46BB
:10D4900000270024ADB9002311A212A130460CF0E0
:10D4A000F3F90746002F18DA304600F033F8044647
:10D4B0009CB1206988B100221146501E236998470B
:10D4C0000BE0304600F026F8044634B1206920B164
:10D4D00000221146501E23699847BDE8F0810000E4
:10D4E0004F4646004F4E000070B5054600242846C2
:10D4F00000F010F804465CB1606A10B1606A0AF08E
:10D5000063F904F1280004F0CAFC20460AF05CF933
:10D5100070BD000010B502460021002300240B4816
:10D52000006980B1094801690B6808E0A1F128048D
:10D530002068904201D1204610BD19460B6803486F
:10D5400010308142F2D10020F6E7000038C10020FF
:10D5500070B50546284600F053F804460CB1A068A3
:10D5600070BD0020FCE770B50546284600F062F863
:10D5700004460CB1A06870BD0020FCE770B50546FC
:10D58000284600F03DF804460CB1606870BD0020EC
:10D59000FCE770B50546284600F04CF804460CB18F
:10D5A000606870BD0020FCE770B50546284600F0B5
:10D5B00027F804460CB1206970BD0020FCE770B567
:10D5C0000546284600F036F804460CB1206970BDC7
:10D5D0000020FCE770B50546284600F011F8044627
:10D5E0000CB1E06870BD0020FCE770B50546284628
:10D5F00000F020F804460CB1E06870BD0020FCE7A4
:10D6000030B5024600210123002000BF0CE001EBF1
:10D610008104074D55F82440944204D101EB810464
:10D6200005EB840002E0491C9942F0DB00BF30BDED
:10D63000C808002030B5024600210123002000BFA9
:10D640000CE001EB8104074D55F82440944204D1CD
:10D6500001EB810405EB840002E0491C9942F0DBF8
:10D6600000BF30BDB40800202DE9F05F80468B4636
:10D6700014464FF00009002700260025404600F020
:10D680008DFB074617B94FF0FF3927E016A1384642
:10D6900000F040FB06462EB1F068082802D1706900
:10D6A000206002E04FF0FF3918E010A1384600F08A
:10D6B00031FB05468DB1E86810280ED12869F2F7D4
:10D6C0007FFE00F1010A50460AF0BCFB6060606812
:10D6D00018B129696068F2F795FE00BF384600F07E
:10D6E000D7FA4846BDE8F09F73657100636F6E74AA
:10D6F000656E74002DE9F84F804615464FF000091D
:10D70000002700240026A34600200090404600F099
:10D7100045FB074617B9601EBDE8F88F27A13846BC
:10D7200000F0F8FA04462CB1E068082802D16069DC
:10D73000686002E04FF0FF393AE021A1384600F07E
:10D74000E9FA04462CB1E068082802D16069286033
:10D7500002E04FF0FF392BE01AA1384600F0DAFA68
:10D7600004462CB1E068082802D16069A86002E094
:10D770004FF0FF391CE015A1384600F0CBFA064601
:10D780008EB1F06810280ED13069F2F719FE00F161
:10D79000010A50460AF056FBE860E86818B13169A2
:10D7A000E868F2F72FFE0021286801F089FC00BF2D
:10D7B000384600F06DFA4846AEE700007365710028
:10D7C00061636B00636F6465000000006D73670048
:10D7D0002DE9F05F80468B46144600270026002581
:10D7E000A946404600F0DAFA074617B9681EBDE8B8
:10D7F000F09F1AA1384600F08DFA06467EB1F06817
:10D8000020280CD1304600F07CFA8146B9F1000F97
:10D8100002DD0120206004E00020206001E0002003
:10D82000206010A1384600F075FA05468DB1E86811
:10D8300010280ED12869F2F7C3FD00F1010A504605
:10D840000AF000FB6060606818B129696068F2F74F
:10D85000D9FD384600F01CFA0020C8E763617073F8
:10D8600000000000636F6E74656E74002DE9F84F60
:10D87000804614464FF00009002700260025AB46DD
:10D8800000200090404600F089FA074617B9681E4C
:10D89000BDE8F88F15A1384600F03CFA06462EB1D7
:10D8A000F068082802D17069206002E04FF0FF396B
:10D8B00016E00FA1384600F02DFA05467DB1E86864
:10D8C00010280CD12869F2F77BFD00F1010A5046BF
:10D8D000FEF74CFC606029696068F2F793FD00BFB9
:10D8E000384600F0D5F94846D2E70000736571006C
:10D8F0006D736700F8B504460D4616461F4633465D
:10D900002A46214601200097FFF7DEFBF8BD10B53F
:10D91000044621460120FFF79FFC10BDF8B50446E0
:10D920000D4616461F4633462A46214601200097DB
:10D93000FFF792FDF8BD10B5044621460120FFF720
:10D94000A3FD10BD70B50024002600250E48006917
:10D95000C0B10D480469266810E0A4F12805686884
:10D96000012809D12868012806D02868B0F5807FF1
:10D9700002D02868FFF720FA3446266802481030A3
:10D980008442EAD170BD000038C10020F8B50446D9
:10D990000E462546002000906978D5E90232686875
:10D9A0000AF0DCFBF8BD10B500F030FF002010BD20
:10D9B00010B5017042701C0A8470C37010BD000065
:10D9C00070B500240AF020F805460AF019F806465A
:10D9D000034A29460AF0AEFA0446204670BD00000C
:10D9E00055DA020870B500240AF020F80546012D2A
:10D9F00003D1FFF7E5FF044604E0022D02D100F059
:10DA000093F804461CB1214601480AF069FF70BD35
:10DA1000C0D9002010B5002405480AF0F3FA0446E6
:10DA2000002C03DA214603480AF05AFF10BD00001B
:10DA300001DB0208C0D9002070B505460448046D1A
:10DA400024B10020024908652846A04770BD0000A7
:10DA5000C0D900202DE9F04105460C4600260027DC
:10DA6000B04685BB2046F2F7ABFC064604F18000C9
:10DA7000F2F7A6FC074609F0D9FF8046002E1CDD10
:10DA8000802E1ADA002F18DD802F16DAB8F1010F78
:10DA900002D102200BF02CF820460BF00FF804F115
:10DAA00080000BF033F804F58470D4F800110AF00C
:10DAB00057FF08480AF027FF0AE06FF49A710548FB
:10DAC0000AF00EFF04E0FFE7294602480AF008FFCB
:10DAD000BDE8F081C0D9002070B504460D4644B9B8
:10DAE00005F1080029680AF03BFF04480AF00BFF23
:10DAF00003E0214601480AF0F3FE70BDC0D90020C2
:10DB000070B5044615461E463CB9284631460BF012
:10DB100017F804480AF0F7FE03E0214601480AF02E
:10DB2000DFFE70BDC0D9002070B5002409F06CFF85
:10DB3000054609F065FF0646034A29460AF02EFA13
:10DB40000446204670BD0000D9DA020810B504462C
:10DB5000094A114609480AF0EAFE1CB1084907487B
:10DB60000AF0B6FE074905480AF0B2FE03480AF07B
:10DB7000E9FE002010BD000039DA0208C0D90020FB
:10DB800015DA0208E5D9020870B504460D460026EC
:10DB90000CB9B61E0AE00648006D28B904480465B1
:10DBA0002846FFF7D3FF01E06FF00606304670BD50
:10DBB000C0D9002070B505460E46AC6806B970BDE8
:10DBC0000CB9AE6009E000E0246814B120680028B8
:10DBD000FAD1314620460CF01DF900BFEFE70000F6
:10DBE00070B506460D46144604B970BD206A18B1DA
:10DBF0000649206A09688847284600F03FF92062F4
:10DC000021463046FFF7D6FF00BFEEE7240900208B
:10DC100010B500F0B3F804460CB12020E0602046B7
:10DC200010BD10B52DED028BB0EE408AF0EE608A8B
:10DC300000F0A4F8044644B10820E06084ED068BAF
:10DC400051EC180BF2F7C3FD60612046BDEC028B6E
:10DC500010BD10B500F092F804460CB14020E06011
:10DC6000204610BD70B5054600F088F8044664B142
:10DC70001020E060284600F001F92061206920B9F9
:10DC8000204600F005F8002070BD2046FCE70000AB
:10DC900070B5044622E02568A08900F4807020B9A0
:10DCA000A06810B1A068FFF7F3FFA08900F48070AE
:10DCB00028B9206918B10B49206909688847A089EB
:10DCC00000F4007028B9206A18B10649206A096872
:10DCD000884720460349096888472C46002CDAD13A
:10DCE00070BD00002409002002460AB1936800E0DC
:10DCF0000023184601E0491E006808B10029FADC3B
:10DD0000704701468A68002001E0401C1268002A22
:10DD1000FBD1704770B505460E460DB1A86800E00E
:10DD20000020044600E024682CB13146206A00F04F
:10DD30007EF80028F7D1204670BD000030B90B49AD
:10DD40000B4A11600B490C4A11607047016809B118
:10DD5000016800E00549064A1160416809B141685F
:10DD600000E00449044A116000BFEEE76DC10208FB
:10DD70002009002075B102082409002010B52820D0
:10DD800005490968884704461CB128212046F2F756
:10DD9000D8FA204610BD00002009002010B5044626
:10DDA00000221146204600F001F810BD2DE9F04791
:10DDB00081460D46904600240DB1284600E01648E5
:10DDC0000646FFF7DBFF0746002030600FB9BDE8CD
:10DDD000F08748460BF0C8FE824632465146384628
:10DDE00008F0F6F9044624B93846FFF751FF002041
:10DDF000EDE7B8F1000F0BD020460BF0B5FE04465E
:10DE0000207828B13846FFF743FF34600020DEE772
:10DE100005B12C603846DAE71C09002010B504462D
:10DE200000231A461946204608F05CFF10BD10B5C5
:10DE300002460B462AB99A4201D0012010BD0020AB
:10DE4000FCE70BB90120F9E705E0107808B90020DC
:10DE5000F4E7521C5B1C107800F03FF80446187879
:10DE600000F03BF88442F0D0107800F036F8044619
:10DE7000187800F032F8201AE0E7000070B5044688
:10DE80002046F2F79DFA451C28460649096888474E
:10DE9000061E00D170BD2A4621463046F2F72AFA06
:10DEA0003046F7E72009002001464FF0FF300029F7
:10DEB00002DD072900DA0020704770B504460D46E0
:10DEC000002634B1207820B12046F2F779FAA84232
:10DED00001D34FF0FF36304670BD0146412901D3D2
:10DEE0005B2901D30846704701F12000FBE70000E1
:10DEF000002000BF06E00022044B03EB00139A60F1
:10DF0000DA60401C0D28F6D370470000B8070020E7
:10DF100010B500200A49086080210948001DF2F769
:10DF200010FA802106488430F2F70BFA8021054868
:10DF3000F2F707FA802103488030F2F702FA10BDA9
:10DF400038DA00203CDB00202DE9F04105460024B2
:10DF5000002600272C68266808E02746384603F08C
:10DF6000A4FF384609F030FC34462668AC42F4D1B0
:10DF7000BDE8F0810146002042F6F923CA1A994211
:10DF800018D009DCA1F51C52A2F111026AB1012AD4
:10DF90000ED0022A19D113E0012A0ED0B2F57A7FF1
:10DFA0000FD0A2F2E93282B90CE06FF001000EE06E
:10DFB00008480CE06FF49C7009E00648801C06E0FD
:10DFC00000BF00BF0348C43801E0034800BF00BFE2
:10DFD00070470000CAFEFFFF6179FEFF02466FF046
:10DFE000CD000A2A1ED2DFE802F0050714171D1D16
:10DFF0001D1D1D1A002015E0012902D16FF0CE0071
:10E0000006E0022902D16FF0CF0001E06FF0D700E7
:10E0100008E06FF0D40005E06FF0D80002E06FF088
:10E02000D90000BF00BF7047014600200B291AD25B
:10E03000DFE801F0190609070C0D0E111614150082
:10E0400000BF0B4811E06FF4FC700EE000BF00BF92
:10E050006FF49B7009E00648C23006E000BF00BFC5
:10E060000348C63001E0034800BF00BF704700000E
:10E0700006FEFFFF6179FEFF2DE9F04385B00646FD
:10E080000D46EF004FF0FF3814216846F2F759F9BA
:10E090004FF00009182414216846F2F752F90A22B9
:10E0A000214630460BF064F91FFA80F9B9F1010FEF
:10E0B00009D0B9F1040F0AD0B9F1080F0BD0B9F1AA
:10E0C000200F10D10BE047208DF802000FE0522006
:10E0D0008DF802000BE045208DF8020007E0432098
:10E0E0008DF8020003E04E208DF8020000BF00BF53
:10E0F0000A341022214630460BF03AF980B2ADF8CE
:10E10000040010341E22214630460BF031F90290F3
:10E110001E340122214630460BF02AF9C0B28DF898
:10E120000100641C0722214630460BF021F9C0B2E1
:10E130008DF80000E41D3B4622466946304600F05B
:10E1400005F88046404605B0BDE8F0832DE9FF4F55
:10E1500095B00D46164698460020149013908146BF
:10E1600000278246402103A8F2F7EBF80020029036
:10E17000834601900090012410E001223146159859
:10E180000BF0F6F8012806D103A800F8094009F1C0
:10E19000010000F0FF09761C601CC4B2402CECDDCD
:10E1A00085F80C90012414E00122314615980BF0FB
:10E1B000DFF801280AD1601E012101FA00F001995F
:10E1C000084301901398401CC0B21390761C601C49
:10E1D000C4B2202CE8DDB2B22946139B159800F09A
:10E1E0009FF8002803DA4FF0FF3000906FE013989B
:10E1F00009FB006B002700BF4DE04FF0000A002430
:10E2000036E00120A0400199084070B30122314658
:10E2100015980BF0ADF8012820D102225946159827
:10E220000BF0A6F8C0B214900BF1020BC34503DD4E
:10E230004FF0FF3000901DE0286900EBC7004068F8
:10E2400000F81A401498296901EBC701496801EBED
:10E250004A0148700AF1010000F0FF0A761C4645A9
:10E2600004D94FF0FF30009004E0FFE7601CC4B217
:10E27000202CC6DB00BF0098401C00B90EE003A8AC
:10E28000C05D296901F83700286900EBC70080F8F4
:10E2900001A0781CC7B2287BB842AEDC00BF009852
:10E2A000401CA0B1A8EB0B00072803DD4FF0FF30A6
:10E2B00000900CE01348406848B1142002901148C7
:10E2C000436829461048029A984700200090286920
:10E2D00098B12969081D00F019F8002406E0002013
:10E2E000296901EBC4014860601CC4B2287BA042CC
:10E2F000F5DC05F1100000F009F8009819B0BDE850
:10E30000F08F0000F0E7002001000C0010B504467B
:10E31000206820B12068FCF72DFF0020206010BD90
:10E320002DE9FF4F93B00C4690469A46002012907C
:10E33000002683460027402101A8F2F702F8B146E3
:10E34000207B06EBC0061EB9781E17B0BDE8F08F23
:10E35000304609F077FD2061206918B94FF0FF3091
:10E3600012904DE031462069F1F7EBFF00260025C1
:10E370001EE000270020119010E001224146139872
:10E380000AF0F6FF012801D1781CC7B208F101009C
:10E390001FFA80F81198401CC0B211901198504596
:10E3A000EBDB01A8475506EB470086B2681CC5B2F7
:10E3B000207BA842DDDC16B94FF0FF30C5E73046C0
:10E3C00009F040FD8146B9F1000F03D14FF0FF3055
:10E3D000129015E031464846F1F7B3FF00250CE0F6
:10E3E00009EB4B00216901EBC501486001A8405DC4
:10E3F00058441FFA80FB681CC5B2207BA842EFDCA2
:10E400001298A2E72DE9F84F06460F469046994626
:10E41000002000908246002583460024F568D5F848
:10E4200000B016E02C467CB1A068B8420CD1E06880
:10E43000404509D12069484506D1204603F029FD11
:10E44000204609F0C1F901E00AF1010A5D46D5F85C
:10E4500000B006F10C008542E4D1BAF1000F05D1FD
:10E46000304603F016FD304609F0AEF90098BDE8DD
:10E47000F88F2DE9F0410546002400260027EC68BE
:10E48000266809E027462FB1384603F002FD3846DA
:10E4900009F09AF93446266805F10C008442F1D15E
:10E4A000284603F0F6FC284609F08EF9BDE8F08115
:10E4B0002DE9F04105464FF0000800240026002712
:10E4C0001148D0F85C08D8B10F48D0F85C0804694E
:10E4D00026680FE027462946F868F1F778FF38B933
:10E4E000384603F0E2FC384609F06EF94FF00108B7
:10E4F000344626680448D0F85C081030A042E9D1C0
:10E500004046BDE8F081000050D100202DE9F041E7
:10E5100080460D460024002600272C68266810E05F
:10E5200027464046F968F1F752FF40B9384603F0F4
:10E53000BCFC384609F048F90120BDE8F0813446BA
:10E540002668AC42ECD10020F7E710B5044604F190
:10E550001000FFF7F9FC204609F036F910BD000065
:10E560002DE9F0410646002700240025A0460C486E
:10E57000D0F8544825680BE0A04608F11001304659
:10E58000FFF7C4FF012801D1012704E02C462568CC
:10E5900004488442F0D100BF3846BDE8F081000055
:10E5A00050D10020A4D900204FF47A714843AFF332
:10E5B0000080002140E000BF00BF00BF00BF00BFDF
:10E5C00000BF00BF00BF00BF00BF00BF00BF00BF53
:10E5D00000BF00BF00BF00BF00BF00BF00BF00BF43
:10E5E00000BF00BF00BF00BF00BF00BF00BF00BF33
:10E5F00000BF00BF00BF00BF00BF00BF00BF00BF23
:10E6000000BF00BF00BF00BF00BF00BF00BF00BF12
:10E6100000BF00BF00BF00BF00BF00BF00BF00BF02
:10E6200000BF00BF00BF00BF00BF00BF00BF00BFF2
:10E6300000BF00BF00BF491C8142BCD3704700002F
:10E6400070B50B4C0E46C928206105D0BDE870405E
:10E65000014608A0F7F7F4B801254FF48D620C4885
:10E660006560F1F747FE304600F0A0F8257070BDF8
:10E670000C0100205B44454D4F5D61757468206658
:10E6800061696C65642C20636F64653D25640A00D4
:10E69000D81D0020F8B5144613460E460A46054616
:10E6A00001460EA0F7F7CCF8012D05D02946BDE8AC
:10E6B000F84014A0F7F7C4B818A0F7F7C1F8002085
:10E6C000009069460220FCF741FAA2B24FF47A7337
:10E6D00031460098F6F7A3FDF8BD00005B44454DB8
:10E6E0004F5D206F6E20646174613A2025642C2098
:10E6F0007074723A2025702C206C656E3A20256467
:10E700000A0000005B44454D4F5D756E6B6E6F7780
:10E710006E20747970653A2025640A005B44454D8B
:10E720004F5D5158575A5F53444B5F444154415FCA
:10E73000545950455F5241575F4E4F53520A0000A3
:10E740000A4610B5014603A0F7F77AF80D490120F3
:10E75000886010BD5B44454D4F5D6F6E20737461E2
:10E760007274206361703A7374617475735F636F60
:10E7700064653D25642C206361705F69643D256498
:10E780000A0000000C010020014601A0F7F758B86C
:10E790005B44454D4F5D206F6E20737461747573DB
:10E7A00020636F64653A2025640A00007FB5054642
:10E7B000016800240CA0F7F743F810E0C4EBC40094
:10E7C00005EBC000D0E90412CDE90212417B0091B3
:10E7D000037B8268611C0C48F7F732F8641C2868D8
:10E7E000A042EBD87FBD00005B44454D4F5D746F88
:10E7F00074616C206361706162696C6974696573CE
:10E800003A2025640A00000070B003082DE9F041A9
:10E810000025002400261348006800B3114804684E
:10E82000266819E0A4F11805A5B109F049F90746D1
:10E830000846D5E904321146FA1A60EB010042F2AB
:10E84000107300219A1A814104D24FF0FF312846FB
:10E8500000F080FC3446266802488442E2D1BDE8DC
:10E86000F0810000AC0800202DE9F0411C46002694
:10E870000E27002545E02078D22804D00020A4F8F7
:10E880001A03461E41E00A22394620460AF070FD6E
:10E89000C01C85B2B4F81A13E81C814200DA34E0D7
:10E8A000E81C1A2804DA0020A4F81A03861E2CE0BB
:10E8B0002946204608F0D2FE8046E900182220466C
:10E8C0000AF056FD804504D00020A4F81A03C61EA5
:10E8D0001BE029462046FFF7CFFB002804DA002082
:10E8E000A4F81A03461E10E0B4F81A13E81C081A1C
:10E8F000A4F81A03B4F81A236019C11C2046F1F7D2
:10E90000F9FCB4F81A030028B5DC00BF3046BDE8B6
:10E91000F0812DE9F043A7B004460D461646DDE927
:10E920002F892E9F182120A8F1F70BFD8021684622
:10E93000F1F707FD684609F0A5F8CDF880D02194DD
:10E94000229520A8C660CDE9247849460AF0C0F98E
:10E9500027B0BDE8F08310B50446E06808B1E06870
:10E960008047606910B16069804702E0606809F023
:10E9700053FF10BD10B504460421362000F049F8BD
:10E9800014B140F4006201E020F400620421BDE80B
:10E990001040362000F05DB938B540208DF80000F9
:10E9A00000210E2000F035F80446002211460E200A
:10E9B00000F04FF96B46012200210D2000F058F9BC
:10E9C000084A00210F2000F044F900F01BF922460C
:10E9D00000210E2000F03DF90349002081F82C00B1
:10E9E00038BD0000F8FF27241C7B002038B54FF607
:10E9F000FF7489B280B26B46022200F01DF830B974
:10EA00009DF800009DF8011000EB012084B2204623
:10EA100038BD38B54FF0FF3489B280B26B4604225E
:10EA200000F00AF830B903216846425C491E02EB47
:10EA30000424FAD5204638BD08B551B140F0400055
:10EA40008DF80000C8B27F2907D88DF80100022098
:10EA50000BE08DF80000012007E040F080008DF809
:10EA60000100C8098DF80200032069460AF0ACFCD9
:10EA700008BD30B414460A462146034630BC112076
:10EA8000FFF7DABF0346052200211520FFF7D4BFA8
:10EA90000346052200211720FFF7CEBF38B50546F3
:10EAA00000208DF8000000F0ADF84FF4807422468D
:10EAB0000DB14FF4407200210D2000F0BDF89DB162
:10EAC0006B46012203210F20FFF7B6FF9DF80000DF
:10EAD000000709D5FFF760FF224600210D2000F056
:10EAE000ABF84FF0FF3038BD002038BD02460121A1
:10EAF0000A2000F0AEB810B5044600211A20FFF736
:10EB000088FFC4F313026FF3130002430021BDE832
:10EB100010401A2000F09DB838B505466B4601221A
:10EB200003210420FFF788FF104C75B12A4600210D
:10EB30000C2000F081F89DF8000040F010008DF8E6
:10EB40000000A06940F0805008E09DF8000020F02F
:10EB500010008DF80000A06920F08050A0616B4685
:10EB600001220321042000F083F838BD1C7B002023
:10EB7000F8B500240546224F26468DF80040800750
:10EB80000BD580208DF800006B46012200210D205E
:10EB900000F06EF8012087F82C00E8079DF80000CF
:10EBA00021D040F006008DF800006B4601220021C4
:10EBB0000D2000F05DF803210F20FFF717FF10F480
:10EBC000816F1AD040208DF800006B460122002191
:10EBD0000D2000F04DF80020FFF7CCFE87F82C60E8
:10EBE0004FF0FF3409E040F002008DF800006B4662
:10EBF000012200210D2000F03BF82046F8BD000066
:10EC00001C7B00201CB56B46012203210F20FFF75F
:10EC100013FF9DF8000000F0800100F04000B1EB10
:10EC2000400F08D001208DF80400024601AB0321FB
:10EC30000D2000F01DF81CBD08B589B28DF800202C
:10EC4000120A8DF8012080B26B46022200F010F803
:10EC500008BD38B500236C46E254120A5B1C042B35
:10EC6000FADB89B280B22346042200F001F838BDF5
:10EC700008B551B140F0C0008DF80000C8B27F293E
:10EC800009D88DF8010002200DE040F080008DF8D9
:10EC90000000012007E040F080008DF80100C80965
:10ECA0008DF80200032069460BF03EFA08BD10B54E
:10ECB00014460244B2F5806F02D94FF0FF3010BD08
:10ECC0000B46821E21460920FFF7D2FF002010BD0F
:10ECD000054A10B5126940EA81500243002108201C
:10ECE000FFF7B7FF002010BD1C7B00202DE9F0418D
:10ECF00004460E460CB1206810B90020BDE8F08132
:10ED0000A06806446068B04203DBA168206808443C
:10ED1000F4E7304607F0BCFA074638460D49096863
:10ED2000884705463DB90C49206809688847002096
:10ED300060602060E2E725B12846D4E90012F1F7CF
:10ED4000D9FA054920680968884767602560A06886
:10ED50002844D3E72009002024090020F0B5044608
:10ED60000D4616460020002100270022E1680F68AA
:10ED700011E00A466AB1D2F808C0AC4509D1D2F810
:10ED80000CC0B44505D1D2F810C09C4501D101207A
:10ED900005E039460F6804F10C0C6145E9D100BF6C
:10EDA000F0BD82B0CDE9000121F0004001909DED61
:10EDB000000B02B051EC100B704710B5002142540B
:10EDC000120A42EA03621B0A491C0429F7DB10BD40
:10EDD000016911B10121017001E00021017070474A
:10EDE00007480068401C18B900200549086004E085
:10EDF00003480068401C02490860014800687047E9
:10EE0000A80800202DE9F043A3B004460E4615469D
:10EE10000027B846802103A8F1F793FAB94608F015
:10EE200005FE804603A808F0F3FD1CB9B81E23B008
:10EE3000BDE8F083B8F1010F02D10FF23C0908E000
:10EE4000B8F1020F02D10FF2340902E06FF00100B5
:10EE5000EDE703A823460AA22946CDE900903046F3
:10EE6000FCF72AF90746002F01DBAF4202D36FF00F
:10EE70000100DCE70020DAE7616B000064736B00DF
:10EE800025732F25732F2573000000000146888805
:10EE90004FF6FF72904201D1012001E08888401CAA
:10EEA00080B288807047000070B504464FF0FF358F
:10EEB0000AA12046F1F78BFA08B900250CE009A158
:10EEC0002046F1F784FA08B9012505E007A120469C
:10EED000F1F77DFA00B90225284670BD4155544F1F
:10EEE000000000004D414E55414C00005445524D2C
:10EEF000494E414C0000000001460248806908402C
:10EF000070470000D48200200246002100BF07E0C5
:10EF100001EB810012F8200008B908467047491C2F
:10EF20001029F5DB4FF0FF30F8E710B503460C462B
:10EF3000002100BF16E001EB810013F8200080B132
:10EF400001EB810003EB800090F90100A04208D1A1
:10EF500001EB810003EB80008088904201D10846DC
:10EF600010BD491C1029E6DB4FF0FF30F8E77CB5F7
:10EF7000002425466846FFF785FD042069462D02DA
:10EF800045EA146522020C5C1443401EF7D5204666
:10EF900029467CBD7CB5002425466846FFF778FDF0
:10EFA000042069462D0245EA146522020C5C1443D4
:10EFB000401EF7D5204629467CBD00002DE9F84FBC
:10EFC00081468B460027002400250026A046A24645
:10EFD0004846FEF7E3FE07460FB9BDE8F88F2DA1BE
:10EFE0003846FEF797FE044624B1E068082801D1B0
:10EFF000D4F814A028A13846FEF78CFE0446002C55
:10F0000037D0E068102834D1206990B32069FEF72A
:10F01000C5FE05466DB3E86840282AD120A12846E0
:10F02000FEF778FE064626B3F068082821D17069FD
:10F03000A0F59C40213840B1B0F57A7F08D0A0F20D
:10F04000E93040B101280CD108E06FF4FD7809E007
:10F050006FF0C90806E06FF0C80803E06FF0D6084B
:10F0600000E000BF00BFB8F1000F02D0404608F03A
:10F0700001F92846FEF70CFE3846FEF709FE00208F
:10F0800003460246514600900120FDF78DFF00BF68
:10F09000A3E70000736571006572726F7200000073
:10F0A000636F64650000000070B504460D4604F10E
:10F0B000180002F0F4FE204608F086FB70BD000048
:10F0C0002DE9F041054688460026002400270C481B
:10F0D000006898B10A48046827680BE0A4F1180694
:10F0E0007068A84204D141463046FFF7DDFF04E0D6
:10F0F0003C46276802488442F0D100BFBDE8F08159
:10F10000AC0800202DE9F04106460F4600250024FA
:10F11000A0460F480068C0B10D480468D4F80080CC
:10F120000FE0A4F118052868B04207D1287AB84248
:10F1300004D100212846FFF7B7FF05E04446D4F884
:10F14000008003488442ECD100BFBDE8F08100009C
:10F15000AC08002070B505460E4600242868FEF76E
:10F16000D9F904461CB1206908B1206A00B92FE022
:10F17000287A012806D002280AD0032814D0632850
:10F1800023D10BE000221146501E236998471DE051
:10F1900000221146501E2369984717E069686FF0F6
:10F1A0000B00226A904711E0A068401CA060A06894
:10F1B000032809D10A48406820B1094841686FF026
:10F1C000DC0088470020A06000E000BF00BF00BF57
:10F1D00005F1180002F063FE284608F0F5FA70BD4C
:10F1E00038C1002070B502460B46002000240021E3
:10F1F000094D2869046809E0014629B1D1E906658D
:10F20000B6185D41C1E9066520460468024D103517
:10F21000A842F1D170BD000018DA00202DE9F041BC
:10F2200004460F461546002660682844A1688842B7
:10F2300006D360682844411C204600F01FF80646AB
:10F240006EB9D4E9001288182A463946F1F752F807
:10F250006068284460600020D4E900128854304679
:10F26000BDE8F08110B50446206830B1206808F090
:10F27000ABFA002020606060A06010BD2DE9F04175
:10F2800004460D464FF0FF3700267808854208D225
:10F290002946206809F000F9064616B12660A560E7
:10F2A00000273846BDE8F081F0B587B004460E4629
:10F2B000174600250020059006900C4B0FCBCDE99A
:10F2C0000323CDE9010109F09BFE0546002D09DB72
:10F2D00025610596ADF8187001AA05A9206909F005
:10F2E0004FFE0546284607B0F0BD0000D0A6030833
:10F2F00010B5502008F0A6FD044664B15021204608
:10F30000F1F71FF84FF0FF3020610020207200BF9E
:10F310002460646000BF204610BD10B5044600BFE5
:10F320000020207200BF204600F085FB04F1200081
:10F33000FFF798FF04F12C00FFF794FFA06B10B1CA
:10F34000A06B08F041FA204608F03EFA10BD00001C
:10F3500070B504460E460025E3681FA2B168306808
:10F36000FBF7AAFE0546002D02DBB068A84202D8D2
:10F370004FF0FF352EE075600025206988B1606987
:10F3800078B1012216A13046FFF748FF002806DBBE
:10F39000314604F1100000F079F8002801DA4FF04E
:10F3A000FF352DB90B220FA13046FFF737FF054679
:10F3B0004DB9A06938B1E06928B1314604F11800AF
:10F3C00000F018F805462DB9022209A13046FFF7D2
:10F3D00025FF0546284670BD47455420257300008B
:10F3E0003F00000020485454502F312E300D0A00A9
:10F3F0000D0A00002DE9F04705460C4600270026BF
:10F40000B04600BF37E0296851F83600F0F7D8FF62
:10F410008146296801EBC6014868F0F7D1FF4844EE
:10F4200000F1030860684044A168884206D3606820
:10F430004044411C2046FFF721FF0746BFB9296819
:10F4400001EBC6014B68296851F83620D4E9001C4D
:10F4500001EB0C000BA1FBF747FE0746474502D026
:10F460004FF0FF3703E06068404460600027781C7D
:10F4700000B903E0761C6868B042C4D800BF3846C3
:10F48000BDE8F08725733A25730D0A002DE9F84F82
:10F4900006460C4600270025A846A94600BF50E0B6
:10F4A000316801EBC501486800F012F98146B9F1F5
:10F4B000000F02D14FF0FF373FE04846F0F780FFE2
:10F4C0008246316851F83500F0F77AFF5044002D3C
:10F4D00001DD012100E00021084400F1010860681D
:10F4E0004044A168884206D360684044411C2046DD
:10F4F000FFF7C4FE0746DFB9CDF80090316851F838
:10F500003530D4E9001C01EB0C00002D01DD10A109
:10F5100000E010A10A4610A1FBF7E6FD07464745AB
:10F5200002D04FF0FF3703E060684044606000277E
:10F53000484608F049F94FF00009781C00B903E08B
:10F540006D1C7068A842ABD800BF3846BDE8F88F84
:10F550002600000000000000257325733D25730080
:10F5600070B58AB004460E4600250020079008902A
:10F5700009900590069003900490009001900290ED
:10F58000E36835A2B1683068FBF796FD0546002DAB
:10F5900002DBB068A84202D84FF0FF3555E0756035
:10F5A00000250B222EA13046FFF738FE05464DB947
:10F5B000A06938B1E06928B1314604F11800FFF7BD
:10F5C00019FF0546002D40D12069002837D0606919
:10F5D000002834D025A0059007A8069001200490AB
:10F5E00005A803904FF400716846FFF747FE002816
:10F5F00006DB694604F11000FFF748FF002801DA36
:10F600004FF0FF351DA20C2107A8019BFBF754FD0D
:10F61000DDB9314603A8FFF7EDFE00280CDB02221E
:10F6200017A13046FFF7FAFD002805DB3046DDE97B
:10F630000012FFF7F3FD40B14FF0FF3505E0022265
:10F640000FA13046FFF7EAFD05466846FFF70AFEC0
:10F6500028460AB070BD0000504F53542025730057
:10F6600020485454502F312E300D0A00436F6E74D1
:10F67000656E742D4C656E6774680000256400002B
:10F680000D0A000070B505460C4600264FF4806157
:10F690002046FFF7F3FD064696B9287A28B9214699
:10F6A0002846FFF755FE06460AE0287A012805D1CC
:10F6B00021462846FFF754FF064601E04FF0FF368B
:10F6C0001EB90020D4E900128854304670BD0000F5
:10F6D0002DE9F047074600240025A0463E46A246F5
:10F6E0003846F0F76DFE814607EB090A09EB490140
:10F6F000481C08F0A7FB05468046B8F1000F2ED045
:10F7000029E016F8014B202C03D12B2005F8010B22
:10F7100021E0302C03DA2D2C01D02E2C0BD1412CE2
:10F7200001DA392C07DC5A2C03DD612C01DA5F2C5D
:10F7300001D17A2C0DDD252028700A4800EB241019
:10F740000078687004F00F000649085CA870ED1C92
:10F7500001E005F8014B5645D3D300202870404600
:10F76000BDE8F0870009002010B5C163026443645E
:10F7700000BF0524047200BF10BD000030B5034671
:10F7800000210024002000220A4D29690C680BE0AA
:10F790000A463AB115699D4204D1157A052D01D06A
:10F7A000104605E021460C68024D1035A942EFD104
:10F7B00000BF30BD18DA00202DE9F05F05464FF09C
:10F7C000000A0027D5F82C80D5E90B1001EB0009C1
:10F7D00000240026B8F1000F04D028A14046F0F71D
:10F7E000C7FD00E000200646002E44D006F10C00C4
:10F7F000814540D309363046F0F72AFE824621A1E2
:10F800003046F0F7B5FD0446DCB122A12046F0F702
:10F81000AFFD48B310342046F0F71AFE07461EA18C
:10F820002046F0F7A5FD0446F4B1A9EB0400001F43
:10F83000B84220DB3B46221D51462846FFF794FF85
:10F8400019E0287A062816D113A13046F0F790FD6A
:10F85000044654B1201DF0F7B3FD83465B46221DDC
:10F8600051462846FFF780FF05E000231A4651461F
:10F870002846FFF779FF0020BDE8F09F4854545018
:10F880002F312E00436F6E74656E742D4C656E675C
:10F8900074683A000D0A00000D0A0D0A000000000D
:10F8A00070B5054600240A4808F038FB2846FFF7E3
:10F8B00065FF044634B1207A012803D100BF02203D
:10F8C000207200BF024808F02BFB002070BD000032
:10F8D00030DA00202DE9F04180460D46164600271B
:10F8E0000024184808F01AFB4046FFF747FF04467B
:10F8F0000CB3207A042802D0207A03281BD105B14A
:10F9000046B900BF0620207200BF2046FFF754FF13
:10F91000074610E03246294604F12C0000F052F868
:10F920000746002F03DA6FF00200E06003E0204694
:10F93000FFF742FF0746034808F0F2FA3846BDE8F1
:10F94000F081000030DA002070B5054600240A4836
:10F9500008F0E4FA2846FFF711FF044634B1207A94
:10F96000032803D100BF0420207200BF024808F022
:10F97000D7FA002070BD000030DA002070B50646CE
:10F980000D4600240E4808F0C9FA3046FFF7F6FE8F
:10F99000044684B1207A012808D0207A022805D0B4
:10F9A000207A032802D0207A042804D1002D02DA1C
:10F9B0006FF00100E060024808F0B2FA002070BD6C
:10F9C00030DA00202DE9F04104460F4615460026A6
:10F9D00060682844A168884206D360682844411CB6
:10F9E0002046FFF74BFC06466EB9D4E90012881892
:10F9F0002A463946F0F77EFC6068284460600020A3
:10FA0000D4E9001288543046BDE8F08170B5044650
:10FA10000025D4E90812206909F084FB05461DB9C8
:10FA200000BF0320207204E0681C10B96FF00100D1
:10FA3000E060284670BD10B504462069002805DB4B
:10FA4000206909F05FFA4FF0FF30206110BD00001F
:10FA50002DE9F0410B3020F00706104D19E0206829
:10FA6000B04215D3B0420AD9871B201DD4F80480B8
:10FA7000F0F740FCA019C0E90078286004E0606855
:10FA80002860201DF0F736FC201D2660BDE8F081BF
:10FA9000251D2C68002CE2D10020F7E7600A002029
:10FAA000F0B5D5B005460F461646802105F1D000C9
:10FAB000F0F747FC802E0DD9684600F0D7F83246A3
:10FAC0003946684600F0EAF8694605F1D00000F0D2
:10FAD00065F805E03246394605F1D000F0F70AFC3A
:10FAE000284600F0C3F83622802134A8F0F722FC23
:10FAF000002408E034A8005D05F1D001095D48400C
:10FB000034A90855641C802CF4D3802234A92846DB
:10FB100000F0C4F855B0F0BDF0B5ADB005460E46E6
:10FB20001746294601A800F039F85C2280210DA86B
:10FB3000F0F700FC002408E00DA8005D05F1D001FD
:10FB4000095D48400DA90855641C802CF4D3284653
:10FB500000F08CF880220DA9284600F09FF8302292
:10FB600001A9284600F09AF8294601A800F016F8E5
:10FB70003A4601A93046F0F7BDFB302101A8F0F765
:10FB8000E0FB2DB0F0BD70B504460D46164632467A
:10FB90002946204600F082F870BD00002DE9FC5F88
:10FBA00005460C46A846002D58D0204600F080F8A7
:10FBB000002250E004EBC20CDCE900014FF0000C25
:10FBC0000CEA0C070E460CEA0C0CCDE900C0DDE98E
:10FBD00000A346EA0A0047EA03014FF0FF2C00EABF
:10FBE0000C0301EA0C0C1B0A43EA0C634FEA1C2AC3
:10FBF0004FF0FF1E00EA0E0901EA0E0C4FEA0C2C32
:10FC00004CEA196C43EA09204AEA0C01DFF858C0B3
:10FC100000EA0C0301EA0C0C1B0C43EA0C434FEA0C
:10FC20001C4A4FF6FF7E00EA0E0B01EA0E094FEA6E
:10FC3000094C4CEA1B4C43EA0B434AEA0C0A04EB1E
:10FC4000C20CCCE9003A04EBC20103C9C8E90001C7
:10FC500008F10808521C062AACDB00BFD021204660
:10FC6000F0F76FFBBDE8FC9F0000FFFF10B50446F6
:10FC700004B910BD402208492046F0F73BFB802123
:10FC800004F15000F0F75DFB0021A164E164216400
:10FC9000616400BFEDE7000068A9030870B5044681
:10FCA0000D46164632462946204602F01FF870BD22
:10FCB0002DE9F05F0446D4E91001C00840EA41761E
:10FCC000C908802200233046F0F780FA1546D4E9AF
:10FCD00010014FF0000808EA08030A4608EA08067F
:10FCE000074642EA060043EA07014FF0FF2800EA10
:10FCF000080C01EA08084FEA1C2C4CEA086C4FEA91
:10FD0000182A4FF0FF1E00EA0E0901EA0E084FEA1A
:10FD1000082848EA19684CEA09204AEA0801DFF88D
:10FD20003C8100EA080C01EA08084FEA1C4C4CEA46
:10FD3000084C4FEA184A4FF6FF7E00EA0E0901EA26
:10FD40000E084FEA084848EA19484CEA094C4AEAC2
:10FD5000080AC4E910CAD4E912014FF0000808EA01
:10FD600008030A4608EA0806074642EA060043EA8C
:10FD700007014FF0FF2800EA080C01EA08084FEAE3
:10FD80001C2949EA08694FEA182A4FF0FF1E00EAC9
:10FD90000E0B01EA0E084FEA082C4CEA1B6C49EAEC
:10FDA0000B204AEA0C01DFF8B48000EA080C01EAF3
:10FDB00008094FEA1C4848EA09484FEA194A4FF631
:10FDC000FF7E00EA0E0B01EA0E094FEA094C4CEAED
:10FDD0001B4C48EA0B484AEA0C0AC4E9128A1DB3D4
:10FDE000802228466D1C04F150010A54702D07D85A
:10FDF000C5F1700104F150025019F0F7A2FA1BE0AE
:10FE0000802D06D2C5F1800104F150025019F0F79F
:10FE100098FA04F15001204600F022F87E2104F106
:10FE20005000F0F78EFA07E0702104F15000F0F76F
:10FE300088FA802084F8500004F15002D4E91201BD
:10FE4000C2E91C0104F15000D4E91021C0E91E21CF
:10FE50000146204600F004F8BDE8F09F0000FFFFD7
:10FE60002DE9F04F99B00646894606F15005D6E9CE
:10FE70000012CDE91612D6E90212CDE91412D6E924
:10FE80000412CDE91212D6E90612CDE91012D6E914
:10FE90000812CDE90E12D6E90A12CDE90C12D6E904
:10FEA0000C12CDE90A12D6E90E12CDE9081200248F
:10FEB00000BFD9E9000109F108094FF0000C0CEA74
:10FEC0000C030A460CEA0C0CCDE900C0DDE900A8E1
:10FED00042EA0A0043EA08014FF0FF2C00EA0C074F
:10FEE00001EA0C0C3F0A47EA0C674FEA1C2A4FF064
:10FEF000FF1E00EA0E0801EA0E0C4FEA0C2C4CEA39
:10FF0000186C47EA08204AEA0C01DFF8A0C400EAAE
:10FF10000C0701EA0C084FEA174C4CEA084C4FEA70
:10FF2000184A4FF6FF7E00EA0E0B01EA0E084FEA70
:10FF3000084747EA1B474CEA0B4C4AEA070A05EB1D
:10FF4000C407C7F800C0C7F804A00E200021DDE9EF
:10FF50000E23F8F7A7FB0746884612200021DDE9AB
:10FF60000E23F8F79FFB424687EA000882EA010762
:10FF700029200021DDE90E23F8F794FB88EA000828
:10FF800087EA0100DDE9081218EB010C5041DDE9B8
:10FF90000E72DDE90C311F400A40DDE90AABDDE9F4
:10FFA0000E312AEA03032BEA01015F4051401CEBAA
:10FFB00007024841FE4B03EBC401D1E90031D218DE
:10FFC000484105EBC40319685B6852185841CDE9F4
:10FFD0000220DDE90237DDE91010C91840EB070205
:10FFE000CDE910121C200021DDE91623F8F75AFB99
:10FFF0000746884622200021DDE91623F8F752FB48
:020000040803EF
:10000000424687EA000882EA010727200021DDE94D
:100010001623F8F747FB88EA000887EA0103DDE9C1
:10002000021018EB010C4341DDE91671DDE91420E3
:1000300017400140DDE912ABDDE9162002EA0A02B1
:1000400000EA0B0057404840DDE9142102EA0A02A9
:1000500001EA0B01574048401CEB07014341CDE941
:100060000813641CD9E9000109F108094FF0000CDC
:100070000CEA0C030A460CEA0C0CCDE900C0DDE9E1
:1000800000CA42EA0C0043EA0A014FF0FF2C00EAE2
:100090000C0701EA0C0C3F0A47EA0C674FEA1C2ADE
:1000A0004FF0FF1E00EA0E0801EA0E0C4FEA0C2C7E
:1000B0004CEA186C47EA08204AEA0C01DFF8ECC267
:1000C00000EA0C0701EA0C0C3F0C47EA0C474FEA28
:1000D0001C4A4FF6FF7E00EA0E0B01EA0E084FEABB
:1000E000084C4CEA1B4C47EA0B474AEA0C0A05EB62
:1000F000C40CCCF80070CCF804A00E200021DDE97F
:100100001023F8F7CFFA0746884612200021DDE9D0
:100110001023F8F7C7FA424687EA000882EA010787
:1001200029200021DDE91023F8F7BCFA88EA00084D
:100130007940DDE90A2018EB020C4141DDE910733A
:10014000DDE90E2017400340DDE90CABDDE91020AE
:100150002AEA02022BEA0000574043401CEB070248
:100160005941934B03EBC400D0E900730846D11901
:10017000584105EBC40213685268C9184241CDE9E1
:100180000212DDE90237DDE91210C91840EB07025F
:10019000CDE912121C200021DDE90823F8F782FACC
:1001A0000746884622200021DDE90823F8F77AFA7D
:1001B000424687EA000882EA010727200021DDE99C
:1001C0000823F8F76FFA88EA000887EA0100DDE9FA
:1001D000022118EB02084141DDE9167CDDE9083017
:1001E0003B4000EA0C00DDE914ABDDE9082702EA38
:1001F0000A0207EA0B079C4603468CEA02007B4092
:10020000DDE9162702EA0A0207EA0B0750407B40A5
:1002100018EB00005941CDE90A01641CD9E900013D
:1002200009F108094FF0000C0CEA0C030A460CEA2D
:100230000C0CCDE900C0DDE900AC42EA0A0043EA5B
:100240000C014FF0FF2C00EA0C0701EA0C0C3F0AEE
:1002500047EA0C674FEA1C2A4FF0FF1E00EA0E081F
:1002600001EA0E0C4FEA0C2C4CEA186C47EA082005
:100270004AEA0C01DFF834C100EA0C0701EA0C0875
:100280004FEA174C4CEA084C4FEA184A4FF6FF7EEB
:1002900000EA0E0B01EA0E084FEA084747EA1B473F
:1002A0004CEA0B4C4AEA070A05EBC407C7F800C042
:1002B000C7F804A00E200021DDE91223F8F7F2F9B7
:1002C0000746884612200021DDE91223F8F7EAF9F3
:1002D000424687EA000882EA010729200021DDE979
:1002E0001223F8F7DFF988EA000887EA0100DDE960
:1002F0000C1218EB010C5041DDE91078DDE9121207
:10030000394002EA0802DDE90EABDDE912732AEAA0
:1003100007072BEA030379405A401CEB01015041C7
:10032000234A02EBC4030CCB8918584105EBC402E5
:1003300013685268C9185041CDE90210DDE902374F
:10034000DDE91410C91840EB0702CDE914121C2096
:100350000021DDE90A23F8F7A5F90746884622209F
:100360000021DDE90A23F8F79DF9424687EA0008F3
:1003700082EA010727200021DDE90A23F8F792F934
:1003800088EA000887EA0100DDE9021218EB010C97
:100390005041DDE90878DDE90A213A4001EA080127
:1003A000DDE916ABDDE90A7304E000000000FFFFA1
:1003B000E8A6030807EA0A0703EA0B037A4081EA82
:1003C0000307089B03EA0A0308EA0B015A404F405F
:1003D0001CEB02017841CDE90C10641CD9E9000145
:1003E00009F108094FF0000C0CEA0C030A460CEA6C
:1003F0000C0CCDE900C0DDE900C742EA0C0043EA7D
:1004000007014FF0FF2C00EA0C0701EA0C0C3F0A31
:1004100047EA0C674FEA1C2A4FF0FF1E00EA0E0B5A
:1004200001EA0E084FEA082C4CEA1B6C47EA0B2045
:100430004AEA0C01DFF8A4C400EA0C0701EA0C0840
:100440004FEA174C4CEA084C4FEA184A4FF6FF7E29
:1004500000EA0E0B01EA0E084FEA084747EA1B477D
:100460004CEA0B4C4AEA070A05EBC407C7F800C080
:10047000C7F804A00E200021DDE91423F8F712F9D3
:100480000746884612200021DDE91423F8F70AF90F
:10049000424687EA000882EA010729200021DDE9B7
:1004A0001423F8F7FFF888EA00087940DDE90E2008
:1004B00018EB020C4141DDE91278DDE914203A40E5
:1004C00000EA0800DDE914736FEA070ADF43DDE99B
:1004D000108B0AEA080307EA0B075A4080EA070371
:1004E0001CEB02005941FE4A02EBC402D2E9007241
:1004F00003460846D919504105EBC4031A685B68E6
:1005000089185841CDE90210DDE90237DDE91610FE
:10051000C91840EB0702CDE916121C200021DDE9C5
:100520000C23F8F7BFF80746884622200021DDE9B2
:100530000C23F8F7B7F8424687EA000882EA010779
:1005400027200021DDE90C23F8F7ACF888EA000841
:100550004F40DDE9021018EB010C4741DDE90C3199
:10056000DDE90A2013400140DDE908ABDDE90C02BA
:1005700000EA0A0002EA0B0243404A40DDE90A01B0
:1005800000EA0A0001EA0B0143404A401CEB030168
:100590005741CDE90E17641CD9E9000109F108099A
:1005A0004FF0000C0CEA0C030A460CEA0C0CCDE9E7
:1005B00000C0DDE9007A42EA070043EA0A014FF091
:1005C000FF2C00EA0C0701EA0C084FEA172C4CEA52
:1005D000086C4FEA182A4FF0FF1E00EA0E0B01EAE2
:1005E0000E084FEA082747EA1B674CEA0B204AEA45
:1005F0000701DFF8E8C200EA0C0701EA0C084FEA3D
:10060000174C4CEA084C4FEA184A4FF6FF7E00EAB6
:100610000E0B01EA0E084FEA084747EA1B474CEA6F
:100620000B4C4AEA070A05EBC407C7F800C0C7F835
:1006300004A00E200021DDE91623F8F733F8074661
:10064000884612200021DDE91623F8F72BF84246F0
:1006500087EA000882EA010729200021DDE9162344
:10066000F8F720F888EA00084F40DDE9101018EB91
:10067000010C4741DDE91430DDE916211A40014043
:10068000DDE916306FEA030AC343DDE9128B0AEA9B
:10069000080003EA0B03424081EA03001CEB02015D
:1006A00047418F4A02EBC4000CC8891847EB03008E
:1006B00005EBC4031A685B68891840EB0302CDE9B7
:1006C0000212DDE90237DDE90810C91840EB070224
:1006D000CDE908121C200021DDE90E23F7F7E2FF27
:1006E0000746884622200021DDE90E23F7F7DAFFCE
:1006F000424687EA000882EA010727200021DDE957
:100700000E23F7F7CFFF88EA00087940DDE90220E1
:1007100018EB020C41410DA889C80C9A1340074000
:10072000DDE90AABDDE90E0200EA0A0002EA0B028B
:1007300058407A40DDE90C3703EA0A0307EA0B0761
:1007400058407A401CEB00005141CDE91001641C77
:10075000D9E9000109F108094FF0000C0CEA0C037B
:100760000A460CEA0C08CDE90080DDE9007A42EA8D
:10077000070043EA0A014FF0FF2C00EA0C0701EAE8
:100780000C084FEA172C4CEA086C4FEA182A4FF075
:10079000FF1E00EA0E0B01EA0E084FEA082747EA9F
:1007A0001B674CEA0B204AEA0701DFF830C100EA78
:1007B0000C0701EA0C084FEA174C4CEA084C4FEAC8
:1007C000184A4FF6FF7E00EA0E0B01EA0E084FEAC8
:1007D000084747EA1B474CEA0B4C4AEA070705EB78
:1007E000C408C8F800C0C8F804700E200021DDE974
:1007F0000823F7F757FF0746884612200021DDE956
:100800000823F7F74FFF424687EA000882EA01070C
:1008100029200021DDE90823F7F744FF88EA0008D2
:1008200087EA0100DDE9121218EB010C5041DDE905
:100830001673DDE908213A401940DDE914ABDDE922
:1008400008732AEA07072BEA03037A404B401CEBA4
:1008500002015841224A02EBC402D2E90032C9180F
:10086000504105EBC40213685268C9185041CDE9E4
:100870000210DDE90237DDE90A10C91840EB070272
:10088000CDE90A121C200021DDE91023F7F70AFF49
:100890000746884622200021DDE91023F7F702FFF2
:1008A000424687EA000882EA010727200021DDE9A5
:1008B0001023F7F7F7FE88EA000887EA0102DDE96E
:1008C000021018EB010C42410FA889C80E990B4089
:1008D0000740DDE90CABDDE9101003E00000FFFF8D
:1008E000E8A6030801EA0A0100EA0B0883EA01000E
:1008F00087EA0807DDE90E1301EA0A0103EA0B03A0
:1009000048405F401CEB00007A41CDE91202641CB4
:10091000D9E9000109F108094FF0000C0CEA0C03B9
:100920000A460CEA0C0CCDE900C0DDE9008742EA7A
:10093000080043EA07014FF0FF2C00EA0C0701EA28
:100940000C084FEA172C4CEA086C4FEA182A4FF0B3
:10095000FF1E00EA0E0B01EA0E084FEA082747EADD
:100960001B674CEA0B204AEA0701DFF8A4C400EA3F
:100970000C0701EA0C0C3F0C47EA0C474FEA1C4AF3
:100980004FF6FF7E00EA0E0B01EA0E084FEA084C14
:100990004CEA1B4C47EA0B474AEA0C0A05EBC40C2D
:1009A000CCF80070CCF804A00E200021DDE90A2369
:1009B000F7F778FE0746884612200021DDE90A2372
:1009C000F7F770FE424687EA000882EA010729200D
:1009D0000021DDE90A23F7F765FE88EA00084F40A9
:1009E000DDE9141018EB010C4741DDE90A32DDE9BD
:1009F00008100B400240DDE90A106FEA010AC1430A
:100A0000DDE9168B0AEA080001EA0B0143404A407F
:100A10001CEB030147EB0200FE4A02EBC402D2E9E1
:100A20000032C918504105EBC40213685268C91856
:100A30004241CDE90212DDE90237DDE90C10C918A7
:100A400040EB0702CDE90C121C200021DDE9122346
:100A5000F7F728FE0746884622200021DDE9122309
:100A6000F7F720FE424687EA000882EA01072720BE
:100A70000021DDE91223F7F715FE88EA00084F4050
:100A8000DDE9021018EB010C474111A80DC81099BF
:100A90000A400340DDE90EABDDE9121001EA0A016C
:100AA00000EA0B0882EA010083EA0803DDE910216D
:100AB00002EA0A0201EA0B0150404B401CEB000025
:100AC0005F41CDE91407641CD9E9000109F1080967
:100AD0004FF0000C0CEA0C030A460CEA0C0CCDE9B2
:100AE00000C0DDE900A742EA0A0043EA07014FF02F
:100AF000FF2C00EA0C0701EA0C0C4FEA172848EA21
:100B00000C684FEA1C2A4FF0FF1E00EA0E0B01EAA8
:100B10000E0C4FEA0C2747EA1B6748EA0B204AEA0B
:100B20000701DFF8ECC200EA0C0701EA0C0C3F0CED
:100B300047EA0C474FEA1C4A4FF6FF7E00EA0E0BCD
:100B400001EA0E084FEA084C4CEA1B4C47EA0B47F7
:100B50004AEA0C0A05EBC40CCCF80070CCF804A0EF
:100B60000E200021DDE90C23F7F79CFD074688469F
:100B700012200021DDE90C23F7F794FD424687EAB5
:100B8000000882EA010729200021DDE90C23F7F79C
:100B900089FD88EA00084F40DDE9161018EB010CCA
:100BA0004741DDE90A20DDE90C1311400340DDE98E
:100BB0000C206FEA020AC243DDE9088B0AEA08004A
:100BC00002EA0B02414053401CEB01015F41914A94
:100BD00002EBC4000CC8891847EB030005EBC40204
:100BE00013685268C9184241CDE90212DDE90237A3
:100BF000DDE90E10C91840EB0702CDE90E121C20EA
:100C00000021DDE91423F7F74DFD07468846222031
:100C10000021DDE91423F7F745FD424687EA000885
:100C200082EA010727200021DDE91423F7F73AFDC6
:100C300088EA00087940DDE9022018EB020C414106
:100C4000DDE91387129B1F40159800EA0800DDE9D3
:100C500010ABDDE9142302EA0A0203EA0B0887EA73
:100C6000020380EA0800DDE9127207EA0A0702EAD5
:100C70000B027B4050401CEB03024141CDE91621A1
:100C8000641C102CFFF615A900BF601C00F00F00BB
:100C900005EBC00001684268CDE906120120002181
:100CA000DDE90623F7F7FEFC074688460820002109
:100CB000DDE90623F7F7F6FC474088EA0100DDE9A5
:100CC0000623D10941EA43614F4080EAD310CDE9C0
:100CD0000670A01E00F00F0005EBC000016842681E
:100CE000CDE9041213200021DDE90423F7F7DAFC33
:100CF000074688463D200021DDE90423F7F7D2FCB2
:100D0000474088EA0108DDE90401800940EA816082
:100D1000474088EA9118CDE904780E200021DDE9EA
:100D20000E23F7F7BFFC0746884612200021DDE9B5
:100D30000E23F7F7B7FC424687EA000882EA01076C
:100D400029200021DDE90E23F7F7ACFC88EA000832
:100D50007940DDE9082018EB020841410DA889C857
:100D60000C9A13400740DDE90E206FEA020AC243E5
:100D7000DDE90ACB0AEA0C0002EA0B029C468CEA87
:100D8000000C87EA020318EB0C0741EB0302214B2E
:100D900003EBC400D0E90030FB18424104F00F001F
:100DA00005EBC0000768D0F804C0E01F00F00F009A
:100DB00005EBC00001684068DDE9048B11EB080811
:100DC00040EB0B00DDE906A118EB0A084141604643
:100DD0008C4617EB080140EB0C0004F00F0705EB05
:100DE000C7073960786059184241CDE90212DDE940
:100DF0000237DDE91010C91840EB0702CDE91012E7
:100E00001C200021DDE91623F7F74CFC074603E020
:100E10000000FFFFE8A60308884622200021DDE944
:100E20001623F7F73FFC424687EA000882EA0107EB
:100E300027200021DDE91623F7F734FC88EA0008B3
:100E40007940DDE9022018EB020C414115A889C860
:100E5000149A13400740DDE912ABDDE9160200EAFF
:100E60000A0002EA0B0243405740DDE9140200EA9F
:100E70000A0002EA0B02434057401CEB030279418F
:100E8000CDE90821641C601C00F00F0105EBC100D6
:100E900001684268CDE9061201200021DDE9062340
:100EA000F7F700FC0746884608200021DDE9062305
:100EB000F7F7F8FB474088EA0101DDE90632D80977
:100EC00040EA4260474081EAD211CDE90671A01E96
:100ED00000F00F0105EBC10001684268CDE9041282
:100EE00013200021DDE90423F7F7DCFB07468846E1
:100EF0003D200021DDE90423F7F7D4FB784088EAA0
:100F00000108DDE90432990941EA8261484088EA32
:100F10009218CDE904080E200021DDE91023F7F72F
:100F2000C1FB0746884612200021DDE91023F7F7B0
:100F3000B9FB424687EA000882EA0107292000211E
:100F4000DDE91023F7F7AEFB88EA000887EA010223
:100F5000DDE90A1018EB010842410FA889C80E9973
:100F600003EA010C07EA0003DDE90CABDDE9101030
:100F70002AEA01012BEA00008CEA010C584018EB28
:100F80000C0342EB0001FE4A02EBC40205CA1B1827
:100F9000514104F00F0005EBC0000768D0F804C011
:100FA000E01F00F00F0005EBC000D0F800A0426881
:100FB000DDE904801AEB08084241DDE906A018EBE0
:100FC0000A0842416046944617EB080240EB0C00C9
:100FD00004F00F0705EBC7073A6078609A184141A3
:100FE000CDE90221DDE90237DDE91210C91840EB35
:100FF0000702CDE912121C200021DDE90823F7F7D2
:1010000051FB0746884622200021DDE90823F7F737
:1010100049FB424687EA000882EA010727200021AF
:10102000DDE90823F7F73EFB88EA00087940DDE9AF
:10103000022018EB020C4141DDE90870DDE91638A9
:101040001F4000EA0800DDE914ABDDE9083203EADD
:101050000A0302EA0B025F405040169B03EA0A03B0
:1010600008EA0B025F4050401CEB07024141CDE90A
:101070000A21641C601C00F00F0005EBC001086829
:101080004968CDE9060101200021DDE90623F7F7D3
:1010900009FB0746884608200021DDE90623F7F70B
:1010A00001FB474088EA0108DDE90621D00940EA52
:1010B0004160474088EAD118CDE90678A01E00F0CB
:1010C0000F0105EBC10001684268CDE9041213204D
:1010D0000021DDE90423F7F7E5FA074688463D20BD
:1010E0000021DDE90423F7F7DDFA474088EA010132
:1010F000DDE90432980940EA8260474081EA9211B2
:10110000CDE904710E200021DDE91223F7F7CAFAB8
:101110000746884612200021DDE91223F7F7C2FABC
:10112000424687EA000882EA010729200021DDE91A
:101130001223F7F7B7FA88EA000887EA0103DDE926
:101140000C1018EB010C4341DDE91272DDE91010BF
:101150000F400240DDE90EABDDE912102AEA010181
:101160002BEA00004F4042401CEB070743EB020113
:10117000834A02EBC40205CA3F18514104F00F0034
:1011800005EBC0000368D0F804C0E01F00F00F00BA
:1011900005EBC002D2F800B05068DDE904A21BEBF9
:1011A0000A085041DDE906AB18EB0A0240EB0B00E0
:1011B000984618EB02024CEB000004F00F0305EB1D
:1011C000C3031A605860BA184141CDE90221DDE934
:1011D0000237DDE91410C91840EB0702CDE91412FB
:1011E0001C200021DDE90A23F7F75CFA0746884650
:1011F00022200021DDE90A23F7F754FA424687EA64
:10120000000882EA010727200021DDE90A23F7F719
:1012100049FA88EA000887EA0100DDE9021218EBC2
:10122000010C5041DDE90871DDE90A323B400A401A
:10123000DDE916ABDDE90A7107EA0A0701EA0B01ED
:101240007B404A40DDE9081701EA0A0107EA0B077B
:101250004B407A401CEB03015041CDE90C10641C5B
:10126000601C00F00F0105EBC10001684268CDE988
:10127000061201200021DDE90623F7F713FA0746DD
:10128000884608200021DDE90623F7F70BFA4740DE
:1012900088EA0108DDE90621D00940EA41604740BB
:1012A00088EAD118CDE90678A01E00F00F0105EB01
:1012B000C10001684268CDE9041213200021DDE974
:1012C0000423F7F7EFF9074688463D200021DDE9C2
:1012D0000423F7F7E7F9474088EA0108DDE904212C
:1012E000900940EA8160474088EA9118CDE9047886
:1012F0000E200021DDE91423F7F7D4F907468846CC
:1013000012200021DDE91423F7F7CCF9424687EAE1
:10131000000882EA010729200021DDE91423F7F7FC
:10132000C1F988EA00087940DDE90E2018EB020CCB
:101330004141DDE91278DDE91403384003EA08038E
:10134000DDE914726FEA070AD743DDE9108B0AEA78
:10135000080207EA0B0750407B401CEB0000594194
:10136000074B03EBC4030CCB8718594104F00F0063
:1013700005EBC0000368D0F804C0E01F02E00000E5
:10138000E8A6030800F00F0005EBC0000268406803
:10139000DDE904AB12EB0A0840EB0B00DDE906AB1C
:1013A00018EB0A0840EB0B0013EB08034CEB0000B2
:1013B00004F00F0205EBC20213605060FA184141BD
:1013C000CDE90221DDE90237DDE91610C91840EB4D
:1013D0000702CDE916121C200021DDE90C23F7F7E6
:1013E00061F90746884622200021DDE90C23F7F742
:1013F00059F9424687EA000882EA010727200021BE
:10140000DDE90C23F7F74EF988EA000887EA0100C6
:10141000DDE9021218EB010C5041DDE90A78DDE943
:101420000C13394003EA0803DDE908ABDDE90C27BA
:1014300002EA0A0207EA0B0751407B400A9F07EACB
:101440000A0708EA0B02794053401CEB010158419E
:10145000CDE90E10641C601C00F00F0005EBC0000D
:1014600001684268CDE9061201200021DDE906236A
:10147000F7F718F90746884608200021DDE906231A
:10148000F7F710F9474088EA0108DDE90621D0099D
:1014900040EA4160474088EAD118CDE90678A01EAD
:1014A00000F00F0105EBC10001684268CDE90412AC
:1014B00013200021DDE90423F7F7F4F807468846F6
:1014C0003D200021DDE90423F7F7ECF8474088EAE6
:1014D0000100DDE90432990941EA82614F4080EA66
:1014E0009210CDE904700E200021DDE91623F7F7F4
:1014F000D9F80746884612200021DDE91623F7F7C0
:10150000D1F8424687EA000882EA01072920002133
:10151000DDE91623F7F7C6F888EA00087940DDE927
:10152000102018EB020C4141DDE91430DDE91627EB
:101530001A400740DDE916306FEA030AC343DDE9CC
:10154000128B0AEA080003EA0B0342405F401CEBDF
:1015500002027941FE4B03EBC40309CB1718594132
:1015600004F00F0005EBC0000368D0F804C0E01FD2
:1015700000F00F0005EBC000D0F800A04068DDE9E6
:10158000048B1AEB080840EB0B00DDE906A218EB10
:101590000A08504113EB08034CEB000004F00F0C59
:1015A00005EBCC0213605060FA184141CDE90221ED
:1015B000DDE90870DDE90232F9185041CDE9081083
:1015C0001C200021DDE90E23F7F76CF8074688465A
:1015D00022200021DDE90E23F7F764F8424687EA6E
:1015E000000882EA010727200021DDE90E23F7F732
:1015F00059F888EA00087940DDE9022018EB020C6E
:1016000041410DA889C80C9A13400740DDE90AAB97
:10161000DDE90E0200EA0A0002EA0B0258407A40B5
:10162000DDE90C3703EA0A0307EA0B0758407A4062
:101630001CEB00005141CDE91001641C601C00F05E
:101640000F0005EBC00108684968CDE906010120DB
:101650000021DDE90623F7F725F80746884608202C
:101660000021DDE90623F7F71DF8474088EA010865
:10167000DDE90601C00940EA4160474088EAD11827
:10168000CDE90678A01E00F00F0105EBC10001684E
:101690004268CDE9041213200021DDE90423F7F7A5
:1016A00001F8074688463D200021DDE90423F6F7CE
:1016B000F9FF784088EA0108DDE90412890941EA66
:1016C0008261484088EA9218CDE904080E20002182
:1016D000DDE90823F6F7E6FF0746884612200021D9
:1016E000DDE90823F6F7DEFF424687EA000882EAD2
:1016F000010729200021DDE90823F6F7D3FF88EA56
:10170000000887EA0102DDE9121018EB010C4241E2
:10171000DDE91678DDE90810394000EA0800DDE966
:1017200008736FEA070ADF43DDE9148B0AEA08034E
:1017300007EA0B07594080EA07031CEB010042EB64
:101740000301834A02EBC4030CCB8718594104F010
:101750000F0005EBC0000368D0F804C0E01F00F0E4
:101760000F0005EBC000D0F800A04068DDE9048B55
:101770001AEB080840EB0B00DDE906A218EB0A089B
:10178000504113EB08034CEB000004F00F0C05EB89
:10179000CC0213605060FA184141CDE90221DDE925
:1017A0000237DDE90A10C91840EB0702CDE90A1239
:1017B0001C200021DDE91023F6F774FF0746884658
:1017C00022200021DDE91023F6F76CFF424687EA6C
:1017D000000882EA010727200021DDE91023F6F73F
:1017E00061FF88EA000887EA0102DDE9021018EBD0
:1017F00001084241DDE910C3DDE90E100CEA010CDD
:1018000003EA0007DDE90CABDDE9100100EA0A009C
:1018100001EA0B018CEA000387EA0100DDE90E17FB
:1018200001EA0A0107EA0B074B40784018EB030175
:101830004241CDE91212641C601C00F00F0005EB60
:10184000C00001684268CDE9061201200021DDE9EF
:101850000623F6F727FF0746884608200021DDE922
:101860000623F6F71FFF784088EA0108DDE9061233
:10187000C90941EA4261484088EAD218CDE9060820
:10188000A01E00F00F0005EBC00108684A68CDE912
:10189000040213200021DDE90423F6F703FF0746C5
:1018A00088463D200021DDE90423F6F7FBFE474092
:1018B00088EA0100DDE90412890941EA82614F40AA
:1018C00080EA9210CDE904700E200021DDE90A23A0
:1018D000F6F7E8FE0746884612200021DDE90A23D4
:1018E000F6F7E0FE424687EA000882EA010729206F
:1018F0000021DDE90A23F6F7D5FE88EA000887EA29
:101900000102DDE9141018EB010C4241DDE9098701
:10191000089B1F400B9800EA0800DDE90A316FEAD6
:10192000030BCB43DDE9168A0BEA080103EA0A033D
:101930004F4080EA03011CEB07005141044A02EBCF
:10194000C4030CCB8718594104F00F0002E00000DB
:10195000E8A6030805EBC0000368D0F804C0E01F48
:1019600000F00F0005EBC00002684068DDE904AB41
:1019700012EB0A0840EB0B00DDE906AB18EB0A029C
:1019800040EB0B00984618EB02024CEB000004F011
:101990000F0305EBC3031A605860BA184141CDE943
:1019A0000221DDE90237DDE90C10C91840EB07021E
:1019B000CDE90C121C200021DDE91223F6F772FE9E
:1019C0000746884622200021DDE91223F6F76AFE49
:1019D000424687EA000882EA010727200021DDE964
:1019E0001223F6F75FFE88EA000887EA0100DDE9C6
:1019F000021218EB010C5041DDE91272DDE91031E1
:101A00001F400A40DDE90EABDDE9121301EA0A01CD
:101A100003EA0B0887EA010382EA0802DDE91017EE
:101A200001EA0A0107EA0B074B407A401CEB03016D
:101A30005041CDE91410641C601C00F00F0005EB50
:101A4000C00108684A68CDE9060201200021DDE9ED
:101A50000623F6F727FE0746884608200021DDE921
:101A60000623F6F71FFE474088EA0101DDE906027A
:101A7000C00940EA4260474081EAD211CDE90671CF
:101A8000A01E00F00F0105EBC10001684268CDE91E
:101A9000041213200021DDE90423F6F703FE0746B4
:101AA00088463D200021DDE90423F6F7FBFD474091
:101AB00088EA0108DDE90401800940EA81604740C5
:101AC00088EA9118CDE904780E200021DDE90C2385
:101AD000F6F7E8FD0746884612200021DDE90C23D1
:101AE000F6F7E0FD424687EA000882EA010729206E
:101AF0000021DDE90C23F6F7D5FD88EA000887EA26
:101B00000102DDE9161018EB010C4241DDE90A780B
:101B1000DDE90C303B4000EA0800DDE908ABDDE917
:101B20000C712AEA07072BEA01017B4041401CEBBC
:101B300003004A416C4B03EBC40188C9C31842EB54
:101B4000070104F00F0005EBC0000768D0F804C0DF
:101B5000E01F00F00F0005EBC00002684068DDE9FF
:101B6000048B12EB080840EB0B02DDE906A018EB32
:101B70000A0842416046944617EB080240EB0C000D
:101B800004F00F0705EBC7073A6078609A184141E7
:101B9000CDE90221DDE90237DDE90E10C91840EB7D
:101BA0000702CDE90E121C200021DDE91423F6F70F
:101BB00079FD0746884622200021DDE91423F6F747
:101BC00071FD424687EA000882EA010727200021CA
:101BD000DDE91423F6F766FD88EA000887EA0102CA
:101BE000DDE9021018EB01084241DDE91230DDE9C0
:101BF000141C19400CEA000CDDE9107BDDE91430FF
